S0210000636F756E7465725F68616E645F646973635F625F626F6172642E73726563DF
S3150802000000000A20B1840208816A0208896A020885
S31508020010916A0208996A0208A16A02080185020819
S315080200200000000000000000000000000185020830
S31508020030A96A02080000000035030208E102020864
S315080200400185020801850208018502080185020860
S315080200500185020801850208018502080185020850
S315080200600185020801850208018502080185020840
S315080200700185020801850208018502080185020830
S315080200800185020801850208018502080185020820
S315080200900185020801850208018502080185020810
S315080200A00185020801850208018502080185020800
S315080200B001850208018502080185020801850208F0
S315080200C001850208018502080185020801850208E0
S315080200D0000000000185020801850208B96A0208C3
S315080200E001850208018502080185020801850208C0
S315080200F001850208018502080185020801850208B0
S31508020100018502080185020801850208018502089F
S31508020110018502080185020801850208018502088F
S315080201200185020801850208CD6A020801850208CE
S31508020130018502080185020801850208018502086F
S31508020140018502080185020801850208018502085F
S31508020150018502080185020801850208018502084F
S31508020160018502080185020801850208018502083F
S31508020170018502080185020801850208018502082F
S31508020180018502080185020801850208018502081F
S31508020190018502080185020801850208018502080F
S315080201A001850208018502080185020801850208FF
S315080201B001850208018502080185020801850208EF
S315080201C001850208018502080185020801850208DF
S315080201D001850208018502080185020801850208CF
S315080201E001850208018502080185020801850208BF
S315080201F001850208018502080185020801850208AF
S31508020200018502080185020801850208000000002E
S3150802021000000000018502080000000001850208AE
S315080202200185020801850208E16A020801850208B9
S31508020230018502080185020801850208018502086E
S3150802024001850208018502080185020800000000EE
S3150802025010B5054C237833B9044B13B10448AFF3F0
S3150802026000800123237010BDBC130020000000008B
S3150802027044EC030808B5034B1BB103490348AFF323
S31508020280008008BD00000000C013002044EC0308EB
S3150802029072B64FF0E0201749C0F8081D16480168E3
S315080202A041F00101016015481249096801604FF0E1
S315080202B0E020134941614FF0070101614FF0000147
S315080202C0C0F8181D4FF07F41C0F81C1D0D49C0F833
S315080202D0201D7047FFF7FEBF01B5BDE80140704714
S315080202E001B500F097F8BDE801407047FFF7FEBF79
S315080202F0FFF7FEBF00000208001000E08CEA0020AB
S315080203008FD003000000FF404FF000002D4A106016
S31508020310EFF3148020F0040080F3148862B64FF0DD
S3150802032080504FF0E021C1F8040DBFF34F8FBFF3A1
S315080203306F8FFEE72448254A4FF00003016891B102
S315080203400360EFF3098C2CE9F00F1EF0100F01D1B0
S315080203502CED108A1E4C4CF804EDC1F808C025682D
S315080203600DB18D61236072B61168D1B1016062B6B2
S315080203704F68174C8D6907F101074F602560D1F860
S315080203800CC08CF30B88D1F808C05CF804EB1EF09D
S31508020390100F01D1BCEC108ABCE8F00F8CF3098867
S315080203A0704772B61168016009B962B6F9E74FF08B
S315080203B000674FF0E028C8F8047D62B6D8E700BFA8
S315080203C07047000028EB002090EA002094EA0020FB
S315080203D094F00020026922F00702A2F144026FF0AB
S315080203E0430313604FF0000353609360D3601361B5
S315080203F053619361D361136253629362D362136347
S3150802040053634FF0FF339363D1634FF080731364E2
S31508020410826070472249086800F101000860214B92
S315080204201A683AB1A2F101021A601AB91E4B4FF0C4
S31508020430010018601D490868026822B11C4B4FF07A
S3150802044001021A6008E000F104001A4B1A68904289
S3150802045001D1194B18680860134B1A6812B9144966
S315080204600868C8B101B51249086808B114F04CFF0A
S315080204700D4B1A6872B114F0B9FE1048016849B9F1
S315080204800F4801680F4A13680F484FF08052994285
S3150802049000D00260BDE80140BFF34F8F70470000ED
S315080204A034EB002094F0002038EB0020C4EB002047
S315080204B0C8EB0020C0EB0020BCEB002028EB002094
S315080204C090EA002094EA002004ED00E0034613F8BF
S315080204D0012B002AFBD1181A0138704781F0004116
S315080204E002E000BF83F0004330B54FEA41044FEA09
S315080204F0430594EA050F08BF90EA020F1FBF54EAA4
S31508020500000C55EA020C7FEA645C7FEA655C00F03F
S31508020510E2804FEA5454D4EB5555B8BF6D420CDD10
S315080205202C4480EA020281EA030382EA000083EA93
S31508020530010180EA020281EA0303362D88BF30BD33
S3150802054011F0004F4FEA01314FF4801C4CEA113189
S3150802055002D0404261EB410113F0004F4FEA0333E8
S315080205604CEA133302D0524263EB430394EA050F73
S3150802057000F0A780A4F10104D5F1200E0DDB02FAE2
S315080205800EFC22FA05F2801841F1000103FA0EF276
S31508020590801843FA05F359410EE0A5F120050EF13C
S315080205A0200E012A03FA0EFC28BF4CF0020C43FA6D
S315080205B005F3C01851EBE37101F0004507D54FF07A
S315080205C0000EDCF1000C7EEB00006EEB0101B1F5CA
S315080205D0801F1BD3B1F5001F0CD349085FEA300010
S315080205E04FEA3C0C04F101044FEA445212F5800F1B
S315080205F080F09A80BCF1004F08BF5FEA500C50F1B8
S31508020600000041EB045141EA050130BD5FEA4C0C9A
S31508020610404141EB0101013C28BFB1F5801FE9D2F7
S3150802062091F0000F04BF01460020B1FA81F308BF1A
S315080206302033A3F10B03B3F120020CDA0C3208DDE6
S3150802064002F1140CC2F10C0201FA0CF021FA02F1C1
S315080206500CE002F11402D8BFC2F1200C01FA02F131
S3150802066020FA0CFCDCBF41EA0C019040E41AA2BF56
S3150802067001EB0451294330BD6FEA04041F3C1CDA1E
S315080206800C340EDC04F11404C4F1200220FA04F03E
S3150802069001FA02F340EA030021FA04F345EA0301E8
S315080206A030BDC4F10C04C4F1200220FA02F001FAAA
S315080206B004F340EA0300294630BD21FA04F029462C
S315080206C030BD94F0000F83F4801306BF81F48011C5
S315080206D00134013D4EE77FEA645C18BF7FEA655C38
S315080206E029D094EA050F08BF90EA020F05D054EA0A
S315080206F0000C04BF1946104630BD91EA030F1EBF0F
S315080207000021002030BD5FEA545C05D14000494112
S3150802071028BF41F0004130BD14F580043CBF01F505
S31508020720801130BD01F0004545F0FE4141F47001EB
S315080207304FF0000030BD7FEA645C1ABF19461046C6
S315080207407FEA655C1CBF0B46024650EA013406BFC7
S3150802075052EA033591EA030F41F4002130BD00BF86
S3150802076090F0000F04BF0021704730B54FF4806443
S3150802077004F132044FF000054FF0000150E700BFC4
S3150802078090F0000F04BF0021704730B54FF4806423
S3150802079004F1320410F0004548BF40424FF0000110
S315080207A03EE700BF42004FEAE2014FEA31014FEA53
S315080207B002701FBF12F07F4393F07F4F81F06051A2
S315080207C0704732F07F4208BF704793F07F4F04BFED
S315080207D041F40021704730B54FF4607401F00045CA
S315080207E021F000411CE700BF50EA010208BF70472A
S315080207F030B54FF000050AE050EA010208BF70471B
S3150802080030B511F0004502D5404261EB41014FF483
S31508020810806404F132045FEA915C3FF4D8AE4FF08B
S3150802082003025FEADC0C18BF03325FEADC0C18BF6E
S31508020830033202EBDC02C2F1200300FA03FC20FABF
S3150802084002F001FA03FE40EA0E0021FA02F114440C
S31508020850BDE600BF70B54FF0FF0C4CF4E06C1CEA25
S3150802086011541DBF1CEA135594EA0C0F95EA0C0F96
S3150802087000F0DEF82C4481EA030621EA4C5123EA09
S315080208804C5350EA013518BF52EA033541F4801138
S3150802089043F4801338D0A0FB02CE4FF00005E1FBEB
S315080208A002E506F00042E0FB03E54FF00006E1FB35
S315080208B003569CF0000F18BF4EF0010EA4F1FF0478
S315080208C0B6F5007F64F5407404D25FEA4E0E6D41B8
S315080208D046EB060642EAC62141EA55514FEAC520C9
S315080208E040EA5E504FEACE2EB4F1FD0C88BFBCF545
S315080208F0E06F1ED8BEF1004F08BF5FEA500E50F1F6
S31508020900000041EB045170BD06F0004646EA0101BB
S3150802091040EA020081EA0301B4EB5C04C2BFD4EBED
S315080209200C0541EA045170BD41F480114FF0000EE6
S31508020930013C00F3AB8014F1360FDEBF002001F054
S31508020940004170BDC4F10004203C35DA0C341BDCCE
S3150802095004F11404C4F1200500FA05F320FA04F0A0
S3150802096001FA05F240EA020001F0004221F00041D4
S3150802097010EBD37021FA04F642EB06015EEA430E47
S3150802098008BF20EAD37070BDC4F10C04C4F1200577
S3150802099000FA04F320FA05F001FA04F240EA02002A
S315080209A001F0004110EBD37041F100015EEA430EFB
S315080209B008BF20EAD37070BDC4F1200500FA05F21B
S315080209C04EEA020E20FA04F301FA05F243EA02039A
S315080209D021FA04F001F0004121FA04F220EA0200A9
S315080209E000EBD3705EEA430E08BF20EAD37070BDEF
S315080209F094F0000F0FD101F00046400041EB0101CF
S31508020A0011F4801F08BF013CF7D041EA060195F0B0
S31508020A10000F18BF704703F00046520043EB03036A
S31508020A2013F4801F08BF013DF7D043EA0603704757
S31508020A3094EA0C0F0CEA135518BF95EA0C0F0CD062
S31508020A4050EA410618BF52EA4306D1D181EA0301A8
S31508020A5001F000414FF0000070BD50EA410606BFA2
S31508020A601046194652EA430619D094EA0C0F02D1E7
S31508020A7050EA013613D195EA0C0F05D152EA03362C
S31508020A801CBF104619460AD181EA030101F000414A
S31508020A9041F0FE4141F470014FF0000070BD41F093
S31508020AA0FE4141F4780170BD70B54FF0FF0C4CF46D
S31508020AB0E06C1CEA11541DBF1CEA135594EA0C0F8C
S31508020AC095EA0C0F00F0A7F8A4EB050481EA030ED9
S31508020AD052EA03354FEA013100F088804FEA0333C0
S31508020AE04FF0805545EA131343EA12634FEA02228E
S31508020AF045EA111545EA10654FEA00260EF000414F
S31508020B009D4208BF964244F1FD0404F5407402D2A0
S31508020B105B084FEA3202B61A65EB03055B084FEA31
S31508020B2032024FF480104FF4002CB6EB020E75EB2E
S31508020B30030E22BFB61A754640EA0C005B084FEA56
S31508020B403202B6EB020E75EB030E22BFB61A7546D3
S31508020B5040EA5C005B084FEA3202B6EB020E75EB1E
S31508020B60030E22BFB61A754640EA9C005B084FEA96
S31508020B703202B6EB020E75EB030E22BFB61A7546A3
S31508020B8040EADC0055EA060E18D04FEA051545EA92
S31508020B9016754FEA06164FEAC30343EA52734FEA3B
S31508020BA0C2025FEA1C1CC0D111F4801F0BD141EAB4
S31508020BB000014FF000004FF0004CB6E711F4801F19
S31508020BC004BF01430020B4F1FD0C88BFBCF5E06FF9
S31508020BD03FF6AFAEB5EB030C04BFB6EB020C5FEA09
S31508020BE0500C50F1000041EB045170BD0EF0004E5E
S31508020BF04EEA113114EB5C04C2BFD4EB0C0541EA90
S31508020C00045170BD41F480114FF0000E013C90E68C
S31508020C1045EA060E8DE60CEA135594EA0C0F08BF50
S31508020C2095EA0C0F3FF43BAF94EA0C0F0AD150EA4F
S31508020C3001347FF434AF95EA0C0F7FF425AF1046E2
S31508020C4019462CE795EA0C0F06D152EA03353FF40A
S31508020C50FDAE1046194622E750EA410618BF52EA87
S31508020C6043067FF4C5AE50EA41047FF40DAF52EA5B
S31508020C7043057FF4EBAE12E74FF0FF3C06E000BFF8
S31508020C804FF0010C02E000BF4FF0010C4DF804CD05
S31508020C904FEA410C7FEA6C5C4FEA430C18BF7FEAC5
S31508020CA06C5C1BD001B050EA410C0CBF52EA430CF3
S31508020CB091EA030F02BF90EA020F0020704710F173
S31508020CC0000F91EA030F58BF994208BF90422CBF02
S31508020CD0D8176FEAE37040F0010070474FEA410CFB
S31508020CE07FEA6C5C02D150EA013C07D14FEA430C19
S31508020CF07FEA6C5CD6D152EA033CD3D05DF8040B8A
S31508020D00704700BF8446104662468C4619466346BB
S31508020D1000E000BF01B5FFF7B7FF002848BF10F192
S31508020D20000F01BD4DF808EDFFF7F4FF0CBF0120D7
S31508020D3000205DF808FB00BF4DF808EDFFF7EAFF53
S31508020D4034BF012000205DF808FB00BF4DF808ED0E
S31508020D50FFF7E0FF94BF012000205DF808FB00BF03
S31508020D604DF808EDFFF7CEFF94BF012000205DF88D
S31508020D7008FB00BF4DF808EDFFF7C4FF34BF01209A
S31508020D8000205DF808FB00BF4FEA410C7FEA6C5C65
S31508020D9002D150EA013C0AD14FEA430C7FEA6C5C65
S31508020DA002D152EA033C02D14FF0000070474FF0DD
S31508020DB0010070474FEA410212F5001215D211D509
S31508020DC06FF47873B3EB625212D94FEAC12343F038
S31508020DD0004343EA505311F0004F23FA02F018BFBA
S31508020DE0404270474FF00000704750EA013005D183
S31508020DF011F0004008BF6FF0004070474FF0000046
S31508020E00704700BF4A0011D212F5001211D20DD551
S31508020E106FF47873B3EB62520ED44FEAC12343F0F0
S31508020E20004343EA505323FA02F070474FF000009A
S31508020E30704750EA013002D14FF0FF3070474FF049
S31508020E40000070474FEA4102B2F1E04324BFB3F50E
S31508020E50001CDCF1FE5C0DD901F0004C4FEAC00221
S31508020E604CEA5070B2F1004F40EB830008BF20F005
S31508020E700100704711F0804F21D113F13872BCBFBF
S31508020E8001F00040704741F480114FEA5252C2F114
S31508020E901802C2F1200C10FA0CF320FA02F018BF5D
S31508020EA040F001004FEAC1234FEAD32303FA0CFCB0
S31508020EB040EA0C0023FA02F34FEA4303CCE77FEA3F
S31508020EC0625307D150EA01331EBF4FF0FE4040F489
S31508020ED04000704701F0004040F0FE4040F4000038
S31508020EE0704700BF53B94AB9002908BF00281CBF7A
S31508020EF04FF0FF314FF0FF3000F0B4B9ADF1080CF6
S31508020F006DE904CE00F03CF8DDF804E0DDE90223E1
S31508020F1004B0704738B50022002304460D46FFF791
S31508020F200BFF28B920462946BDE8384000F00AB822
S31508020F30204605F1004100F005F8404261EB410107
S31508020F4038BD00BFD0B500220B4B06460F46FFF749
S31508020F5081FCFFF757FF0446FFF702FC0022074B06
S31508020F60FFF778FC02460B4630463946FFF7BAFACF
S31508020F70FFF748FF2146D0BD0000F03D0000F041D2
S31508020F802DE9F04F099D0C46002B4DD18A420F469A
S31508020F9084469646B2FA82F360D94BB102FA03FE48
S31508020FA0C3F120029F4000FA03FC20FA02F217431B
S31508020FB04FEA1E461FFA8EF44FEA1C42B7FBF6F1B9
S31508020FC006FB117701FB04F042EA0742904208D970
S31508020FD01EEB020201F1FF3702D2904200F22D8186
S31508020FE03946121A1FFA8CFCB2FBF6F006FB1022DF
S31508020FF000FB04F44CEA024C644508D91EEB0C0CBF
S3150802100000F1FF3202D2644500F21A81104640EA24
S315080210100140ACEB040C002125B12CFA03F30022A3
S31508021020C5E90032BDE8F08F8B4205D90DB1C5E995
S31508021030000100210846F5E7B3FA83F100294DD1EC
S31508021040A342C0F0F280904280F0EF800646234623
S315080210500846002DE6D0C5E90063E3E7002B40F019
S31508021060A2808A1A4FEA1E471FFA8EF60121B2FBA0
S31508021070F7F407FB14204FEA1C4242EA004206FB39
S3150802108004F090420FD91EEB020204F1FF382CBF7E
S315080210904FF001094FF00009904203D9B9F1000F48
S315080210A000F0C8804446121A1FFA8CFCB2FBF7F00D
S315080210B007FB102200FB06F64CEA024C664508D9E5
S315080210C01EEB0C0C00F1FF3202D2664500F2BB8021
S315080210D01046ACEB060C40EA04409DE7C1F1200637
S315080210E08B4004FA01FE22FA06F720FA06FCF440BF
S315080210F08A401F434EEA0C0300FA01FE4FEA1748DC
S315080211004FEA13491FFA87FCB4FBF8F008FB1044B0
S3150802111049EA044400FB0CF9A1450ED93C1900F131
S31508021120FF3A2CBF4FF0010B4FF0000BA14503D934
S31508021130BBF1000F00F093805046A4EB09041FFA96
S3150802114083F9B4FBF8F308FB134403FB0CFC49EAE6
S315080211500444A44506D93C1903F1FF3801D2A44533
S315080211607AD8434643EA0040A4EB0C04A0FB029853
S315080211704445CC46434602D306D1CE4504D201386D
S31508021180B9EB020C68EB07035DB1BEEB0C0264EB2C
S31508021190030404FA06F622FA01F3CC401E43C5E913
S315080211A0006400213EE702FA03FEC3F1200104FAB5
S315080211B003F200FA03FCCC404FEA1E4720FA01F17B
S315080211C01FFA8EF6B4FBF7F00A4307FB1044110C1C
S315080211D041EA044100FB06F48C420ED91EEB0101DA
S315080211E000F1FF382CBF4FF001094FF000098C427D
S315080211F002D9B9F1000F2CD04046091B92B2B1FBB5
S31508021200F7F407FB141142EA014204FB06F1914284
S3150802121007D91EEB020204F1FF3801D2914215D812
S315080212204446521A44EA004121E7861A64EB03034C
S3150802123001200EE7023C724435E702397244D0E6D1
S31508021240F4440238E3E6F444023842E7023C7244C4
S31508021250E7E702387144D0E7023B3C4482E70238AA
S315080212603C446AE7704700BF80B586B002AF786033
S315080212700023FB60342300934FF4E8430B4A0C49DE
S315080212800C4814F0EBFA0346002B0AD1094BBB6053
S31508021290B86801F02FF8F860FB68002B01D000BF90
S315080212A0FDE700BF1037BD4680BD00BFD81300203A
S315080212B060EC0308D887002080B586B000AF786056
S315080212C000237B610023FB607B683B61FF2017F0EC
S315080212D0C3FE00237B6112E03B691B68FB607B69E6
S315080212E003F1016303F57C23FA681146184617F0E1
S315080212F09CFE3B6904333B617B6904337B617B69F2
S31508021300132BE9D9012318461837BD4680BD80B488
S3150802131083B000AF78607B685B6818460C37BD46B9
S315080213205DF8047B704780B483B000AF786039609B
S315080213307B683A685A6000BF0C37BD465DF8047B85
S31508021340704780B483B000AF78607B681B7A184612
S315080213500C37BD465DF8047B704780B483B000AF96
S3150802136078600B46FB707B68FA781A7200BF0C37F6
S31508021370BD465DF8047B704780B483B000AF7860E1
S315080213800B46FB70FB78042B04D8FB787A68134467
S315080213909B7A00E0002318460C37BD465DF8047BAD
S315080213A0704780B483B000AF78600B46FB70134673
S315080213B0BB70FB78042B0DD8BB78002B05D0FB78C5
S315080213C07A68134401229A7204E0FB787A68134415
S315080213D000229A7200BF0C37BD465DF8047B70473F
S315080213E080B483B000AF78607B68DB7B18460C3725
S315080213F0BD465DF8047B704780B483B000AF786061
S315080214007B681B7C18460C37BD465DF8047B704723
S3150802141080B483B000AF78600B46FB707B68FA78BD
S315080214201A7400BF0C37BD465DF8047B704700008E
S3150802143080B483B000AF0346FB71044AFB7913708C
S3150802144000BF0C37BD465DF8047B7047ED9D002052
S3150802145080B586B000AFF8600B467A60FB7200234F
S31508021460FB752D4806F00EFE0023FB754CE0FB7D4E
S315080214702A4A4FF48E7101FB03F313441B78012B9E
S315080214803FD1FB7D4FF48E7202FB03F3234A1344CA
S3150802149002331946224806F0F5FD224806F0F2FD07
S315080214A0FB7D4FF48E7202FB03F318331B4A134477
S315080214B0043319461A4806F0E5FD1B4806F0E2FD14
S315080214C0FB7D164A4FF48E7101FB03F313449C33DA
S315080214D01B782D2B12D0154806F0D4FDFB7D4FF450
S315080214E08E7202FB03F398330C4A134404331946EB
S315080214F00B4806F0C7FD0C4806F0C4FD0A4806F07C
S31508021500C1FDFB7D0133FB75FB7D0F2BAFD900BFF8
S3150802151000BF1837BD4680BD74EC030800000020E2
S315080215209CEC0308A0EC0308A4EC0308A8EC030847
S3150802153080B584B000AFF8600B467A60FB7205F09E
S3150802154069FB0346184605F0C7FB00BF1037BD46C0
S3150802155080BD000080B586B000AFF8600B467A60A1
S31508021560FB7200237B617B6803F5007303224C49F7
S3150802157018461AF0ADF80346002B22D17B6803F50C
S3150802158000731846FEF7A2FF0346032B19D17B68A0
S3150802159003F58063184618F091FF78617B69002B82
S315080215A007D005F037FB03460121184605F08BFCE8
S315080215B071E005F02FFB03460121184605F0A0FC51
S315080215C069E07B6803F500730522364918461AF066
S315080215D07FF80346002B22D17B6803F50073184671
S315080215E0FEF774FF0346052B19D17B6803F5806362
S315080215F0184618F063FF78617B69002B07D005F05F
S3150802160009FB03460421184605F05DFC43E005F094
S3150802161001FB03460421184605F072FC3BE07B6891
S3150802162003F500730322204918461AF051F80346B7
S31508021630002B30D17B6803F500731846FEF746FF88
S315080216400346032B27D17B6803F58063184618F0F7
S3150802165035FF78617B69002B0ED005F0DBFA03466D
S315080216600121184605F02FFC05F0D4FA0346042199
S31508021670184605F028FC0EE005F0CCFA03460121CF
S31508021680184605F03DFC05F0C5FA0346042118463E
S3150802169005F036FCFFE700BF1837BD4680BD00BF20
S315080216A0B4EC0308B8EC0308C0EC030880B586B0AE
S315080216B000AFF8600B467A60FB7200237B61BF4A73
S315080216C007F110031268114619800233120C1A70B8
S315080216D005F0A0FA0346184605F056FCFB7A012BDC
S315080216E040F254827B6803F500730722B449184610
S315080216F019F0EEFF0346002B13D17B6803F500733E
S315080217001846FEF7E3FE0346072B0AD1AD4806F054
S31508021710B9FC03F0A5FB03460121184603F0E9FBD1
S3150802172038E27B6803F500730522A749184619F0C3
S31508021730CFFF0346002B4FD17B6803F5007318468B
S31508021740FEF7C4FE0346052B46D17B6803F5806384
S31508021750184618F0B3FE786179699C4806F092FC3F
S315080217607B69013B042B35D801A252F823F000BF4E
S315080217708517020895170208A5170208B517020861
S31508021780C517020817F054FB01230122652117F039
S3150802179099FB20E017F04CFB01230422652117F080
S315080217A091FB18E017F044FB01230322652117F089
S315080217B089FB10E017F03CFB01230A22652117F08A
S315080217C081FB08E017F034FB01231022652117F08C
S315080217D079FB00E000BFDDE17B6803F500730C22AC
S315080217E07B49184619F074FF0346002B1DD17B6806
S315080217F003F500731846FEF769FE03460C2B14D14F
S315080218007B6803F58063184618F058FE7861796993
S31508021810704806F037FC05F0FDF902467B69DBB233
S315080218201946104605F0E4FDB4E17B6803F500733A
S3150802183008226949184619F04BFF0346002B13D1B3
S315080218407B6803F500731846FEF740FE0346082B2D
S315080218500AD1624806F016FC03F002FB034602218F
S31508021860184603F046FB95E17B6803F500730B22E5
S315080218705B49184619F02CFF0346002B0CD17B68EE
S3150802188003F500731846FEF721FE03460B2B03D118
S31508021890544806F0F7FB7DE17B6803F500730C22DA
S315080218A05149184619F014FF0346002B0CD17B68E0
S315080218B003F500731846FEF709FE03460C2B03D1FF
S315080218C04A4806F0DFFB65E17B6803F500730422EC
S315080218D04749184619F0FCFE0346002B10D17B68CF
S315080218E003F500731846FEF7F1FD0346042B07D1EC
S315080218F0404806F0C7FB01F0ADFF02F041F849E1A6
S315080219007B6803F5007307223B49184619F0E0FE87
S315080219100346002B13D17B6803F500731846FEF7BE
S31508021920D5FD0346072B0AD1344806F0ABFB03F074
S3150802193097FA03460521184603F0DBFA2AE17B6883
S3150802194003F5007306222E49184619F0C1FE03460E
S31508021950002B13D17B6803F500731846FEF7B6FD14
S315080219600346062B0AD1274806F08CFB03F078FAC1
S3150802197003460621184603F0BCFA0BE17B6803F519
S31508021980007306222049184619F0A2FE0346002BC8
S315080219903ED17B6803F500731846FEF797FD0346AA
S315080219A0062B35D1194806F06DFB03F059FA0346A2
S315080219B00721184603F09DFAECE000BF28EF03085A
S315080219C0C4EC0308CCEC0308E8EC0308F0EC0308C3
S315080219D008ED030818ED030840ED03084CED03086B
S315080219E06CED030878ED030894ED0308A4ED0308EB
S315080219F0C0ED0308C8ED0308D8ED0308E0ED0308B7
S31508021A00F8ED030800EE030820EE030828EE0308A3
S31508021A107B6803F5007304226049184619F058FEDC
S31508021A200346002B13D17B6803F500731846FEF7AD
S31508021A304DFD0346042B0AD1594806F023FB03F051
S31508021A400FFA03460321184603F053FAA2E07B680D
S31508021A5003F5007307225349184619F039FE03465F
S31508021A60002B13D17B6803F500731846FEF72EFD8B
S31508021A700346072B0AD14C4806F004FB03F0F0F99B
S31508021A8003460421184603F034FA83E07B6803F51B
S31508021A90007308224549184619F01AFE0346002B18
S31508021AA013D17B6803F500731846FEF70FFD03464C
S31508021AB0082B0AD13E4806F0E5FA03F0D1F90346A7
S31508021AC00121184603F0FAF964E07B6803F500730E
S31508021AD007223849184619F0FBFD0346002B13D195
S31508021AE07B6803F500731846FEF7F0FC0346072BDE
S31508021AF00AD1314806F0C6FA03F0B2F903460021C4
S31508021B00184603F0DBF945E07B6803F50073052206
S31508021B102A49184619F0DCFD0346002B13D17B68C7
S31508021B2003F500731846FEF7D1FC0346052B0AD1C6
S31508021B30234806F0A7FA03F093F903460521184647
S31508021B4003F0BCF926E07B6803F5007308221D49F9
S31508021B50184619F0BDFD0346002B13D17B6803F521
S31508021B6000731846FEF7B2FC0346082B0AD116483C
S31508021B7006F088FA07F1100303221946134817F0EC
S31508021B80CBFF07E0124806F07DFA03E0104806F09C
S31508021B9079FA00BF1837BD4680BD00BF3CEE030880
S31508021BA044EE03085CEE030864EE030880EE0308BD
S31508021BB08CEE0308A4EE0308ACEE0308CCEE030889
S31508021BC0D4EE0308ECEE0308F8EE03080600080054
S31508021BD014EF03082DE9F0418EB002AFF8600B4608
S31508021BE07A60FB7205F016F80346184605F05DF8AA
S31508021BF0F8620023BB6200237B6200233B62002358
S31508021C00FB610023BB6100237B617B6803F50073DC
S31508021C1004226C49184619F05BFD0346002B0FD1C6
S31508021C207B6803F500731846FEF750FC0346042B3F
S31508021C3006D1654806F026FAF86AFFF73DFBE0E1A9
S31508021C407B6803F5007304226049184619F040FDC3
S31508021C500346002B4ED17B6803F500731846FEF740
S31508021C6035FC0346042B45D1F86AFFF750FB0346B9
S31508021C701946574806F006FAF86AFFF762FB034662
S31508021C801946544806F0FEF90021F86AFFF774FB74
S31508021C9003461D460121F86AFFF76EFB03461E46F8
S31508021CA00221F86AFFF768FB034698460321F86A99
S31508021CB0FFF762FB03461C460421F86AFFF75CFB42
S31508021CC0034601930094434632462946424806F0A3
S31508021CD0D9F9F86AFFF784FB034619463F4806F026
S31508021CE0D1F9F86AFFF788FB034619463C4806F01D
S31508021CF0C9F986E17B6803F500731122394918464A
S31508021D0019F0E6FC0346002B20D17B6803F5007325
S31508021D101846FEF7DBFB0346112B17D17B6803F542
S31508021D208063184618F0CAFBB862B96A2E4806F0EC
S31508021D30A9F9BB6A002B05DDBB6A1946F86AFFF7E3
S31508021D40F2FA5EE1294806F09DF95AE17B6803F545
S31508021D5000730E222649184619F0BAFC0346002BD0
S31508021D604CD17B6803F500731846FEF7AFFB0346B2
S31508021D700E2B43D17B6803F58063184618F09EFB49
S31508021D80B862BB6A002B0AD1B96A1A4806F07AF910
S31508021D90BB6ADBB21946F86AFFF7DFFA31E1BB6ABA
S31508021DA0012B0AD1B96A144806F06CF9BB6ADBB290
S31508021DB01946F86AFFF7D1FA23E10C4806F062F9E8
S31508021DC01FE100BF2CEF030834EF030848EF0308AE
S31508021DD050EF03087CEF0308B8EF0308E8EF03089F
S31508021DE018F0030860F0030874F0030814EF0308F8
S31508021DF0A4F00308B4F00308ECF003087B6803F5C3
S31508021E0000730A228149184619F062FC0346002B20
S31508021E1040F098807B6803F500731846FEF756FB78
S31508021E2003460A2B40F08E807B6803F580631846CA
S31508021E3018F044FB78627B6803F5C063184618F00D
S31508021E403DFB38627B6803F50063184618F036FBDB
S31508021E50F8617B6803F52063184618F02FFBB86112
S31508021E607B6803F54063184618F028FB78617B6A9D
S31508021E70002B02D07B6A012B60D13B6A002B02D071
S31508021E803B6A012B5AD1FB69002B02D0FB69012B55
S31508021E9054D1BB69002B02D0BB69012B4ED17B6999
S31508021EA0002B02D07B69012B48D17B6ADBB21A462A
S31508021EB00021F86AFFF775FA3B6ADBB21A46012176
S31508021EC0F86AFFF76EFAFB69DBB21A460221F86A6C
S31508021ED0FFF767FABB69DBB21A460321F86AFFF70E
S31508021EE060FA7B69DBB21A460421F86AFFF759FAE7
S31508021EF00021F86AFFF740FA03461D460121F86AEF
S31508021F00FFF73AFA03461E460221F86AFFF734FA41
S31508021F10034698460321F86AFFF72EFA03461C463B
S31508021F200421F86AFFF728FA034601930094434608
S31508021F3032462946364806F0A5F862E0354806F0E4
S31508021F40A1F85EE07B6803F500730722324918465A
S31508021F5019F0BEFB0346002B27D17B6803F50073F5
S31508021F601846FEF7B3FA0346072B1ED17B6803F51C
S31508021F708063184618F0A2FAB862BB6A002B02D030
S31508021F80BB6A002B0DDDBB6A032B0ADCB96A234840
S31508021F9006F078F8BB6ADBB21946F86AFFF738FA30
S31508021FA02FE01F4806F06EF82BE07B6803F50073F6
S31508021FB01A781C4B1B78D31A002B1ED17B6803F5A3
S31508021FC000731846FEF782FA0346012B15D1164806
S31508021FD006F058F8154806F055F8154806F052F86E
S31508021FE0144806F04FF8144806F04CF8134806F061
S31508021FF049F8134806F046F803E0064806F042F8A0
S3150802200000BF3037BD46BDE8F08100BF24F10308A2
S3150802201030F1030814EF03085CF1030864F10308BE
S3150802202088F10308A8F10308ACF10308C8F103080C
S31508022030E4F1030804F203085CF20308BCF203089D
S3150802204010F3030890B585B000AF78600023BB7320
S315080220500023FB734FF4A0520021204819F030FBED
S3150802206007F10E030A221D49786814F0B7F80346E9
S31508022070012B2ED10023FB7328E0FB7B4FF48E72D3
S3150802208002FB03F3164A13449C1C1448FEF71EFA75
S3150802209003461A461149204619F01AFB0346002B35
S315080220A011D1FB7B0E4A4FF48E7101FB03F31344E5
S315080220B018331B68B97B094A00209847094805F076
S315080220C0E1FF012306E0FB7B0133FB73FB7B0F2B4E
S315080220D0D3D9002318461437BD4690BD0C88002074
S315080220E000000020A4EC030880B582B000AF0346C6
S315080220F0FB71FB790D2B24D14F4B00221A704F48E6
S3150802210005F0C0FF4E4B1B78002B16D04D48FFF743
S3150802211099FF0346012B08D1F02200214A4819F0FB
S31508022120CFFA4849484819F06CFB454B00221A7009
S31508022130F0220021434819F0C3FA444805F0A2FFE9
S3150802214076E0FB790A2B03D13B4B00221A706FE02B
S31508022150FB791B2B03D1384B01221A7068E0FB79F5
S315080221605B2B07D1344B1B78012B03D1324B02224E
S315080221701A705DE0FB79412B1FD12F4B1B78022B7E
S315080221801BD12D4B00221A702D4B1B78002B4FD1D9
S315080221902D492F4805F076FF2B48FEF797F9034697
S315080221A0DAB2274B1A70F0220021264819F088FA6B
S315080221B02549244819F025FB3AE0FB79082B02D079
S315080221C0FB797F2B16D11C4B00221A701C4B1B78ED
S315080221D0002B2DD01A4B1B78013BDAB2184B1A701A
S315080221E0174B1B781A46174B00219954194805F0C4
S315080221F049FF1DE0124B1B785A1CD1B2104A1170C6
S315080222001946104AFB7953540D4B1A78124BA3FB05
S315080222100213D9090B461B015B1A1B01D31ADAB240
S31508022220074B1A70FB7919460C4805F02BFFFFE796
S3150802223000BF0837BD4680BDEE9D0020A4EC03080A
S31508022240EC9D0020FC9C00200C9C002064F30308F3
S315080222509CEC030868F30308898888886CF30308EA
S3150802226080B500AF1C2301221449154813F096FBCA
S315080222701C2301221349144813F090FB1C23012244
S315080222801249134813F08AFB1C23012211491248EA
S3150802229013F084FB1C2301221049114813F07EFB1C
S315080222A01C2301220F49104813F078FB1C23012234
S315080222B00E490F4813F072FB00BF80BD78F303087E
S315080222C0B0A000208CF30308CCA00020B0F30308CA
S315080222D0E8A00020C8F3030804A10020E0F30308DD
S315080222E020A10020F4F303083CA1002010F40308FF
S315080222F058A1002080B58EB008AF786000237B61B4
S315080223007B683B6107F10C0100234FF400723869C0
S3150802231013F030FA0346002B01D0022348E0FB688B
S31508022320B022069201220592002204920A22039200
S315080223300A2202924FF400720192009300231E4A67
S315080223401E491F4813F020FC0346002B01D00E231A
S315080223502EE0062210211B4805F06AFF786805F070
S31508022360C3FC0346002B03D0174805F08BFE02E098
S31508022370164805F087FE786805F02CFD0346002B03
S3150802238003D0134805F07EFE02E0124805F07AFEF5
S31508022390786805F04DFC0346002B03D00E4805F07D
S315080223A071FE02E00D4805F06DFEFFF759FF7B69E5
S315080223B018461837BD4680BDE123020828F40308EB
S315080223C0F09D002038F403084CF4030868F4030867
S315080223D084F40308A0F40308BCF40308DCF4030835
S315080223E080B584B000AF78607B68BB600023FB735E
S315080223F0174805F047FE174805F044FE164B1B78AA
S315080224000133DAB2144B1A70134B1B78092B15D900
S31508022410114B00221A7005F0E3FF01210F4807F05D
S3150802242097FEFB7B032B03D1FB7B0133FB7305E092
S31508022430FB7B032B02D8FB7B0133FB73BB68DBB246
S31508022440184605F09FFF642012F0FEFBD6E700BF90
S31508022450FCF4030824F5030874A1002000140242C0
S3150802246080B500AF12F090F800BF80BD80B400AF0F
S31508022470034B1B681846BD465DF8047B704700BFD0
S3150802248078A1002080B500AF4FF400620E490F48CC
S3150802249013F00EFF4FF400620D490E4813F008FFC1
S315080224A04FF400720C490D4813F002FF4FF4006214
S315080224B00B490C4813F0FCFE4FF400620A490B481C
S315080224C013F0F6FE00BF80BD8CA100207CA100207F
S315080224D09CA900208CA90020D0B10020C0B1002000
S315080224E010B40020D0B3002050BC002010BC00203D
S315080224F084B0B0B400AF07F10C0484E80F00074BB0
S315080225001D4607F10C040FCC0FC50FCC0FC5236867
S315080225102B6000BFBD46B0BC04B070479CB100201A
S3150802252080B586B000AF78600B467B800023FB75CA
S3150802253000233B610023FB600023BB6000F09CFC88
S315080225400346002B0BD0444BD3F844323B61424B33
S31508022550D3F8843AFB607B681B68BB600AE03E4B93
S31508022560D3F844323B613C4BD3F8843AFB607B6830
S315080225701B68BB603A69BB689A4227D1364B93F807
S315080225806832002B0AD1344BD3F850227B88134485
S31508022590314AC2F850320123FB7558E02E4BB3F884
S315080225A06C321A467B881344B3F5006F0BDA2A4B52
S315080225B0B3F86C227B8813449AB2274BA3F86C2291
S315080225C00123FB7543E00023FB7540E0FA68BB680C
S315080225D09A4227D1204B93F8A83A002B0AD11E4BD0
S315080225E0D3F850227B8813441B4AC2F8503202237E
S315080225F0FB752CE0184BB3F8AC3A1A467B881344A1
S31508022600B3F5006F0BDA144BB3F8AC2A7B88134484
S315080226109AB2114BA3F8AC2A0223FB7517E00023E2
S31508022620FB7514E03B69002B07D1242279680B4815
S3150802263019F0FDF80123FB7509E0FB68002B06D1AA
S3150802264024227968064819F0F2F80223FB75FB7D05
S3150802265018461837BD4680BD9CB10020E0B300205D
S3150802266020BC002080B584B000AF03463960FB71F8
S315080226701346BB800023FB81FB79012B18D100236B
S31508022680FB8110E0FB893A6813440122194618486F
S3150802269013F0B4FE0346002B02D1164805F0F2FCED
S315080226A0FB890133FB81FA89BB889A42EAD31AE08D
S315080226B0FB79022B17D10023FB8110E0FB893A68CC
S315080226C01344012219460C4813F098FE0346002BC0
S315080226D002D10A4805F0D6FCFB890133FB81FA8947
S315080226E0BB889A42EAD300BF1037BD4680BD00BFF9
S315080226F0D0B300205CF5030810BC002080F503085F
S3150802270080B582B000AF0346FB71FB1D0122194654
S31508022710074813F073FE0346002B04D1FB791946CA
S31508022720044805F0AFFC00BF0837BD4680BD00BFB0
S31508022730C0B10020A4F50308F0B5ABB008AFF86144
S31508022740B9617A610023C7F88430F86906F029FB73
S31508022750C7F880000023C7F8843051E0D7F88430E0
S315080227605A1CC7F88420B3F5FA7F49D907F15003F2
S315080227701946F86906F048FC3B6D3B617A6DFA60CA
S31508022780B86DB860FB6D3A6E796EB86EFC6E7C6099
S315080227903D6F7E6FBC6F0794069605957C68049418
S315080227A00390029101920093BB68FA68396931482D
S315080227B005F068FC7B6E002B07D0FB691B689A69DB
S315080227C0FB691B6822F001029A61F86906F0E9FAC8
S315080227D0C7F88000D7F88010F86906F0EEFA0023E9
S315080227E0C7F8843004F016FA03460121184604F0A5
S315080227F04DFB0346002B0BD01F4805F043FC07E0B0
S315080228000721F86906F050FC0346002BA6D100E022
S3150802281000BF7A69B969F86906F07FFAF86900F0C3
S31508022820A5FA0346FB67FB6F002B1ED007F12003B0
S3150802283030220021184618F043FFF86900F05CFAC6
S3150802284003460E4A1360F86900F071FA03460B4A0A
S3150802285053600A4B1A68094B5B6807F1200008495E
S3150802286018F09AFEF86F00F0D5FA00BF8C37BD460D
S31508022870F0BD00BFCCF5030810F6030850C40020CB
S3150802288034F5030880B592B000AF3B4640220021DA
S31508022890184618F015FF0023A7F8423000237B6478
S315080228A09C4813F08FFD034683F00103DBB2002B2D
S315080228B000F0C480984B93F86832002B50D1964B9F
S315080228C0D3F850329AB2944BA3F86C22924B0F2249
S315080228D0C3F8502210233B703B785AB28E4BB3F89A
S315080228E06C321B0A9BB25BB203F00F035BB2134353
S315080228F05BB2DBB23B70884BB3F86C32DBB27B70EF
S315080229003B4602333E221946824813F0B2FD03467D
S31508022910002B00F0FC80FFF7A9FD3B461A467F49CB
S31508022920FFF70AFF7C4BB3F86C323E3B9AB27A4BFE
S31508022930A3F86C22784BB3F86A3201339AB2764B13
S31508022940A3F86A22744B012283F86822724BFF228B
S3150802295083F86E22704B4FF4FA62C3F87022D6E0FF
S315080229606D4B93F86E32002B05D06B4B93F86E3293
S31508022970012B40F0CC80684BB3F86C323E2B02D95F
S3150802298040237B6404E0644BB3F86C3201337B6406
S3150802299020233B703B785AB25F4BB3F86A325BB27C
S315080229A003F00F035BB213435BB2DBB23B707B6C83
S315080229B05A1E3B4601331946564813F05AFD03463A
S315080229C0002B00F0A4807B6C9BB2184600F084FAB8
S315080229D00346514AC2F85032FFF748FD3B461A46AB
S315080229E04E49FFF7A9FE4C4BB3F86C227B6C9BB29F
S315080229F0D31A9BB201339AB2474BA3F86C22464BC1
S31508022A00B3F86A3201339AB2434BA3F86A22424BAD
S31508022A10B3F86C32002B7AD1242200213F4818F0F1
S31508022A204FFE3D4B002283F868223B4B0022A3F857
S31508022A306A22394BFF2283F86E2268E0384813F07F
S31508022A40C1FC034683F00103DBB2002B5FD03B4691
S31508022A5001221946324813F00CFD0346002B53D0C7
S31508022A603B781B09DBB2032B14D13B460133022206
S31508022A7019462B4813F0FDFC0346002B47D0264B7C
S31508022A800322DA60FFF7F2FC3B461A462249FFF7B1
S31508022A9053FE3CE03B781B09DBB2002B37D13B46A1
S31508022AA00133012219461E4813F0E3FC0346002BA4
S31508022AB02CD03B781B029BB203F47063A7F8423012
S31508022AC07B781A46B7F842301343A7F84230B7F86C
S31508022AD042203B4602331946114813F0CAFC034604
S31508022AE0002B14D0B7F8423002339BB2184600F0D6
S31508022AF0F3F90346084AD360FFF7B8FC3B461A4681
S31508022B000549FFF719FE02E000BF00E000BF48379B
S31508022B10BD4680BDD0B300209CB10020E0B30020A2
S31508022B20C0B1002080B59AB000AF3B4668220021AA
S31508022B30184618F0C5FD0E4813F044FC034683F008
S31508022B400103DBB2002B0ED004E03B46682118468F
S31508022B5000F010F83B4668221946054813F089FC2E
S31508022B600346002BF1D100BF6837BD4680BD00BFC2
S31508022B708CA9002080B582B000AF78600B467B80B6
S31508022B80786800F07FFC00BF0837BD4680BD0000AC
S31508022B9080B500AF194B93F86832002B2BD0174B30
S31508022BA093F86E32FF2B26D1144BD3F87032002BD2
S31508022BB007D0124BD3F87032013B104AC2F8703272
S31508022BC019E0242200210E4818F07AFD4FF400621B
S31508022BD00C490D4813F06CFB084B002283F8682257
S31508022BE0064B0022A3F86A22044BFF2283F86E22C0
S31508022BF0064805F047FA00BF80BD00BF9CB1002019
S31508022C00E0B3002010B40020D0B3002034F6030845
S31508022C1080B582B000AF78600B467B80786800F09A
S31508022C2057FB00BF0837BD4680BD000080B582B09D
S31508022C3000AF78600B467B807B881A46796806481F
S31508022C4013F0DCFB0346002B02D1044805F01AFAFE
S31508022C5000BF0837BD4680BD7CA1002048F60308A0
S31508022C6080B59AB000AF3B4668220021184618F094
S31508022C7027FD0E4813F0A6FB034683F00103DBB2D9
S31508022C80002B0ED004E03B4668211846FFF7C0FF2A
S31508022C903B4668221946054813F0EBFB0346002B10
S31508022CA0F1D100BF6837BD4680BD00BF7CA10020B8
S31508022CB080B582B000AF78600B4A7B681360FFF775
S31508022CC0E1FB24220021094818F0FAFC24220021FB
S31508022CD0074818F0F5FC24220021064818F0F0FCF3
S31508022CE000BF0837BD4680BD78A100209CB10020F0
S31508022CF0E0B3002020BC002080B485B000AF786025
S31508022D007B681B681B6CBB600023FB60BB68DBB27D
S31508022D10002B05D0BB68DBB2FB60FB68DBB2FB604D
S31508022D20FB6818461437BD465DF8047B704780B4C5
S31508022D3085B000AF78607B681B681B6CBB6000239C
S31508022D40FB60BB6803F4FE43002B07D0BB6803F4A1
S31508022D50FE43FB60FB681B0ADBB2FB60FB68184696
S31508022D601437BD465DF8047B7047000080B485B011
S31508022D7000AF78607B681B685B6CBB600023FB60F6
S31508022D80BB6803F00703002B3BD0BB6803F00703BD
S31508022D90013B052B2CD801A252F823F0B52D0208C7
S31508022DA0BF2D0208C92D0208D32D0208DD2D0208FF
S31508022DB0E72D0208FB6843F00103FB6019E0FB6894
S31508022DC043F00203FB6014E0FB6843F00303FB6075
S31508022DD00FE0FB6843F00403FB600AE0FB6843F07C
S31508022DE00503FB6005E0FB6843F00603FB6000E0B1
S31508022DF000BF7B681B685A6C7B681B6822F0070257
S31508022E005A64FB68DBB218461437BD465DF8047B84
S31508022E10704700BF80B483B000AF78607B68013B1F
S31508022E20052B10D801A252F823F000BF452E02083E
S31508022E30452E0208452E0208452E0208452E02088E
S31508022E40452E020800BF00BF0C37BD465DF8047B5D
S31508022E50704700BF80B483B000AF0346FB71054AD2
S31508022E60FB791370012318460C37BD465DF8047BBF
S31508022E70704700BFC011002080B400AF034B1B7817
S31508022E801846BD465DF8047B704700BFC011002096
S31508022E9080B500AFFFF7F0FF0346002B02D04FF4D0
S31508022EA0807301E04FF48073184680BD80B400AF8A
S31508022EB04FF480231846BD465DF8047B704780B5FB
S31508022EC000AFFFF7D9FF0346002B02D04FF48573F4
S31508022ED000E00023184680BD80B483B000AF0346E5
S31508022EE0FB80FB88002B01D1002346E0FB88012BDF
S31508022EF001D1012341E0FB88022B01D102233CE0E8
S31508022F00FB88032B01D1032337E0FB88042B01D16D
S31508022F10042332E0FB88052B01D105232DE0FB882B
S31508022F20062B01D1062328E0FB88072B01D10723AC
S31508022F3023E0FB88082B01D108231EE0FB880C2B13
S31508022F4001D8092319E0FB88102B01D80A2314E0BB
S31508022F50FB88142B01D80B230FE0FB88182B01D80A
S31508022F600C230AE0FB88202B01D80D2305E0FB88F9
S31508022F70302B01D80E2300E00F2318460C37BD4626
S31508022F805DF8047B704780B483B000AF78607B68D5
S31508022F90002B01D1002346E07B68012B01D10123D6
S31508022FA041E07B68022B01D102233CE07B68032BBC
S31508022FB001D1032337E07B68042B01D1042332E0D5
S31508022FC07B68052B01D105232DE07B68062B01D1F1
S31508022FD0062328E07B68072B01D1072323E07B68B9
S31508022FE0082B01D108231EE07B68092B01D80C2384
S31508022FF019E07B680A2B01D8102314E07B680B2B97
S3150802300001D814230FE07B680C2B01D818230AE099
S315080230107B680D2B01D8202305E07B680E2B01D88F
S31508023020302300E0402318460C37BD465DF8047B82
S315080230307047B0B5A4B006AFF860B9601346FB8016
S315080230400023A7F87630FB683B65FFF715FF0346B2
S31508023050002B03D04FF080437B6501E000237B659C
S315080230600023BB65FB8802339BB21846FFF734FF81
S315080230700346FB6500233B664FF480137B664FF4D9
S315080230800013BB660023FB6600233B6700233B74E1
S315080230903B7C5AB2FB881B0A9BB25BB203F00F0356
S315080230A05BB213435BB2DBB23B74FB88DBB27B7465
S315080230B00223A7F8763010E0B7F87630023BBA68F2
S315080230C01A44B7F87630127878333B4403F8682CFA
S315080230D0B7F876300133A7F87630B7F87620FB884A
S315080230E001339A42E8DD0023A7F876300DE0B7F8F7
S315080230F0763078333B4413F8683C1846FFF700FBF2
S31508023100B7F876300133A7F87630B7F87620FB8819
S3150802311001339A42EBDD6D4607F160040FCC0FC509
S3150802312023682B6007F150030FCBFFF7E1F900BFC5
S315080231307837BD46B0BD80B58EB000AFF860B960CD
S315080231401346FB80002387F83730FB683B61FFF79D
S3150802315093FE0346002B03D04FF080437B6101E0C8
S3150802316000237B610023BB61FB88FB6100233B6272
S315080231704FF480137B624FF40013BB620023FB6299
S3150802318000233B63FA8807F1100311461846FFF736
S31508023190C7F9034687F8373097F83730002B06D039
S315080231A0FA8897F83730B9681846FFF75BFA00BF0E
S315080231B03837BD4680BDB0B5A2B006AF78600846BE
S315080231C011461A460346FB700B46BB7013467B70C4
S315080231D0002387F86F307B68BB64FFF74DFE034612
S315080231E0002B03D04FF08043FB6401E00023FB640D
S315080231F000233B6503237B650023BB654FF48013DD
S31508023200FB654FF400133B6600237B660023BB660F
S3150802321030233B723B7A5AB297F9033003F00F0315
S315080232205BB213435BB2DBB23B72BB787B727B78D1
S31508023230BB72002387F86F300DE097F86F30703352
S315080232403B4413F8683C1846FFF75AFA97F86F306A
S31508023250013387F86F3097F86F30022BEDD96D4638
S3150802326007F158040FCC0FC523682B6007F14803F2
S315080232700FCBFFF73DF900BF7037BD46B0BD80B52D
S3150802328082B000AF78600023002200217868FFF739
S3150802329092FF00BF0837BD4680BD80B584B000AF37
S315080232A0F860B9601346FB80FB883E2B06D8FB887C
S315080232B01A46B968F868FFF7BCFE05E0FB881A46A5
S315080232C0B968F868FFF737FF00BF1037BD4680BDFB
S315080232D080B588B000AF7860FF23FB7600237B6158
S315080232E00023FB6100237B827B68FB60FB6893F803
S315080232F028301B09FB76FB681B687B61FFF7D6FD46
S3150802330002467B69934202D1FFF7D9FDF861FB7E3B
S31508023310032B00F2A78001A252F823F02D330208EC
S315080233206F330208B933020807340208FB6893F8B8
S31508023330283003F00F039AB24C4B1A804B4B1B886A
S315080233401B029AB2494B1A80FB6893F829301A462F
S31508023350464B1B8813439AB2444B1A80FB682A339E
S31508023360424A12881146184600F010FF7AE0FB68B6
S3150802337093F8283003F00F039AB23C4B1A803B4B62
S315080233801B881B029AB2394B1A80FB6893F82930BC
S315080233901A46364B1B8813439AB2344B1A80344B5F
S315080233A001221A70FB682A333E21184600F0EEFE07
S315080233B0F869FFF764FF55E02D4B1B781A46FB6840
S315080233C093F8283003F00F039A4248D1FB68DB686A
S315080233D01846FFF7D8FD0346013B7B82FB68293373
S315080233E07A8A1146184600F0D1FE214B1B78013322
S315080233F0DAB21F4B1A701E4B1B780F2B2FD91C4B98
S3150802340000221A702BE01B4BD3F84432FA699A420F
S315080234100FD1FB6893F8283003F00F03DAB2154B85
S3150802342083F86E22FB6893F82920124B83F86F22E1
S3150802343017E0104BD3F8843AFA699A4211D1FB681D
S3150802344093F8283003F00F03DAB20A4B83F8AE2A50
S31508023450FB6893F82920074B83F8AF2A01E000BFDF
S3150802346000E000BF00BF2037BD4680BD68C400200B
S315080234706AC400209CB1002080B500AF16F0AEFAEF
S3150802348000BF80BD80B584B000AF78607B68FB6002
S31508023490FFF7F2FC0346002B0AD0FB681B68B3F55C
S315080234A0806F10D1FB6893F82830002B0BD10AE005
S315080234B0FB681B68B3F5806F05D1FB6893F8283063
S315080234C0002B00D100BF00BF1037BD4680BD0000EB
S315080234D080B500AF174B1B78DBB2002B27D1154BF3
S315080234E001221A7022220221134818F0E9F8124B17
S315080234F001221A77012200210F4800F081F80122E1
S3150802350001210D4800F07CF8012202210A4800F048
S3150802351077F801220321084800F072F801220421F3
S31508023520054800F06DF80121034800F07DF8024BCA
S31508023530184680BD6EC4002070C4002080B483B0D3
S3150802354000AF78600B46FB70FB787A6813445B79A8
S31508023550012B01D1012308E0FB787A6813445B79D1
S31508023560022B01D1022300E0002318460C37BD4680
S315080235705DF8047B704780B483B000AF78600B4671
S31508023580FB701346BB70FB787A681344BA785A7193
S31508023590012318460C37BD465DF8047B704780B494
S315080235A083B000AF78600B46FB70FB787A681344E9
S315080235B01B7B012B01D1012308E0FB787A681344AF
S315080235C01B7B022B01D1022300E0002318460C378D
S315080235D0BD465DF8047B704780B483B000AF78605F
S315080235E00B46FB701346BB70FB787A681344BA78AD
S315080235F01A73012318460C37BD465DF8047B7047DB
S3150802360080B483B000AF78600B46FB701346BB707C
S31508023610FB787A681344BA78DA74012318460C37A9
S31508023620BD465DF8047B704780B483B000AF78600E
S315080236300B46FB707B68FA789A76012318460C3794
S31508023640BD465DF8047B704780B500AF03F0E2FA29
S3150802365003460121184603F07CFD0222012164205B
S3150802366000F008F9002102480CF090FF00BF80BD67
S3150802367084D8002080B500AF03F0CCFA03460121B6
S31508023680184603F083FD01220121642000F0F2F8B6
S31508023690042102480CF07AFF00BF80BD84D80020BE
S315080236A080B500AF03F0B6FA03460021184603F0C8
S315080236B08AFD03F0AFFA03460021184603F049FDD6
S315080236C003F0A8FA03460021184603F05FFD032219
S315080236D00121642000F0CEF8042104480CF056FFBC
S315080236E0002102480CF052FF00BF80BD84D800209A
S315080236F080B500AF03F08EFA03460021184603F0A0
S3150802370062FD03F087FA03460021184603F021FDFD
S3150802371003F080FA03460021184603F037FD042118
S3150802372009480DF093F8002107480DF08FF8012299
S315080237300121002000F09EF802220121002000F05B
S3150802374099F800BF80BD00BF84D8002080B500AFBD
S3150802375003F060FA03460121184603F076FD0122BA
S315080237600221642000F086F8082102480CF00EFFB8
S3150802377000BF80BD38D8002080B500AF03F04AFAF2
S3150802378003460121184603F043FD02220221642062
S3150802379000F070F80C2102480CF0F8FE00BF80BD5C
S315080237A0ECD7002080B500AF03F034FA03460021B7
S315080237B0184603F067FD03F02DFA03460021184662
S315080237C003F043FD03F026FA03460021184603F0E8
S315080237D01FFD02220221002000F04CF801220221DC
S315080237E0002000F047F80C2104480DF02FF80821B4
S315080237F003480DF02BF800BF80BD00BFECD70020B0
S3150802380038D8002080B500AF03F004FA0346002139
S31508023810184603F037FD03F0FDF903460021184662
S3150802382003F013FD03F0F6F903460021184603F0E8
S31508023830EFFC03220121632000F01CF8042104484E
S315080238400CF0A4FE002102480CF0A0FE00BF80BDC9
S3150802385084D8002080B500AFFFF73AFE034602215E
S31508023860184600F09DF8024B00221A7000BF80BD70
S315080238706CC4002080B483B000AF0346FB710B46CC
S31508023880BB7113467B713A4AFB791370FB79002B9D
S315080238904DD0BB79012B23D17B79012B08D1354B2E
S315080238A01B6800225A63334B1B68FA799A6358E0FD
S315080238B07B79022B08D12F4B1B6800229A632D4B6A
S315080238C01B68FA795A634CE07B79032B49D1294B59
S315080238D01B68FA799A63274B1B68FA795A6340E0A0
S315080238E0BB79022B3DD17B79012B08D1224B1B6870
S315080238F0FA79DA63214B1B6800221A6431E07B7974
S31508023900022B08D11C4B1B680022DA631B4B1B686F
S31508023910FA791A6425E07B79032B22D1164B1B68A8
S31508023920FA79DA63154B1B68FA791A6419E0FB7996
S31508023930002B16D1BB79012B08D10E4B1B6800222E
S315080239405A630C4B1B6800229A630AE0BB79022B66
S3150802395007D1094B1B680022DA63084B1B68002251
S315080239601A6400BF0C37BD465DF8047B704700BF7A
S315080239706BC4002084D8002038D80020ECD7002059
S3150802398080B500AFFFF7A4FD03460221184600F0F2
S3150802399007F8024B00221A7000BF80BD6DC40020D2
S315080239A080B483B000AF78600B46FB707B68FA7808
S315080239B05A7700BF0C37BD465DF8047B7047000096
S315080239C090B583B000AF04215B4806F091FB03462D
S315080239D0012B0CBF01230023DBB2BB710023FB7151
S315080239E0564B1B78BA799A424FD1FFF771FD0346B7
S315080239F000211846FFF7A2FD0346022B28D1504B99
S31508023A001B881C4603F006F90346184603F04DF9CF
S31508023A1003461846FDF77BFC03469C4202D3BB7954
S31508023A20FB7147E0464B1B8801339AB2444B1A8016
S31508023A30FFF74EFD034600211846FFF77FFD0346B2
S31508023A40012B02D10123FB7134E00023FB7131E023
S31508023A503B4B1B88312B02D9BB79FB712AE0384BC9
S31508023A601B8801339AB2364B1A80FFF731FD03469B
S31508023A7000211846FFF762FD0346012B02D10123F6
S31508023A80FB7117E00023FB7114E02C4ABB79137013
S31508023A902B4B00221A80FFF71BFD0346002118460E
S31508023AA0FFF74CFD0346012B02D10123FB7101E00E
S31508023AB00023FB71FB79002B1DD0FFF709FD034696
S31508023AC0012200211846FFF756FD1E4B1B78FA798C
S31508023AD09A422DD003F09EF803460421184603F0B5
S31508023AE0D5F90346002B02D0174804F0CBFA154A3B
S31508023AF0FB7913701CE0FFF7EBFC03460222002158
S31508023B001846FFF738FD0F4B1B78FA799A420FD001
S31508023B1003F080F803460421184603F0B7F9034672
S31508023B20002B02D0094804F0ADFA064AFB79137055
S31508023B3000BF0C37BD4690BD0004024292C4002065
S31508023B4094C4002096C4002004F903084CF903081B
S31508023B5080B582B000AF0221424806F0C9FA034690
S31508023B60012B0CBF01230023DBB2BB710023FB71BF
S31508023B703D4B1B78BA799A421CD13C4B1B88312B98
S31508023B8002D9BB79FB712AE0384B1B8801339AB2FA
S31508023B90364B1A80FFF79CFC034601211846FFF7AD
S31508023BA0CDFC0346012B02D10123FB7117E000234A
S31508023BB0FB7114E02C4ABB7913702C4B00221A8035
S31508023BC0FFF786FC034601211846FFF7B7FC0346B2
S31508023BD0012B02D10123FB7101E00023FB71FB7962
S31508023BE0002B1DD0FFF774FC03460122012118465B
S31508023BF0FFF7C1FC1E4B1B78FA799A422DD003F0C7
S31508023C0009F803460421184603F040F90346002B37
S31508023C1002D0184804F036FA154AFB7913701CE0EC
S31508023C20FFF756FC0346022201211846FFF7A3FCBA
S31508023C300F4B1B78FA799A420FD002F0EBFF034634
S31508023C400421184603F022F90346002B02D00A483B
S31508023C5004F018FA064AFB79137000BF0837BD4606
S31508023C6080BD00BF0004024297C4002098C4002009
S31508023C709AC4002094F90308E0F9030880B582B0D3
S31508023C8000AF4FF40061424806F032FA0346012BB0
S31508023C900CBF01230023DBB2BB710023FB713D4B32
S31508023CA01B78BA799A421CD13B4B1B78312B02D925
S31508023CB0BB79FB712AE0384B1B780133DAB2364BF3
S31508023CC01A70FFF705FC034601211846FFF767FC41
S31508023CD00346012B02D10123FB7117E00023FB7176
S31508023CE014E02C4ABB7913702B4B00221A70FFF78B
S31508023CF0EFFB034601211846FFF751FC0346012B49
S31508023D0002D10123FB7101E00023FB71FB79002B31
S31508023D101DD0FFF7DDFB0346012201211846FFF7F6
S31508023D205BFC1E4B1B78FA799A422DD002F072FF81
S31508023D3003460421184603F0A9F80346002B02D0CD
S31508023D40174804F09FF9154AFB7913701CE0FFF730
S31508023D50BFFB0346022201211846FFF73DFC0F4B23
S31508023D601B78FA799A420FD002F054FF03460421CF
S31508023D70184603F08BF80346002B02D0094804F0D4
S31508023D8081F9064AFB79137000BF0837BD4680BD24
S31508023D90001402429BC400209CC400209DC400203B
S31508023DA010FD03084CFD030880B582B000AF4FF43E
S31508023DB08051424806F09CF90346012B0CBF0123A9
S31508023DC00023DBB2BB710023FB713D4B1B78BA792A
S31508023DD09A421CD13B4B1B78312B02D9BB79FB711A
S31508023DE02AE0384B1B780133DAB2364B1A70FFF7E2
S31508023DF06FFB034602211846FFF7D1FB0346012B48
S31508023E0002D10123FB7117E00023FB7114E02C4A4F
S31508023E10BB7913702B4B00221A70FFF759FB034626
S31508023E2002211846FFF7BBFB0346012B02D10123E9
S31508023E30FB7101E00023FB71FB79002B1DD0FFF714
S31508023E4047FB0346012202211846FFF7C5FB1E4B14
S31508023E501B78FA799A422DD002F0DCFE0346042139
S31508023E60184603F013F80346002B02D0174804F04D
S31508023E7009F9154AFB7913701CE0FFF729FB03467B
S31508023E80022202211846FFF7A7FB0F4B1B78FA7985
S31508023E909A420FD002F0BEFE03460421184602F0EB
S31508023EA0F5FF0346002B02D0094804F0EBF8064A50
S31508023EB0FB79137000BF0837BD4680BD0014024265
S31508023EC09EC400209FC40020A0C400208CFD0308C5
S31508023ED0C8FD030880B582B000AF78600B467B80C8
S31508023EE00D4812F011FA02467B889A420FD34FF018
S31508023EF0FF310A4811F0E8FD7B881A4679680648B8
S31508023F0012F0EBFB054811F021FE012300E0002325
S31508023F1018460837BD4680BDA4C400203CA100202F
S31508023F2080B5C4B000AF024607F58873A3F2091339
S31508023F301A70002387F80F314AE007F10C034FF491
S31508023F4080720021184617F0BBFB4FF0FF31294853
S31508023F5011F0BAFD07F10C031946274812F034FC92
S31508023F60034687F80F31234811F0F0FD4FF0FF3171
S31508023F70204811F0A9FD07F10C0319461E4812F054
S31508023F80BDFB034687F80F311A4811F0DFFD4FF4DF
S31508023F907A711A4811F098FD0346002B0DD1FEF7E7
S31508023FA08EFF97F80F319AB207F10C031946FFF7FD
S31508023FB074F9124811F0CAFD02E0114804F062F8D9
S31508023FC007F58873A3F209131B78184604F0DAF981
S31508023FD0094812F0F7F9034683F00103DBB2002B16
S31508023FE003D0084B1B78002BA7D000BF07F58877AC
S31508023FF0BD4680BD3CA10020A4C4002058A10020D3
S31508024000F0020408B4C5002080B483B000AF78601B
S315080240100B467B8000BF00BF0C37BD465DF8047BAC
S315080240207047000080B582B000AF0023FB712D4BAC
S315080240301B78002B4ED02C4B1B780133DAB22A4B55
S315080240401A70294B1B78092B47D9274B00221A705D
S31508024050244B5B78012B1FD8224B5B780133DAB2EB
S31508024060204B5A704FF47A71204811F02DFD034601
S31508024070002B0DD1FEF723FF03461A4A92F8832036
S315080240801B491846FFF709F9184811F05FFD24E0A5
S31508024090184803F0F7FF20E00023FB7102E0FB79E2
S315080240A00133FB710F4B93F88330FA799A42F6D3B0
S315080240B04FF0FF31104811F007FD0D490F4812F075
S315080240C01DFB0D4811F042FD84220021054817F018
S315080240D0F7FA02E0044B00221A7000BF0837BD4601
S315080240E080BD00BFB4C5002038C6002058A10020F4
S315080240F0B7C50020F00204083CA10020A4C4002091
S3150802410080B500AF4FF480720249034812F0D0F826
S3150802411000BF80BDB4C40020A4C4002080B500AF8F
S31508024120FFF7EEFF00BF80BD80B582B000AF7860B2
S3150802413039603B68DBB21946786800F04BF800BF75
S315080241400837BD4680BD80B582B000AF7860396059
S315080241503B689BB219467868FFF7BCFE00BF083772
S31508024160BD4680BD80B582B000AF78603960064B27
S315080241701B683A6892B27968184611F093FE00BF36
S315080241800837BD4680BD00BFC411002080B582B085
S3150802419000AF78603960054B1B683A68796818463B
S315080241A011F01AFF00BF0837BD4680BDC4110020B2
S315080241B080B500AF044B1868044B054A002111F07C
S315080241C036FE00BF80BD00BFC41100204741020869
S315080241D02941020890B585B000AF78600B46FB709E
S315080241E002F018FDF860FB789BB219467868FFF76B
S315080241F00BFF7B681B780F2B17D00F2B3FDC012B8D
S3150802420002D0052B25D03AE01F49204814F0B7FF03
S315080242101D4815F002F804461B4815F00AF803462D
S3150802422019462046FFF79EFF2AE0194B01221A700B
S315080242301549174814F0C6FF134814F0EEFF044652
S31508024240114814F0F6FF034619462046FFF78AFF7F
S3150802425016E0104803F016FFF86802F03DFD0A481A
S3150802426014F0C9FF084814F0D8FF0446064814F0AB
S31508024270E0FF034619462046FFF774FF00E000BF39
S3150802428000BF1437BD4690BD68D6002070D70020FF
S315080242906CD700201003040880B500AF03480DF060
S315080242A095FE02480DF052FD00BF80BD1CD90020C4
S315080242B080B500AF00F0F4FA03F0D4FE00BF80BD6B
S315080242C080B500AF224B234A9A6062B600BF04F05B
S315080242D019F900F04DF800F02FFB00F0B3F800F0E2
S315080242E0F9F800F019F900F0CBF900F023FA00F01A
S315080242F01BF900F085FA00F0D3FA0C2116480CF0E7
S3150802430045F9082115480CF041F9002114480CF02A
S315080243103DF9042112480CF039F915F015FBFFF79F
S31508024320FDFEFFF745FF02F075FC03F09BFE0D4804
S31508024330FEF7BEFC00F02AFD0B4803F0A3FE0C2193
S315080243400A4803F063FEFEF78BF800BFFDE700BFDD
S3150802435000ED00E000000208ECD7002038D8002063
S3150802436084D8002074D700202C03040838030408D4
S3150802437080B59CB000AF07F12003502200211846F1
S3150802438017F09EF907F1080300221A605A609A602C
S31508024390DA601A615A612A4B1B69294A43F03003CB
S315080243A01361274B1B6903F030037B607B6800BFF0
S315080243B0234B5B6903F00803082BF9D109233B62F7
S315080243C04FF480337B624FF08063BB630223BB6486
S315080243D00323FB6403233B657D237B650223BB65BD
S315080243E00223FB6502233B6608237B660023BB6622
S315080243F00023FB6607F12003184605F05BFF034618
S31508024400002B01D000F0A2FB1F23BB600323FB6035
S3150802441000233B6100237B610023BB610023FB6110
S3150802442007F108030521184606F07CFB0346002B14
S3150802443001D000F08BFB00BF7037BD4680BD00BFC0
S315080244400008024480B500AF204B214A1A601F4B70
S3150802445000225A601D4B4FF440729A601B4B002291
S31508024460DA601A4B00221A74184B00225A74174B38
S3150802447000229A74154B05225A61144B0A229A6134
S31508024480124B2722DA61114B0A221A620F4B0522B6
S315080244905A620E4B02229A620C4B0722DA620B4BC5
S315080244A002221A63094B01225A63084B01229A63B4
S315080244B0064B0022DA63054804F022FA0346002B6B
S315080244C001D000F043FB00BF80BD00BF74D70020B7
S315080244D000A4004080B500AF0D4B0E4A1A600C4B83
S315080244E005225A600A4B40F2ED22DA60084B40F286
S315080244F0ED229A60064B00221A61054805F042FE33
S315080245000346002B01D000F021FB00BF80BD00BF8F
S31508024510D8D700200030004080B400AF00BFBD46A7
S315080245205DF8047B7047000080B598B000AF07F1CC
S31508024530540300221A605A609A6007F1380300226F
S315080245401A605A609A60DA601A615A619A613B1D6A
S3150802455034220021184617F0B3F8474B474A1A6027
S31508024560454B40F6C3125A60434B00229A60424BAF
S315080245706322DA60404B00221A613F4B00225A61DD
S315080245803D4B00229A613C480BF0A8FF0346002BDC
S3150802459001D000F0DBFA00237B650023BB6500230C
S315080245A0FB6507F15403194633480DF0A7F903468C
S315080245B0002B01D000F0CAFA6023BB630023FB6319
S315080245C000233B6400237B640023BB640023FB6453
S315080245D000233B6507F138030422194626480CF0E6
S315080245E037FB0346002B01D000F0B0FA07F1380377
S315080245F00822194620480CF02BFB0346002B01D053
S3150802460000F0A4FA07F138030C2219461A480CF0EE
S315080246101FFB0346002B01D000F098FA00237B60AB
S315080246200023BB600023FB6000233B6100237B6100
S315080246304FF40053BB610023FB6100233B62002356
S315080246407B624FF00073BB620023FB6200233B636D
S3150802465000237B633B1D194607480DF01FFA0346E4
S31508024660002B01D000F072FA034802F023F800BFCB
S315080246706037BD4680BD00BFECD70020002C014044
S3150802468080B58AB000AF07F11C0300221A605A608F
S315080246909A603B4600221A605A609A60DA601A618A
S315080246A05A619A61224B4FF080421A60204B40F6BB
S315080246B0C3125A601E4B00229A601D4B6322DA60AF
S315080246C01B4B00221A611A4B00229A6118480BF0FA
S315080246D005FF0346002B01D000F038FA0023FB61E0
S315080246E000237B6207F11C03194611480DF006F9EF
S315080246F00346002B01D000F029FA60233B60002311
S315080247007B600023BB6000233B613B4608221946B7
S3150802471007480CF09DFA0346002B01D000F016FA62
S31508024720034801F0C7FF00BF2837BD4680BD00BF5A
S3150802473038D8002080B58AB000AF07F11C030022E2
S315080247401A605A609A603B4600221A605A609A605A
S31508024750DA601A615A619A61274B284A1A60264B0F
S3150802476040F6C3125A60244B00229A60224B6322F7
S31508024770DA60214B00221A611F4B00229A611E48F9
S315080247800BF0ACFE0346002B01D000F0DFF9002344
S31508024790FB6100237B6207F11C03194616480DF0DC
S315080247A0ADF80346002B01D000F0D0F960233B6038
S315080247B000237B600023BB6000233B613B4600224B
S315080247C019460D480CF044FA0346002B01D000F0B6
S315080247D0BDF93B460422194607480CF039FA034646
S315080247E0002B01D000F0B2F9034801F063FF00BFC5
S315080247F02837BD4680BD00BF84D800200008004087
S3150802480080B588B000AF3B1D00221A605A609A60D4
S31508024810DA601A615A619A611F4B204A1A601E4B66
S31508024820F9225A601C4B00229A601B4B6322DA60FB
S31508024830194B00221A61184B00229A6116480BF08E
S315080248404DFE0346002B01D000F080F960237B6001
S315080248500023BB600023FB6000237B613B1D002213
S3150802486019460D480CF0F4F90346002B01D000F066
S315080248706DF93B1D0422194607480CF0E9F903466F
S31508024880002B01D000F062F9034801F013FF00BFC4
S315080248902037BD4680BD00BFD0D800200018004092
S315080248A080B500AF224B234A1A60214B4FF4E132FE
S315080248B05A601F4B00229A601D4B0022DA601C4B7D
S315080248C000221A611A4B0C225A61194B00229A616C
S315080248D0174B0022DA61164B00221A62144B002289
S315080248E05A62134B00229A6211480DF0DFF9034609
S315080248F0002B01D000F02AF900210D480FF04FFADB
S315080249000346002B01D000F021F9002108480FF0D8
S3150802491084FA0346002B01D000F018F904480FF078
S3150802492005FA0346002B01D000F010F900BF80BD3E
S315080249301CD900200038014080B58CB000AF07F1C1
S315080249401C0300221A605A609A60DA601A616F4B79
S31508024950D3F88C306D4A43F02003C2F88C306B4B87
S31508024960D3F88C3003F02003BB61BB69674BD3F8DD
S315080249708C30664A43F08003C2F88C30634BD3F816
S315080249808C3003F080037B617B69604BD3F88C30F3
S315080249905E4A43F00103C2F88C305C4BD3F88C3084
S315080249A003F001033B613B69584BD3F88C30574AF5
S315080249B043F00403C2F88C30544BD3F88C3003F01E
S315080249C00403FB60FB68514BD3F88C304F4A43F023
S315080249D00203C2F88C304D4BD3F88C3003F0020335
S315080249E0BB60BB68494BD3F88C30484A43F0100386
S315080249F0C2F88C30454BD3F88C3003F010037B6039
S31508024A007B68424BD3F88C30404A43F00803C2F81D
S31508024A108C303E4BD3F88C3003F008033B603B687E
S31508024A20002201213A4805F07BFB00221021394871
S31508024A3005F076FB0123FB6101233B6200237B62BF
S31508024A400023BB6207F11C031946314805F042F9F7
S31508024A501023FB6101233B6200237B620023BB62B6
S31508024A6007F11C0319462B4805F034F9C023FB61EC
S31508024A7000233B6200237B6207F11C031946254883
S31508024A8005F028F93023FB6100233B6200237B6291
S31508024A9007F11C031946204805F01CF942F20703E0
S31508024AA0FB6100233B6200237B6207F11C03194664
S31508024AB01A4805F00FF94FF4C053FB6100233B6215
S31508024AC000237B6207F11C031946114805F002F917
S31508024AD04FF40243FB6100233B6200237B6207F12A
S31508024AE01C0319460E4805F0F5F84FF40063FB61FE
S31508024AF000233B6200237B6207F11C03194609481F
S31508024B0005F0E8F800BF3037BD4680BD000C024408
S31508024B100014024200000242000802420004024255
S31508024B2000100242000C024280B582B000AF7860E3
S31508024B307B681B68044A934201D103F009FD00BF52
S31508024B400837BD4680BD00BF0020004080B400AFD4
S31508024B5072B600BF00BFFDE7B0B596B000AF786089
S31508024B60396000237B65684B684A4021786804F0FF
S31508024B7043F90346002B03D0654803F083FA51E054
S31508024B80FEF77AF90346002B03D0604B1B687B6558
S31508024B9002E05E4B1B687B65FEF788F902467B6D71
S31508024BA0934204D168215948FEF740F83AE012F0D8
S31508024BB0E3FD02467B6D934229D012F020FE02469F
S31508024BC07B6D934223D012F0C9FD02467B6D934258
S31508024BD01DD012F057FE02467B6D934217D012F093
S31508024BE047FE02467B6D934211D012F025FE02461D
S31508024BF07B6D93420BD012F059FE02467B6D9342AF
S31508024C0005D012F049FE02467B6D93420AD13F4B0C
S31508024C10DB681846FEF7B7F903461A463A49786D2D
S31508024C2014F0CAFE7868FEF7A1F803461A46394B0D
S31508024C309A607868FEF760F80346364A1360786821
S31508024C40FEF775F80346334A5360324B9B68002BCE
S31508024C5012D0304B1A682F4B5B6807F10C002E49AD
S31508024C6016F09AFC07F10C03184603F00BFA294BC7
S31508024C709B681846FEF7CEF80C222649274816F0F6
S31508024C800FFD0346002B36D0224B1B68DAB207F11A
S31508024C9050031146184612F0F7FB1E4B5B68DAB250
S31508024CA007F150031146184612F009FC194B9B6886
S31508024CB0DAB207F150031146184612F01BFC07F147
S31508024CC00C0207F150031146184612F00AFD12F0BB
S31508024CD06FFD044607F10C03184612F01AFC054646
S31508024CE007F10C03184612F020FC03461A46294619
S31508024CF0204614F011FF094B064A07CA83E8070043
S31508024D0000BF5837BD46B0BDD8D90020B0D900205B
S31508024D104803040850C40020680304085CC4002041
S31508024D2080B58CB002AFF860B9607A604FF0804304
S31508024D303B6100237B61FB68BB610123FB61BB68A6
S31508024D403B627B687B6207F110031946074803F04A
S31508024D5031FF01230093012302220221034803F0B3
S31508024D6083FF00BF2837BD4680BD00BF74D7002029
S31508024D7080B500AF044803F0A8FF002201210248CB
S31508024D8004F0A8F900BF80BD74D7002080B500AF33
S31508024D90FEF78CF803461A466FF060410220FFF7C9
S31508024DA0BFFFFFF7E5FF00BF80BD000080B58EB0EC
S31508024DB000AFF860B9601346FB71FB79002B02D08D
S31508024DC0FB79402B01D900233FE007F11403242283
S31508024DD00021184616F074FCFB687B61FEF74CF856
S31508024DE00346002B03D04FF08043BB6101E000234A
S31508024DF0BB610023FB61FB799BB21846FEF76CF890
S31508024E0003463B6200237B624FF48013BB624FF476
S31508024E100013FB6200233B6300237B634FF47A7122
S31508024E200C4810F051FE0346002B0AD107F1140371
S31508024E30BA6819460848FDF77FFC064810F086FE50
S31508024E4002E0064803F01EF9012318463837BD4624
S31508024E5080BD00BF20A1002074D700208C0304085F
S31508024E6080B500AF074B1B78DBB2002B07D1054B89
S31508024E7001221A7004220021034816F021FC024B73
S31508024E80184680BD33DA00201CDA002080B584B0CB
S31508024E9000AF0346FB7103233B7320237B73FB7925
S31508024EA0BB7307F10C0303221946034814F066FD87
S31508024EB000BF1037BD4680BD0600080080B483B027
S31508024EC000AF78600B46FB707B68FA78DA7000BF31
S31508024ED00C37BD465DF8047B704780B483B000AFDB
S31508024EE078607B68DB7818460C37BD465DF8047B2C
S31508024EF0704780B483B000AF78600B46FB707B685E
S31508024F00FA789A70002318460C37BD465DF8047B7A
S31508024F10704780B483B000AF78607B689B78184688
S31508024F200C37BD465DF8047B704780B500AFFEF7C7
S31508024F30CFFA034600211846FEF700FB0346022B6A
S31508024F4007D101F067FE03460221184602F0DCF992
S31508024F503BE0FEF7BDFA034601211846FEF7EEFAD4
S31508024F600346022B07D101F055FE034601211846D6
S31508024F7002F0CAF929E0FEF7ABFA03460121184600
S31508024F80FEF7DCFA0346022B18D1FEF7A1FA03460E
S31508024F9000211846FEF7D2FA0346022B0ED101F07B
S31508024FA039FE03466421184602F0CBF913F040FF96
S31508024FB001230B22652113F085FF06E001F02AFE84
S31508024FC003460021184602F09FF9FEF781FA0346C6
S31508024FD001211846FEF7E3FA0346022B07D101F030
S31508024FE019FE03460121184602F0E5F93BE0FEF7F1
S31508024FF06FFA034602211846FEF7D1FA0346022B38
S3150802500007D101F007FE03460221184602F0D3F93A
S3150802501029E0FEF75DFA034602211846FEF7BFFAB3
S315080250200346022B18D1FEF753FA03460121184606
S31508025030FEF7B5FA0346022B0ED101F0EBFD034645
S315080250406521184602F0B7F913F0F2FE01230A2287
S31508025050652113F037FF06E001F0DCFD0346002167
S31508025060184602F0A8F900BF80BD000080B500AF5F
S3150802507001F0D0FD0346184602F07BF80346002BE2
S3150802508048D001F0C7FD0346184602F0ACF80346BD
S315080250901A4641F657339A4240F28580FEF728FBB4
S315080250A001F0B8FD03460021184602F08CF888483C
S315080250B003F04EF801F0AEFD03460021184602F051
S315080250C048F801F0A7FD03460121184602F05EF8EA
S315080250D06620FFF7DBFE7F4B00221A707E4B00220A
S315080250E01A707E4B00221A7001F094FD034666215F
S315080250F0184602F026F913F09BFE012303226521C6
S3150802510013F0E0FEFFF7ACFE034602211846FFF74E
S31508025110F0FE48E001F07EFD0346184602F046F826
S315080251200346002B3FD001F075FD0346184602F0F0
S315080251305AF803461A4641F657339A4233D9FEF7C6
S31508025140D7FA01F067FD03460021184602F03BF83C
S31508025150634802F0FDFF01F05DFD03460021184693
S3150802516002F014F86720FFF791FE5A4B00221A70D4
S31508025170594B00221A70594B00221A70FFF770FE1B
S31508025180034600211846FFF7B4FE01F043FD034625
S315080251906721184602F0D5F813F04AFE01230422C5
S315080251A0652113F08FFE01F035FD0346184602F01D
S315080251B03FF80346002B40D001F02CFD0346184663
S315080251C002F070F803461A4641F657339A427DD9D9
S315080251D0FEF7E8FA01F01EFD03460021184602F022
S315080251E051F8404802F0B4FF01F014FD03460021CD
S315080251F0184602F00DF86820FFF748FE354B0022E4
S315080252001A70354B00221A70344B00221A70FFF7B7
S3150802521027FE034600211846FFF76BFE01F0FAFC4B
S3150802522003466821184602F08CF813F001FE0123A2
S315080252300122652113F046FE48E001F0EBFC034625
S31508025240184602F012F80346002B3FD001F0E2FCA2
S315080252500346184602F026F803461A4641F657331D
S315080252609A4233D9FEF79EFA01F0D4FC034600218E
S31508025270184602F007F81C4802F06AFF01F0CAFC59
S3150802528003460021184601F0E0FF6920FFF7FEFDFC
S31508025290104B00221A70104B00221A700F4B002274
S315080252A01A70FFF7DDFD034600211846FFF721FEB7
S315080252B001F0B0FC03466921184602F042F813F0E1
S315080252C0B7FD01230222652113F0FCFD00BF80BD54
S315080252D0AC03040820DA002021DA002022DA0020B2
S315080252E0E0030408140404084404040880B500AF63
S315080252F04C4B1B8801339AB24A4B1A804A4B1B788D
S31508025300022B44D0022B00F38480002B02D0012BFF
S3150802531013D07EE0FEF7DCF8034600211846FEF7B6
S315080253200DF90346022B76D1404802F011FFFEF72B
S315080253308BF93D4B01221A706DE03A4B1B8840F6F9
S31508025340B73293420DD9374B00221A80384802F0F9
S31508025350FFFE354B00221A70FEF7A2F94FF0FF3313
S315080253605DE0FEF7B5F8034600211846FEF7E6F8B3
S315080253700346012B51D12F4802F0EAFEFEF790F9B7
S31508025380294B02221A70274B00221A8045E0254B28
S315080253901B8840F6B73293420DD9224B00221A8057
S315080253A0254802F0D5FE204B00221A70FEF778F93E
S315080253B04FF0FF3333E0FEF78BF803460021184619
S315080253C0FEF7BCF80346022B20D11C4802F0C0FEA9
S315080253D0FEF766F9144B00221A70124B00221A8045
S315080253E0FEF776F8034601211846FEF7A7F80346A4
S315080253F0022B09D1124802F0ABFE13F019FD012364
S315080254000E22652113F05EFD012308E0FEF732F94C
S3150802541004E000BF02E000BF00E000BF0023184618
S3150802542080BD00BF30DA00202EDA0020740404089A
S31508025430A4040408CC040408E00404080C050408BF
S31508025440300504082DE9F04182B002AFD04B1B7833
S315080254500D2B00F2108701A252F823F09554020888
S3150802546077620208776202087762020877620208A0
S315080254707762020877620208776202087762020890
S3150802548041560208E5570208495902086D5D0208A5
S31508025490E1610208BF4B00221A70BF4B00221A7044
S315080254A0BE4B1B78002B10D1BC4B01221A7013F08D
S315080254B0F9FE0346184613F078FF034600211846FC
S315080254C012F041FFB24B09221A70FFF7C9FC0346D4
S315080254D01846FFF71EFD0346052B26D1B04B0022C0
S315080254E01A8001F097FB03460121184601F046FF90
S315080254F001F090FB03460221184601F0E8FE13F07C
S31508025500D1FE0346184613F050FF034602211846F9
S3150802551012F019FFA34B01221A709D4B09221A7029
S31508025520A14802F015FE00F0A8BEFFF799FC034653
S315080255301846FFF7EEFC0346062B2AD101F06AFB52
S3150802554003460121184601F019FF01F063FB0346E1
S315080255500421184601F0BBFE13F0A4FE03461846C2
S3150802556013F023FF03460421184612F0ECFE8F4B74
S3150802557001221A70FFF774FC034601211846FFF749
S31508025580B8FC834B0B221A70894802F0E1FD00F041
S3150802559074BEFFF765FC03461846FFF7BAFC0346D6
S315080255A0012B08D0FFF75CFC03461846FFF7B1FC4F
S315080255B00346022B06D1764B0B221A707D4802F05F
S315080255C0C7FD3BE0FFF74CFC03461846FFF7A1FC74
S315080255D00346032B08D0FFF743FC03461846FFF79A
S315080255E098FC0346042B06D1694B0C221A707248A2
S315080255F002F0AEFD22E0FFF733FC03461846FFF73A
S3150802560088FC0346072B04D1614B0D221A7000F061
S3150802561034BEFFF725FC03461846FFF77AFC034615
S31508025620092B40F02A86654802F092FD644B012256
S315080256301A70574B09221A7000F01FBE00F01DBEE1
S31508025640FDF746FF034600211846FDF777FF034696
S31508025650022B65D1FDF73CFF034601211846FDF7EB
S315080256606DFF0346012B5BD1564B1B680133554A26
S315080256701360544B1B68012B50DD524B00221A60F3
S31508025680002201210020FEF7F5F8FEF731F84E4810
S3150802569002F05EFD13F006FE0346184613F085FE79
S315080256A003460221184612F05DFE3A4B01221A7091
S315080256B0464B1B78002B2DD1454B01221A7001212E
S315080256C0444804F015FD0346012B0ED113F0EAFDFA
S315080256D00346184613F069FE03460121184612F0DE
S315080256E032FE3D4802F034FD0DE013F0DBFD0346C1
S315080256F0184613F05AFE03460121184612F041FED7
S31508025700364802F025FD314B01221A70204B002241
S315080257101A7005E01E4B0A221A7001E0FDF7E8FF2F
S3150802572004212C4804F0E4FC0346012B2BD0022169
S31508025730284804F0DDFC0346012B24D0FDF7D8FFE8
S31508025740274802F005FD174B00221A70104B00225B
S315080257501A70FFF785FB034600211846FFF7C9FBB7
S315080257606420FFF793FB01F055FA034664211846B5
S3150802577001F0E7FD13F05CFB01230B22652113F010
S31508025780A1FB00F07FBDFDF775FF00F07BBD00BFF2
S3150802579020DA002024DA002025DA00202CDA00207C
S315080257A018DA002021DA00205406040822DA00203A
S315080257B0780604089C060408B4060408CC060408FD
S315080257C023DA002028DA0020EC0604082DDA002065
S315080257D032DA00200004024200070408140704080B
S315080257E028070408FDF774FE034601211846FDF74B
S315080257F0D6FE0346022B53D1FDF76AFE0346022163
S315080258001846FDF7CCFE0346012B49D1AE4B1B6861
S315080258100133AD4A1360AC4B1B68632B3DDDAA4BC3
S3150802582000221A60A94802F093FCFDF7BBFFA84BB9
S3150802583001221A70A74B1B78012B11D1A64802F038
S3150802584087FCA64B1B78002B1BD0FFF709FB0346E8
S3150802585001211846FFF74DFBA14B0B221A7010E0E7
S31508025860A04B1B78012B0CD19F4802F071FCFFF765
S31508025870F7FA034601211846FFF73BFB984B0B2222
S315080258801A7013F00FFD0346184613F08EFD0346F1
S315080258900321184612F066FD54E0FDF783FF51E036
S315080258A0FDF716FE034601211846FDF778FE034664
S315080258B0022B2DD1FDF70CFE034602211846FDF7F1
S315080258C06EFE0346022B23D1FDF76CFF874802F0D2
S315080258D03FFC804B00221A70814B00221A70FFF798
S315080258E0BFFA034600211846FFF703FB6520FFF7B8
S315080258F0CDFA01F08FF903466521184601F021FD1C
S3150802590013F096FA01230A22652113F0DBFA19E04D
S315080259100121774804F0ECFB0346012B0ED07548AB
S3150802592002F016FCFFF79CFA034601211846FFF718
S31508025930E0FA6B4B0B221A7000F0A4BCFDF71CFFB1
S3150802594000F0A0BC00F09EBCFFF78AFA0346184690
S31508025950FFF7DFFA0346012B40F0D480FDF7B8FDC6
S31508025960034601211846FDF7E9FD0346022B6DD1D0
S31508025970FDF7AEFD034600211846FDF7DFFD034697
S31508025980012B63D1504B1B6801334F4A13604E4BB0
S315080259901C6801F03FF90346184601F039FD034633
S315080259A09C4250DB484B00221A60FDF779FEFDF750
S315080259B029FF01F02FF90346184601F029FD03468F
S315080259C019464D4802F0C4FB01F024F903460021AA
S315080259D0184601F00DFD13F065FC0346184613F050
S315080259E0E4FC03460121184612F0BCFCFFF738FA1C
S315080259F0034600211846FFF77CFA364B1B78012B23
S31508025A0003D0384B1B78012B0AD1FFF729FA034634
S31508025A1003211846FFF76DFA314B0C221A70A4E1DE
S31508025A20364B1B78012B0AD1FFF71AFA03460421D3
S31508025A301846FFF75EFA2A4B0C221A7095E1284B94
S31508025A4000221A7091E1FDF7FFFD8EE1FDF740FD98
S31508025A50034601211846FDF771FD0346022B30D194
S31508025A60FDF736FD034600211846FDF767FD034696
S31508025A70022B26D1224802F06BFBFDF739FE154BA5
S31508025A8000221A701D4B00221A70154B00221A703A
S31508025A90FFF7E6F9034600211846FFF72AFA6420BB
S31508025AA0FFF7F4F901F0B6F803466421184601F047
S31508025AB048FC13F0BDF901230B22652113F002FA03
S31508025AC053E1FDF7C1FDDAE328DA00205807040896
S31508025AD025DA002021DA00206C07040824DA0020DF
S31508025AE020DA002023DA002084070408A407040821
S31508025AF000040242D8070408EC07040822DA002048
S31508025B000C080408FFF7ACF903461846FFF701FA32
S31508025B100346022B40F0B383FDF7DAFC0346002165
S31508025B201846FDF70BFD0346022B40F0E080FDF711
S31508025B30CFFC034601211846FDF700FD0346012B5B
S31508025B4040F0D580B74B1B680133B64A1360B54B94
S31508025B501B68312B40F3C880B24B00221A60FDF74E
S31508025B60C7FDB14802F0F4FA13F09CFB0346184647
S31508025B7013F01BFC03460221184612F0F3FBFFF74B
S31508025B806FF9034600211846FFF7B3F9A74B1B78AE
S31508025B90012B30D1FDF7ACFDA54802F0D9FA13F076
S31508025BA081FB0346184613F000FC034603211846F8
S31508025BB012F0C9FBFFF754F9034600211846FFF70E
S31508025BC098F901219B4804F093FA0346012B03D066
S31508025BD0994802F0BDFA02E0984802F0B9FA00F0D4
S31508025BE05FFB974B00221A70904B00221A70954B56
S31508025BF003221A70B9E0944B1B78012B47D19348BC
S31508025C0002F0A6FA13F04EFB0346184613F0CDFB34
S31508025C1003460521184612F096FBFFF721F90346BB
S31508025C2000211846FFF765F90121824804F060FA57
S31508025C300346012B14D1864802F08AFA0320FFF79D
S31508025C4025F900F0E7FF03460021184601F0B4F9EA
S31508025C5000F0E0FF03460021184601F0CAF90CE0FD
S31508025C607C4802F075FA0420FFF710F913F0E0F801
S31508025C7001231122652113F025F9714B00221A70AE
S31508025C80714B00221A706F4B03221A706DE0724B29
S31508025C901B78012B24D10121664804F029FA034610
S31508025CA0012B06D06D4802F053FA0720FFF7EEF8EB
S31508025CB005E06B4802F04CFA0820FFF7E7F8694856
S31508025CC002F046FAFFF7CCF8034600211846FFF71A
S31508025CD010F9614B00221A70594B00221A7044E0DF
S31508025CE0574B00221A7040E0FDF7DAFC3DE0FDF75B
S31508025CF0EFFB034600211846FDF720FC0346022B5C
S31508025D0030D1FDF7E5FB034601211846FDF716FCDF
S31508025D100346022B26D1FDF7C3FC534802F018FAB4
S31508025D20424B00221A70484B00221A70FFF798F865
S31508025D30034600211846FFF7DCF86420FFF7A6F8A9
S31508025D4000F068FF03466421184601F0FAFA3C4B54
S31508025D5000221A7013F06CF801230B22652113F046
S31508025D60B1F802E0FDF786FC89E288E2FFF778F8E7
S31508025D7003461846FFF7CDF80346042B40F0B680D3
S31508025D80FDF7A6FB034601211846FDF708FC034664
S31508025D90022B6DD1FDF79CFB034602211846FDF73F
S31508025DA0FEFB0346012B63D11E4B1B6801331D4ABA
S31508025DB013601C4B1B68632B30DD1A4B00221A60DA
S31508025DC02A4802F0C5F9FDF7EDFCFFF749F8034644
S31508025DD000211846FFF78DF813F064FA03461846B1
S31508025DE013F0E3FA03460321184612F0BBFA164BE0
S31508025DF01B78012B03D0184B1B78012B0AD1FFF70E
S31508025E002FF8034602211846FFF773F80C4B0B22AC
S31508025E101A70C4E10A4B00221A70C0E1FDF7ACFC05
S31508025E20BDE100BF28DA00205008040821DA002064
S31508025E30680804080004024284080408980804084A
S31508025E4020DA00202CDA002022DA0020AC08040826
S31508025E50C8080408D808040823DA0020F008040849
S31508025E601C0904084809040874090408A409040852
S31508025E70FDF72EFB034601211846FDF790FB034664
S31508025E80022B30D1FDF724FB034602211846FDF703
S31508025E9086FB0346022B26D1FDF784FCC04802F096
S31508025EA057F9C04B00221A70BF4B00221A70FEF730
S31508025EB0D7FF034600211846FFF71BF8BB4B002203
S31508025EC01A706520FEF7E2FF00F0A4FE034665217C
S31508025ED0184601F036FA12F0ABFF01230A226521B1
S31508025EE012F0F0FF5BE1FDF747FCCAE1FEF7B8FFE7
S31508025EF003461846FFF70DF80346032B40F0C18107
S31508025F00A84B1B78012B04D0A94B1B78012B40F018
S31508025F10BB80FDF7DDFA034602211846FDF73FFB73
S31508025F200346022B37D1FDF7D3FA03460121184659
S31508025F30FDF735FB0346012B2DD19E4B1B6801331A
S31508025F409C4A13609B4B1B68B3F5FA7F20DB9A4B7E
S31508025F5000221A80974B00221A60984802F0F8F835
S31508025F60FDF720FCFEF77CFF034602211846FEF7E2
S31508025F70C0FF13F097F90346184613F016FA0346BC
S31508025F800421184612F0EEF9884B0B221A707AE0B1
S31508025F90FDF7DCFB77E0FDF79BFA0346022118467C
S31508025FA0FDF7FDFA0346022B30D1FDF791FA0346B7
S31508025FB001211846FDF7F3FA0346022B26D1FDF70F
S31508025FC0F1FB7F4802F0C4F8764B00221A70764B32
S31508025FD000221A70FEF744FF034600211846FEF710
S31508025FE088FF6520FEF752FF00F014FE034665217E
S31508025FF0184601F0A6F96D4B00221A7012F018FF26
S3150802600001230A22652112F05DFF3CE06A4B1B88D8
S3150802601001339AB2684B1A80674B1B88B3F5FA6F3D
S315080260202ED30121674804F063F80346012B03D0F7
S31508026030654802F08DF802E0644802F089F85E4B82
S3150802604000221A80FDF7AEFBFEF70AFF034602217D
S315080260501846FEF74EFF13F025F90346184613F0C5
S31508026060A4F903460421184612F07CF9584802F0AE
S315080260706FF8584802F06CF84C4B0B221A708EE0F7
S31508026080FDF764FB8BE08AE0FDF722FA034602215C
S315080260901846FDF784FA0346022B42D1FDF718FA91
S315080260A0034601211846FDF77AFA0346012B38D131
S315080260B0404B1B6801333F4A13603E4B1B68632BF8
S315080260C02CDD3C4B00221A60434802F041F8FDF7EA
S315080260D069FB13F0E7F80346184613F066F9034618
S315080260E00421184612F03EF9314B1B78012B0AD1CE
S315080260F0FEF7B6FE034602211846FEF7FAFE2B4BBA
S315080261000B221A704BE0294B00221A70FEF7A8FEE2
S31508026110034600211846FEF7ECFE40E0FDF716FBA3
S315080261203DE0FDF7D5F9034602211846FDF737FA91
S315080261300346022B30D1FDF7CBF903460121184657
S31508026140FDF72DFA0346022B26D1FDF72BFB234832
S3150802615001F0FEFF134B00221A70134B00221A702D
S31508026160FEF77EFE034600211846FEF7C2FE6520AC
S31508026170FEF78CFE00F04EFD03466521184601F037
S31508026180E0F80A4B00221A7012F052FE01230A2284
S31508026190652112F097FE02E0FDF7D8FA71E070E089
S315080261A0B409040821DA002022DA002020DA0020C5
S315080261B023DA002028DA002018DA0020E809040881
S315080261C0000A040800040242340A0408480A0408B9
S315080261D0600A0408800A0408AC0A0408BC0A04080F
S315080261E004212B4803F084FF0346012B0CBF01232D
S315080261F00023DBB21D460221254803F079FF034638
S31508026200012B0CBF01230023DBB21E464FF480513B
S31508026210204803F06DFF0346012B0CBF0123002320
S31508026220DBB298464FF400611A4803F061FF034651
S31508026230012B0CBF01230023DBB21C4601211448A3
S3150802624003F056FF0346012B0CBF01230023DBB2E2
S31508026250019300944346324629460F4801F078FFD7
S31508026260FEF7FEFD034600211846FEF742FE0B4BDB
S3150802627000221A7006E000BF04E000BF02E000BF79
S3150802628000E000BF00231846BD46BDE8F08100BF06
S315080262900004024200140242F00A040820DA00202E
S315080262A080B500AF00F0B6FC0346184600F0D2FEF1
S315080262B0034619465F4801F04BFF00F0ABFC034664
S315080262C00921184600F0B6FE00F0A4FC034618465B
S315080262D000F0C0FE0346023B042B00F29A8001A29C
S315080262E052F823F0F96202082B6302085D6302087A
S315080262F08F630208E163020801214F4803F0F8FEA2
S315080263000346012B0DD000F085FC034603211846EF
S3150802631000F0DDFF0120FEF7B9FD484801F018FF3D
S3150802632086E0474801F014FF82E00121424803F063
S31508026330DFFE0346012B0DD000F06CFC0346032159
S31508026340184600F0C4FF0120FEF7A0FD3D4801F003
S31508026350FFFE6DE03A4801F0FBFE69E0012136488E
S3150802636003F0C6FE0346012B0DD000F053FC03468C
S315080263700321184600F0ABFF0120FEF787FD3248DD
S3150802638001F0E6FE54E02E4801F0E2FE50E001215B
S31508026390294803F0ADFE0346012B0DD000F03AFC66
S315080263A003460321184600F092FF0120FEF76EFD10
S315080263B0264801F0CDFE3BE001211F4803F098FE76
S315080263C00346012B02D1224801F0C2FE00F022FC4C
S315080263D00346184600F06BFE1E4801F0B9FE27E098
S315080263E00121154803F084FE0346012B0DD000F067
S315080263F011FC03460321184600F069FF0120FEF747
S3150802640045FD154801F0A4FE12E00D4801F0A0FE74
S315080264100EE00120FEF73AFD00F0FCFB03461846A3
S3150802642000F018FE034619460C4801F091FE00BF1B
S3150802643000BF80BD6C0B040800040242A00B0408CE
S31508026440E40B0408100C0408540C0408980C0408FD
S31508026450DC0C0408180D0408500D0408940D0408F1
S3150802646080B500AF074B1B78DBB2002B07D1054B73
S3150802647001221A7014220021034815F021F9024B51
S31508026480184680BD34DA002038DA002080B483B09A
S3150802649000AF78600B46FB707B68FA781A7000BF0B
S315080264A00C37BD465DF8047B704780B400AF00BF69
S315080264B0BD465DF8047B704780B5CCB000AF07F5E2
S315080264C09873A3F59673186007F58E7300221A60FF
S315080264D05A609A60DA601A6107F59873A3F59073A1
S315080264E018464FF484731A46002115F0E9F807F5A1
S315080264F09873A3F596731B681B68384A934267D14B
S3150802650007F59873A3F590714FF000024FF0040354
S31508026510C1E9002307F59873A3F590734FF48072C7
S31508026520C3F8BC2007F11003184604F075FE0346AB
S31508026530002B01D0FEF70AFB294BD3F8A030284AD4
S3150802654043F40073C2F8A030254BD3F8A03003F405
S31508026550007207F59873A3F592731A6007F5987394
S31508026560A3F592731B681E4BD3F88C301C4A43F072
S315080265700103C2F88C301A4BD3F88C3003F00102AF
S3150802658007F59873A3F594731A6007F59873A3F53C
S3150802659094731B684FF4C053C7F81C310223C7F81B
S315080265A020310023C7F824310323C7F828310923E9
S315080265B0C7F82C3107F58E7319460A4803F08AFB89
S315080265C000220021272002F0BFF8272002F0D6F881
S315080265D000BF07F59877BD4680BD00BF00A40040FE
S315080265E0000C02440000024280B487B000AF786013
S315080265F07B681B682B4A93420FD12B4BD3F8A430E6
S31508026600294A43F40063C2F8A430274BD3F8A430CE
S3150802661003F400637B617B693DE07B681B68B3F129
S31508026620804F0FD1204BD3F89C301F4A43F0010309
S31508026630C2F89C301C4BD3F89C3003F001033B6133
S315080266403B6928E07B681B68184A93420FD1164BB0
S31508026650D3F89C30144A43F00403C2F89C30124B18
S31508026660D3F89C3003F00403FB60FB6813E07B68F5
S315080266701B680F4A93420ED10B4BD3F89C300A4A39
S3150802668043F04003C2F89C30074BD3F89C3003F022
S315080266904003BB60BB6800BF1C37BD465DF8047B80
S315080266A0704700BF002C0140000C0244000800405D
S315080266B00018004080B58CB000AF786007F11C0363
S315080266C000221A605A609A60DA601A617B681B684F
S315080266D04C4A934220D14C4BD3F88C304A4A43F069
S315080266E01003C2F88C30484BD3F88C3003F01003F1
S315080266F0BB61BB694FF4D043FB6102233B620023B3
S315080267007B620023BB620123FB6207F11C03194665
S315080267103E4803F0DFFA70E07B681B68B3F1804FEE
S3150802672020D1394BD3F88C30374A43F00203C2F8EA
S315080267308C30354BD3F88C3003F002037B617B69CE
S315080267404FF48063FB6102233B6200237B620023D2
S31508026750BB620123FB6207F11C0319462C4803F0AE
S31508026760B9FA4AE07B681B682A4A934220D1264B2B
S31508026770D3F88C30244A43F00803C2F88C30224BF3
S31508026780D3F88C3003F008033B613B694FF440535E
S31508026790FB6102233B6200237B620023BB62022366
S315080267A0FB6207F11C0319461B4803F093FA24E01F
S315080267B07B681B68194A93421FD1134BD3F88C3056
S315080267C0114A43F00203C2F88C300F4BD3F88C30CF
S315080267D003F00203FB60FB684FF44043FB610223AC
S315080267E03B6200237B620023BB620223FB6207F142
S315080267F01C031946064803F06DFA00BF3037BD463A
S3150802680080BD00BF002C0140000C02440010024269
S315080268100004024200080040000C02420018004030
S3150802682080B5CCB000AF07F59873A3F596731860D8
S3150802683007F58E7300221A605A609A60DA601A6146
S3150802684007F59873A3F5907318464FF484731A469E
S31508026850002114F035FF07F59873A3F596731B68A4
S315080268601B68374A934265D107F59873A3F5907169
S315080268704FF001024FF00003C1E9002307F59873B0
S31508026880A3F590730022DA6507F11003184604F09F
S31508026890C3FC0346002B01D0FEF758F9294BD3F85F
S315080268A0A430284A43F48043C2F8A430254BD3F8CF
S315080268B0A43003F4804207F59873A3F592731A601D
S315080268C007F59873A3F592731B681E4BD3F88C30A1
S315080268D01C4A43F00103C2F88C301A4BD3F88C30A9
S315080268E003F0010207F59873A3F594731A6007F586
S315080268F09873A3F594731B684FF4C063C7F81C31E9
S315080269000223C7F820310023C7F824310023C7F829
S3150802691028310723C7F82C3107F58E7319460A481A
S3150802692003F0D8F9002200213A2001F00DFF3A209F
S3150802693001F024FF00BF07F59877BD4680BD00BF6A
S3150802694000380140000C02440000024280B582B0C1
S3150802695000AF78607B681B680B4A93420FD10B4BDA
S31508026960D3F8A430094A23F48043C2F8A4304FF47A
S31508026970C061074803F000FB3A2001F00DFF00BF93
S315080269800837BD4680BD00BF00380140000C0244EE
S315080269900000024280B58EB000AF7860334BD3F860
S315080269A09C30324A43F48073C2F89C302F4BD3F89A
S315080269B09C3003F48073BB60BB6807F10C0207F1D5
S315080269C010031146184604F0EFFBFB69FB62FB6AEB
S315080269D0002B03D104F0A6FB786304E004F0A2FBC3
S315080269E003465B007B637B6B5B09214AA2FB03239D
S315080269F0DB09013BBB621F4B1F4A1A601D4B632210
S31508026A00DA601C4ABB6A53601A4B00221A61194B98
S31508026A1000229A60174809F051FC034687F833307A
S31508026A2097F83330002B18D1124809F0A9FC03460F
S31508026A3087F8333097F83330002B0ED17B680F2B4B
S31508026A4008D8002279687A2001F07EFE0B4A7B6814
S31508026A50136002E0012387F833307A2001F08EFEB4
S31508026A6097F8333018463837BD4680BD000C0244C5
S31508026A70C55A7C0A4CDA002000200040CC110020BE
S31508026A8080B400AF00BFFDE780B400AF00BFFDE7EA
S31508026A9080B400AF00BFFDE780B400AF00BFFDE7DA
S31508026AA080B400AF00BFFDE780B400AF00BFBD46AB
S31508026AB05DF8047B7047000080B500AF024802F01B
S31508026AC0EFFB00BF80BD00BF74D7002080B500AFC2
S31508026AD002480BF02FFB00BF80BD00BF1CD9002067
S31508026AE080B500AF024809F069FF00BF80BD00BF4C
S31508026AF04CDA002080B400AF01231846BD465DF883
S31508026B00047B704780B582B000AF7860396014F0B4
S31508026B104BFE034616221A604FF0FF331846083713
S31508026B20BD4680BD80B582B000AF78604FF0FF31B8
S31508026B307868FFF7E7FF00BFFDE780B586B000AFCC
S31508026B40F860B9607A6000237B610AE0AFF30080DF
S31508026B500146BB685A1CBA60CAB21A707B6901330D
S31508026B607B617A697B689A42F0DB7B68184618373C
S31508026B70BD4680BD80B586B000AFF860B9607A6060
S31508026B8000237B6109E0BB685A1CBA601B78184669
S31508026B90AFF300807B6901337B617A697B689A422D
S31508026BA0F1DB7B6818461837BD4680BD80B483B0D2
S31508026BB000AF78604FF0FF3318460C37BD465DF8D4
S31508026BC0047B704780B483B000AF786039603B6855
S31508026BD04FF400525A60002318460C37BD465DF83A
S31508026BE0047B704780B483B000AF786001231846EF
S31508026BF00C37BD465DF8047B704780B485B000AF9C
S31508026C00F860B9607A60002318461437BD465DF805
S31508026C10047B704780B500AF184B1B78DBB2002B9C
S31508026C2029D1164B01221A70FC220021144814F0AD
S31508026C3047FD12F07DFA03461B0A9BB2DBB2092B0B
S31508026C400BDD01210E4800F021F80120FCF702F9BC
S31508026C5017210C4801F0DAF90AE00021084800F089
S31508026C6015F80020FCF7F6F81421074801F0CEF9CA
S31508026C700120FCF7EFF8024B184680BD94DB002092
S31508026C8098DA0020C80F0408E00F040880B483B01D
S31508026C9000AF78600B46FB707B68FA781A7500BFFE
S31508026CA00C37BD465DF8047B704780B483B000AFED
S31508026CB078607B6818460C37BD465DF8047B7047DA
S31508026CC080B483B000AF78607B685B7D18460C376A
S31508026CD0BD465DF8047B704780B483B000AF786028
S31508026CE07B6801225A75012318460C37BD465DF8A2
S31508026CF0047B704780B483B000AF78607B68DB7D25
S31508026D0018460C37BD465DF8047B704780B483B0DD
S31508026D1000AF78600B46FB707B68FA78DA7500BFBD
S31508026D200C37BD465DF8047B704780B483B000AF6C
S31508026D3078607B681B7E18460C37BD465DF8047B77
S31508026D40704780B483B000AF78607B6801221A76F8
S31508026D5000BF0C37BD465DF8047B704780B485B02A
S31508026D6000AFF8600B4687ED010AFB721346BB7249
S31508026D70BB7A002B08D1FB7AFA6806339B001344C8
S31508026D8004337A681A6016E0BB7A012B08D1FB7ABB
S31508026D90FA6816339B00134404337A681A600AE0C9
S31508026DA0BB7A022B07D1FB7AFA6826339B00134477
S31508026DB004337A681A6000BF1437BD465DF8047B4F
S31508026DC0704780B485B000AFF8607B600B46FB72F3
S31508026DD01346BB72BB7A002B07D1FB7AFA680E33CD
S31508026DE09B0013447A685A6014E0BB7A012B07D1D8
S31508026DF0FB7AFA681E339B0013447A685A6009E0E4
S31508026E00BB7A022B06D1FB7AFA682E339B0013440F
S31508026E107A685A6000BF1437BD465DF8047B70472E
S31508026E2080B483B000AF78607B6893F8DC3018468C
S31508026E300C37BD465DF8047B704780B483B000AF5B
S31508026E4078600B46FB707B68FA7883F8DC2000BF13
S31508026E500C37BD465DF8047B704780B584B000AF39
S31508026E6078607868FFF7DCFF0346FB73FB7B002B31
S31508026E7007D0FB7B013BFB73FB7B19467868FFF760
S31508026E80DCFFFB7B18461037BD4680BD80B485B053
S31508026E9000AF78600B46FB70FB78002B01D100230C
S31508026EA00BE07B6893F8DD20FB781340DBB2002BFE
S31508026EB014BF01230023FB73FB7B18461437BD4618
S31508026EC05DF8047B704780B483B000AF78600B46E8
S31508026ED0FB70FB78002B01D100230BE07B6893F84B
S31508026EE0DD20FB781343DAB27B6883F8DD207B6802
S31508026EF093F8DD3018460C37BD465DF8047B7047BB
S31508026F0080B483B000AF78600B46FB70FB78002B29
S31508026F1001D1002310E07B6893F8DD305AB297F965
S31508026F200330DB435BB213405BB2DAB27B6883F8A9
S31508026F30DD207B6893F8DD3018460C37BD465DF8D0
S31508026F40047B704780B483B000AF78600B46FB7051
S31508026F50FB78002B01D1002310E07B6893F8DE3022
S31508026F605AB297F90330DB435BB213405BB2DAB22B
S31508026F707B6883F8DE207B6893F8DE3018460C3788
S31508026F80BD465DF8047B704780B582B000AF786075
S31508026F9001217868FFF7D6FF02217868FFF7D2FF4A
S31508026FA004217868FFF7CEFF08217868FFF7CAFF41
S31508026FB000BF0837BD4680BD80B483B000AF786095
S31508026FC00B467B807B687A88A3F8E22000BF0C37E1
S31508026FD0BD465DF8047B704780B483B000AF786025
S31508026FE07B68B3F8E23018460C37BD465DF8047B79
S31508026FF0704780B483B000AF78600B46FB707B683D
S31508027000FA7883F8E42000BF0C37BD465DF8047BA6
S31508027010704780B483B000AF78600B46FB70FB788C
S315080270209AB27B68A3F8E02000BF0C37BD465DF82C
S31508027030047B704780B483B000AF78600B46FB7060
S315080270407B68FA7883F8E52000BF0C37BD465DF801
S31508027050047B704780B483B000AF78607B6893F88E
S31508027060E53018460C37BD465DF8047B704780B498
S3150802707083B000AF78600B46FB707B68FA7883F8BA
S31508027080E62000BF0C37BD465DF8047B704780B426
S3150802709083B000AF78600B46FB707B68FA7883F89A
S315080270A0E72000BF0C37BD465DF8047B704780B405
S315080270B083B000AF78607B6893F8E73018460C37E0
S315080270C0BD465DF8047B704780B485B000AFF860B2
S315080270D087ED020AD7ED027AFCEEE77AC7ED017A66
S315080270E03B79DAB2FB6883F8E92000BF1437BD465C
S315080270F05DF8047B704780B485B000AFF86087ED11
S31508027100020AD7ED027AFCEEE77AC7ED017A3B79F5
S31508027110DAB2FB6883F8EA2000BF1437BD465DF889
S31508027120047B704780B485B000AFF86087ED020A29
S31508027130D7ED027AFCEEE77AC7ED017A3B79DAB245
S31508027140FB6883F8EB2000BF1437BD465DF8047B65
S31508027150704780B483B000AF78600B46FB707B68DB
S31508027160FA7883F8EC2000BF0C37BD465DF8047B3D
S31508027170704780B483B000AF78607B6893F8EC30D0
S3150802718018460C37BD465DF8047B704780B483B059
S3150802719000AF78600B46FB707B68FA7883F8ED20BF
S315080271A000BF0C37BD465DF8047B704780B483B0D8
S315080271B000AF78607B6893F8ED3018460C37BD4609
S315080271C05DF8047B704780B483B000AF78600B46E5
S315080271D07B807B687A88A3F8EE2000BF0C37BD4611
S315080271E05DF8047B704780B483B000AF78607B6833
S315080271F0B3F8EE3001339AB27B68A3F8EE207B68C7
S31508027200B3F8EE3018460C37BD465DF8047B704776
S3150802721080B483B000AF78600B46FB707B68FA785F
S3150802722083F8F02000BF0C37BD465DF8047B704733
S3150802723080B483B000AF78607B6893F8F030184664
S315080272400C37BD465DF8047B704780B483B000AF47
S3150802725078600B46FB707B68FA7883F8F12000BFEA
S315080272600C37BD465DF8047B704780B483B000AF27
S3150802727078607B6893F8F13018460C37BD465DF89E
S31508027280047B704780B483B000AF78600B467B807E
S315080272907B687A88A3F8F22000BF0C37BD465DF8F2
S315080272A0047B704780B483B000AF78607B68B3F81C
S315080272B0F23001339AB27B68A3F8F2207B68B3F8FE
S315080272C0F23018460C37BD465DF8047B704780B429
S315080272D083B000AF78600B46FB707B68FA7883F858
S315080272E0F42000BF0C37BD465DF8047B704780B4B6
S315080272F083B000AF78607B6893F8F43018460C3791
S31508027300BD465DF8047B704780B483B000AF7860F1
S315080273100B46FB707B68FA7883F8F52000BF0C37BA
S31508027320BD465DF8047B704780B483B000AF7860D1
S315080273307B6893F8F53018460C37BD465DF8047B32
S31508027340704780B483B000AF78600B46FB707B68E9
S31508027350FA7883F8F62000BF0C37BD465DF8047B41
S31508027360704780B483B000AF78607B6893F8F630D4
S3150802737018460C37BD465DF8047B704780B483B067
S3150802738000AF78600B46FB707B68FA7883F8F720C3
S3150802739000BF0C37BD465DF8047B704780B483B0E6
S315080273A000AF78607B6893F8F73018460C37BD460D
S315080273B05DF8047B704780B483B000AF78600B46F3
S315080273C0FB707B68FA7883F8F82000BF0C37BD4655
S315080273D05DF8047B704780B483B000AF78607B6841
S315080273E093F8F83018460C37BD465DF8047B7047AB
S315080273F080B483B000AF78600B46FB707B68FA787E
S3150802740083F8F92000BF0C37BD465DF8047B704748
S3150802741080B483B000AF78607B6893F8F930184679
S315080274200C37BD465DF8047B7047000080B586B010
S3150802743000AF7860144A154BD31A7B617B693B61AE
S31508027440134B1B68002B02D1114B124A1A60104BC0
S315080274501A687B6813443A699A4207D214F0A4F967
S3150802746003460C221A604FF0FF3309E0084B1B68EB
S31508027470FB60074B1A687B681344054A1360FB686E
S3150802748018461837BD4680BD00000A2000040000D1
S3150802749098DB002060FA002080B483B000AF354B39
S315080274A0D3F88830334A43F47003C2F88830324B33
S315080274B001221A60304B0022DA612F4B00221A622F
S315080274C02D4B1A682C492D4B13400B602A4B002270
S315080274D09A62294B0022DA62274B00221A63264B4C
S315080274E0274A5A63244B00229A63234B244ADA63B7
S315080274F0214B00221A64204B214A5A641E4B002251
S315080275009A641D4B1B681C4A23F4802313601A4B8A
S3150802751000221A65174B4FF000629A60194B9B6955
S3150802752003F060437B607B68B3F1604F03D07B68EE
S31508027530B3F1404F17D1134BDB6903F00103002B5C
S3150802754005D0104B104ADA600E4B104ADA600D4B22
S31508027550DB690C4A43F00203D3610A4BDB69094A29
S3150802756043F00103D36100BF0C37BD465DF8047BC7
S31508027570704700BF00ED00E0000C0244E3EAE2EACD
S3150802758080020101002002403B2A19087F6E5D4CE9
S31508027590B0B5A2B000AF11F04BFC0346184611F085
S315080275A05DFC0346002B36D03B1D0121184610F020
S315080275B0F0FD3B1D0121184610F006FE11F038FCBD
S315080275C00346184611F072FC02463B1D1146184640
S315080275D010F01AFE07F144023B1D1146184610F038
S315080275E072FE10F071F9044607F14403184610F0CA
S315080275F01BFE054607F14403184610F021FE034612
S315080276001A462946204612F087FA11F011FC03465B
S31508027610184611F03DFC0A4B1B685A1C08490A60B9
S31508027620632B08D911F004FC0346184611F022FC14
S31508027630034B00221A6000BF8837BD46B0BD00BFA3
S3150802764000DE002080B500AFFFF7E4FA03461846CD
S31508027650FFF74DFE034619461E4810F0E5FEFFF7F2
S31508027660D9FA03461846FFF75FFE03461946194834
S3150802767010F0F5FEFFF7CEFA03461846FFF771FE3D
S3150802768003461946134810F005FFFFF7C3FA0346E7
S315080276901846FFF783FE034619460E4810F015FFF3
S315080276A0FFF7B8FA03461846FFF795FE034619464A
S315080276B0084810F025FF0849064810F0BAFF10F0EE
S315080276C069F80346044A12780449184612F056F92C
S315080276D000BF80BDE8DD00209CDB00209DDB00208A
S315080276E0B0B582B000AF104B1A883B1D114618463A
S315080276F010F07FFE3B1D0D49184610F07BFF10F077
S3150802770064F80446094810F00AFF0546074810F0CF
S3150802771012FF03461A462946204612F0FDF900BF13
S315080277200837BD46B0BD00BFEEDD00209CDB002059
S3150802773080B500AF064B1B680133054A1360044B3C
S315080277401B68322B01DCFBF7ABFF00BF80BD00BF15
S31508027750FCDD00202DE9F04182B002AF6C4B1B68BC
S3150802776001336B4A13606A4B1B68002B58DB684B64
S315080277701B6841F28832934252DC664B1B78002B17
S3150802778040F0C180644800F07DFC0421634802F0A1
S31508027790AFFC0346012B0CBF01230023DBB21D46B7
S315080277A002215E4802F0A4FC0346012B0CBF01230A
S315080277B00023DBB21E464FF48051594802F098FC6A
S315080277C00346012B0CBF01230023DBB298464FF474
S315080277D00061534802F08CFC0346012B0CBF0123BF
S315080277E00023DBB21C4601214C4802F081FC034609
S315080277F0012B0CBF01230023DBB2019300944346FD
S3150802780032462946474800F03DFCFDF729FB034668
S3150802781001211846FDF76DFB3E4B01221A7072E0F4
S315080278203B4B1B6841F28832934257DD384B1B6843
S3150802783042F21072934251DC364B1B78012B62D10D
S31508027840394800F01FFC0421344802F051FC034673
S31508027850012B0CBF01230023DBB21D4602212F4850
S3150802786002F046FC0346012B0CBF01230023DBB2C0
S315080278701E464FF480512A4802F03AFC0346012B71
S315080278800CBF01230023DBB298464FF4006124485B
S3150802789002F02EFC0346012B0CBF01230023DBB2A8
S315080278A01C4601211D4802F023FC0346012B0CBF8E
S315080278B001230023DBB2019300944346324629464C
S315080278C0184800F0DFFBFDF7CBFA034602211846FB
S315080278D0FDF70FFB0F4B00221A7014E00C4B1B68C6
S315080278E042F2107293420EDD094B00221A600F4BC8
S315080278F01B6801330D4A13600C4B1B6819460C486A
S3150802790000F0C0FBFFE700BFBD46BDE8F08100BF3F
S31508027910F0DD0020F4DD0020D8100408000402423D
S3150802792000140242F010040848110408F8DD002089
S315080279306011040890B585B000AF78607B687B73E8
S31508027940FEF78EFD034600211846FEF79FFDFFF758
S3150802795061F9034600211846FFF74AFD0023FB7327
S315080279600023BB60A54B1B8801339AB2A34B1A802E
S315080279707B7B1846FCF7D4FAFDF764FDFDF776FB28
S31508027980FDF7D3FA9E4B1B78012B49D1FDF7AEFCC6
S31508027990B860BB68012B2DD19A4800F0D9FB984BE9
S315080279A000221A70FFF736F9034601211846FFF737
S315080279B08EFC954995480EF00CFA93480EF0D6F9C6
S315080279C0044691480EF0DEF9034619462046FCF7AE
S315080279D0C9FB01218E4810F0F1FC8E498C4810F043
S315080279E0EAFD0FF0FFFE8B4B1B781A468A4912F006
S315080279F093F815E0BB68002B12DA814B00221A7045
S31508027A000121834810F0DAFC8249814810F0D3FD3F
S31508027A100FF0E8FE7F4B1B781A467F4912F07CF876
S31508027A20FDF71EFA03461846FDF757FA0346012BD9
S31508027A3002D1FFF78FFE16E0FDF712FA0346184643
S31508027A40FDF74BFA0346052B0DD1FDF709FA034656
S31508027A5000211846FDF732FAFFF76AFEFBF748FEE1
S31508027A606E4800F00FFBFBF7FBF8FBF75BF8FAF73B
S31508027A7009FFFBF78DF8FBF7A3FFFCF769F8FCF79C
S31508027A80FDF8FCF791F95D4B1B88654AA2FB0312C8
S31508027A905209642101FB02F29B1A9BB2002B16D1F2
S31508027AA07B7B184600F06EFCFCF7BCFAFFF7B2F8CF
S31508027AB003461846FFF7B4F90346002B05D0FFF72D
S31508027AC0A9F803461846FFF7C8F9FFF761FD4B4BBD
S31508027AD01B88544AA2FB031252094FF4FA7101FB9E
S31508027AE002F29B1A9BB2002B01D1FFF7ABFD434B67
S31508027AF01B884C4AA2FB031292094FF47A7101FBC6
S31508027B0002F29B1A9BB2002B5AD1474B1B880133B0
S31508027B109AB2454B1A80FB7B0133FB73FFF77AF85F
S31508027B2003461846FFF7E6F80346002B2DD0FFF763
S31508027B3071F803461846FFF7DDF80346012B0ED106
S31508027B40FFF768F8034602211846FFF7DFF8FEF743
S31508027B5087FC034600211846FEF798FC15E0FFF756
S31508027B6059F803461846FFF7C5F80346022B0CD107
S31508027B70FFF750F8034600211846FFF7C7F8FFF744
S31508027B8049F803461846FFF7A7F80023BB730023F4
S31508027B90BB7309E0FFF73EF8034601211846FFF7D3
S31508027BA075F9BB7B0133BB73BB7B072BF2D9002369
S31508027BB0BB7302E0BB7B0133BB73BB7B072BF9D9D3
S31508027BC00E4B1B88194AA2FB0312120B43F6982185
S31508027BD001FB02F29B1A9BB2002B04D1074B00222F
S31508027BE01A80FBF749FCFB7B3B2B03D90023FB736B
S31508027BF0FFF776FD01200DF027F8B3E604DE002034
S31508027C0032DA002074110408E4DB00208C1104081F
S31508027C10E0DB00209CDB00209DDB0020AC11040881
S31508027C201F85EB51D34D6210EEDD002073B2E74596
S31508027C3080B58EB008AF78607B687B6107F10C016E
S31508027C40002340F6FF7278690DF094FD0346002B77
S31508027C5001D0022323E000233B61062218211248A1
S31508027C6000F0E6FA03463B61FB68B022069201225F
S31508027C700592002204920A2203920A22029240F6EE
S31508027C80FF72019200933B69084A074908480DF0BA
S31508027C907BFF0346002B01D00E2300E00023184683
S31508027CA01837BD4680BD00BFC411040835790208DD
S31508027CB000A0002080B584B000AF78607B68FB60C6
S31508027CC0FB68DBB21846F9F7B3FBFB68DBB218466A
S31508027CD000F0D4F8FB68DBB2184600F053FB6420C8
S31508027CE00CF0B2FF00BFF0E780B58EB008AF78603F
S31508027CF07B687B6107F10C0100234FF40062786907
S31508027D000DF038FD0346002B01D0022323E00023A1
S31508027D103B6106221421124800F08AFA03463B61A7
S31508027D20FB68B022069201220592002204920A22D8
S31508027D3003920A2202924FF40062019200933B696F
S31508027D40084A074908480DF01FFF0346002B01D0D1
S31508027D500E2300E0002318461837BD4680BD00BF33
S31508027D60E0110408B57C0208A09E002080B584B004
S31508027D7000AF78607B68FB60FEF74CFF0346802104
S31508027D801846FFF7A0F8FB68DBB2184600F0EEF8D3
S31508027D90FB68DBB2184611F09FFB0D4B1B880133BB
S31508027DA09AB20B4B1A800A4B1B88632B0BD9084BCA
S31508027DB000221A8011F09AFD11F0AAFCFB68DBB2C8
S31508027DC0184600F0DFFA01200CF03EFFDBE700BFA1
S31508027DD006DE002080B58EB008AF78607B687B61CE
S31508027DE007F10C01002340F6FF7278690DF0C2FC18
S31508027DF00346002B01D0022323E000233B6106221F
S31508027E001421124800F014FA03463B61FB68B022BB
S31508027E10069201220592002204920A2203920A225B
S31508027E20029240F6FF72019200933B69084A07499B
S31508027E3008480DF0A9FE0346002B01D00E2300E0E8
S31508027E40002318461837BD4680BD00BFF81104083E
S31508027E506D7D0208509F002080B582B000AF0346B0
S31508027E60FB71FB1D0122194603480EF0C7FA00BF33
S31508027E700837BD4680BD00BF08DE002080B584B045
S31508027E8000AF0346FB710023FB7322480EF09AFAF1
S31508027E90034683F00103DBB2002B15D009E0FB7B16
S31508027EA01846FAF721F90023FB73FB79184600F006
S31508027EB069FA07F10F030122194616480EF0D9FA94
S31508027EC00346002BEBD120E013480AF027FC0346B1
S31508027ED0202B0DD1104B0122A3F85C200E4B012258
S31508027EE0A3F85E2001220D490B480AF00DF80CE0B2
S31508027EF0094BB3F85C20084BB3F85E309BB29A4242
S31508027F0003D0FCF7C9F9FCF7D3F900BF1037BD4611
S31508027F1080BD00BF08DE00201CD90020AAE400208C
S31508027F2080B582B000AF78600B467B800D480EF0B4
S31508027F30EBF902467B889A420FD34FF0FF310A4883
S31508027F400DF0C2FD7B881A46796806480EF056FA85
S31508027F5005480DF0FBFD012300E00023184608370B
S31508027F60BD4680BD18DE0020B0A0002080B5ADF564
S31508027F70826D00AF024607F58263A3F209431A70BF
S31508027F800023A7F80E342BE007F10C034FF48062A6
S31508027F900021184613F094FB4FF0FF3118480DF0F4
S31508027FA093FD07F10C034FF48062194615480EF04B
S31508027FB060FA0346A7F80E3411480DF0C7FDB7F864
S31508027FC00E2407F10C014FF47A730F4809F0FDFEEF
S31508027FD007F58263A3F209431B78184600F0D2F923
S31508027FE008480EF0EFF9034683F00103DBB2002BD3
S31508027FF0CAD100BF00BF07F58267BD4680BD00BF74
S31508028000B0A0002018DE00201CD9002080B582B05E
S3150802801000AF78600B467B807A884FF47A7379686A
S31508028020034809F0D2FE012318460837BD4680BD2B
S315080280301CD9002080B500AF8022064906480EF0FA
S3150802804037F94FF48062054905480EF031F900BF49
S3150802805080BD00BF28DE002008DE0020A8DE002042
S3150802806018DE002080B500AFFFF7E4FF01220349BE
S31508028070034809F049FF00BF80BD00BFAAE40020FB
S315080280801CD900200FB480B582B000AFFEF7C2FD3E
S31508028090034680211846FEF7F9FE034683F00103DC
S315080280A0DBB2002B01D0002325E04FF481720021B8
S315080280B0144813F005FB4FF480720021124813F09E
S315080280C0FFFA07F114033B603A6839690E4813F060
S315080280D0DDFA78600C4A0D490A4813F05DFA094838
S315080280E0F8F7F4F903469BB219460648FFF718FF54
S315080280F003467B607B6818460837BD46BDE8804064
S3150802810004B07047B0E40020B4E500201012040859
S3150802811080B582B000AF78607B681B68094A9342D3
S315080281200CD1094B1B781846FFF796FE064B002220
S315080281301A7001220449054809F0E6FE00BF08370D
S31508028140BD4680BD00380140AAE400201CD90020A3
S315080281500FB490B583B000AFFEF75CFD03468021ED
S315080281601846FEF793FE034683F00103DBB2002BA3
S3150802817001D000232EE04FF481720021194813F032
S315080281809FFA4FF480720021174813F099FA07F103
S315080281901C033B603A68B969134813F077FA7860AA
S315080281A0114A12490F4813F0F7F90E491048FFF71A
S315080281B069FF10490B480DF00CFE0E480DF0D6FD6E
S315080281C004460C480DF0DEFD034619462046FBF729
S315080281D0C9FF7B6818460C37BD46BDE8904004B017
S315080281E0704700BFB4E60020B8E700201012040862
S315080281F014120408A8E2002080B582B000AF7860A5
S3150802820078680AF0A0FA0346074A13607B681B6877
S31508028210064A934203D1FCF73FF8FCF749F800BF38
S315080282200837BD4680BD00BFACE4002000380140D7
S3150802823080B584B000AF78600B46FB701346BB70FE
S31508028240FF23FB73484B1B780B2B77D8FB78202B25
S315080282500ED8454B1B781A4613461B0113445B007E
S31508028260424A1344FA787968184613F0E0FA0DE0A0
S315080282703D4B1B781A4613461B0113445B003B4AC7
S31508028280134420227968184613F0D1FA364B1B7824
S315080282901946364A0B461B010B445B00134420332E
S315080282A0BA781A70304B1B7818462F4B1B7819462A
S315080282B02E4A03461B0103445B00134420331878F5
S315080282C02A4A0B461B010B445B0013442133024620
S315080282D01A70254B1B785A1CD1B2234A1170FB73AC
S315080282E01D212348FFF792FE07F10C030322002102
S315080282F0184613F0E5F9FA7B07F10C031D491846EF
S3150802830013F04AF907F10C031846F8F7DFF80346A3
S315080283109AB207F10C0311461846FFF777FE0221B7
S315080283201548FFF773FEFB789BB219467868FFF784
S315080283306DFE02211148FFF769FE0FE0FF23FB736A
S3150802834034210F48FFF762FEFB789BB2194678681C
S31508028350FFF75CFE02210948FFF758FEFB7B184629
S315080283601037BD4680BD00BF50EA0020B8E800209D
S315080283701C1204083C120408401204084412040899
S315080283804812040880B582B000AF0346FB71114B50
S315080283901B78FA799A4213D2F979FA790E480B467A
S315080283A01B010B445B000344203318780A49134621
S315080283B01B0113445B000B44213302461A7004E086
S315080283C0FB7919460548FFF75DFE00BF0837BD462B
S315080283D080BD00BF50EA0020B8E8002080120408D9
S315080283E080B582B000AF0023FB710023BB712A4B14
S315080283F01B78002B4BD10023FB7136E0FA7927490B
S3150802840013461B0113445B000B4421331B78002BD4
S3150802841017D0FA79214913461B0113445B000B4412
S3150802842021331B78BB71BB79013BBB71FA791B49B6
S3150802843013461B0113445B000B442133BA791A70A5
S3150802844010E0FA7913461B0113445B00134A1344DE
S3150802845019461348FFF716FE1248FFF713FE0E4B8E
S3150802846001221A70FB790133FB710F4B1B78FA79DB
S315080284709A42C3D3FEF7CEFB03461846FEF720FC04
S315080284800346002B04D1094801F004FF00E000BFAF
S315080284900837BD4680BD00BF51EA0020B8E8002073
S315080284A0B8120408E412040850EA0020D8D70020BB
S315080284B00D488546FEF7F0FF0C480D490D4A002384
S315080284C002E0D458C4500433C4188C42F9D30A4A79
S315080284D00A4C002301E013600432A242FBD313F0D4
S315080284E069F9FBF7EDFEFEE700000A20000000200E
S315080284F0BC130020201D0408BC1300205CFA0020CF
S31508028500FEE7000080B500AF032000F012F902F082
S31508028510C1FC02460B4B1B6A03F00F030A49CB5CEC
S3150802852022FA03F3094A13600F20FEF733FA0346C9
S31508028530002B01D0012302E0FDF7B7FF00231846FE
S3150802854080BD00BF000C024468180408C811002048
S3150802855080B400AF064B1B781A46064B1B681344B9
S31508028560044A136000BFBD465DF8047B704700BF2E
S31508028570D011002054EA002080B400AF034B1B68D8
S315080285801846BD465DF8047B704700BF54EA0020D2
S3150802859080B485B000AF78607B6803F00703FB60A0
S315080285A00C4BDB68BB60BA684FF6FF031340BB602F
S315080285B0FB681A02BB68134343F0BF6343F40033F4
S315080285C0BB60044ABB68D36000BF1437BD465DF87A
S315080285D0047B704700ED00E080B400AF044BDB6813
S315080285E01B0A03F007031846BD465DF8047B70476D
S315080285F000ED00E080B483B000AF0346FB80B7F914
S315080286000630002B0BDBFB8803F01F020749B7F97C
S3150802861006305B09012000FA02F241F8232000BF66
S315080286200C37BD465DF8047B704700BF00E100E0E9
S3150802863080B483B000AF0346FB80B7F90630002B3F
S3150802864012DBFB8803F01F020A49B7F906305B09F9
S31508028650012000FA02F2203341F82320BFF34F8F9C
S3150802866000BFBFF36F8F00BF00BF0C37BD465DF872
S31508028670047B704700E100E080B483B000AF034694
S315080286803960FB80B7F90630002B0ADB3B68DAB2A1
S315080286900C49B7F906301201D2B20B4483F800230B
S315080286A00AE03B68DAB20849FB8803F00F03043B89
S315080286B01201D2B20B441A7600BF0C37BD465DF8DA
S315080286C0047B704700E100E000ED00E080B489B069
S315080286D000AFF860B9607A60FB6803F00703FB61D4
S315080286E0FB69C3F10703042B28BF0423BB61FB699B
S315080286F00433062B02D9FB69033B00E000237B61A6
S315080287004FF0FF32BB6902FA03F3DA43BB681A4039
S315080287107B699A404FF0FF317B6901FA03F3D9432B
S315080287207B680B40134318462437BD465DF8047B25
S31508028730704780B582B000AF78607868FFF728FF87
S3150802874000BF0837BD4680BD80B586B000AF034678
S31508028750B9607A60FB81FFF73FFF78617A68B9688A
S315080287607869FFF7B3FF0246B7F90E301146184685
S31508028770FFF782FF00BF1837BD4680BD80B582B0BD
S3150802878000AF0346FB80B7F906301846FFF732FFFB
S3150802879000BF0837BD4680BD80B582B000AF03462C
S315080287A0FB80B7F906301846FFF742FF00BF0837C5
S315080287B0BD4680BD80B584B000AF7860FFF7DCFEA9
S315080287C0F8607B68002B01D101236BE07B6893F884
S315080287D05430DBB2022B08D07B6820229A657B686C
S315080287E0002283F84C2001235CE07B681B685A69E7
S315080287F07B681B6842F004025A617B68052283F88B
S31508028800542020E0FFF7B8FE0246FB68D31A052B70
S3150802881019D97B689B6D43F010027B689A657B6861
S31508028820032283F854207B681B6D03F08003002B18
S3150802883003D07B685B6F01221A737B68002283F878
S315080288404C2001232EE07B681B681B6903F4005346
S31508028850002BD7D07B681B685A697B681B6842F075
S3150802886002025A617B68042283F854207B681B68DB
S315080288704FF4FE42DA607B68012283F854207B6853
S315080288801B6D03F08003002B07D07B685B6F012208
S315080288901A737B681B6800229A647B68002283F835
S315080288A04C20002318461037BD4680BD80B483B0DD
S315080288B000AF78607B68002B01D1012319E07B6841
S315080288C093F85430DBB2022B04D07B6820229A65D7
S315080288D001230EE07B68042283F854207B681B6818
S315080288E05B697A68126843F4005343F004035361E0
S315080288F0002318460C37BD465DF8047B7047000016
S3150802890080B584B000AF78607B68002B01D1012363
S3150802891047E17B6893F85C30DBB2002B06D17B68B3
S31508028920002283F85D207868FDF7C6FD7B681B6820
S315080289309A697B681B6822F010029A61FFF71CFE8F
S31508028940F86012E0FFF718FE0246FB68D31A0A2BF4
S315080289500BD97B681B6E43F001027B681A667B683B
S31508028960032283F85C2001231BE17B681B689B6951
S3150802897003F00803082BE5D07B681B689A697B68B5
S315080289801B6842F001029A61FFF7F6FDF86012E0F1
S31508028990FFF7F2FD0246FB68D31A0A2B0BD97B684E
S315080289A01B6E43F001027B681A667B68032283F812
S315080289B05C200123F5E07B681B689B6903F00103D1
S315080289C0002BE5D07B681B689A697B681B6842F0B6
S315080289D002029A617B681B68744A934203D1744AFD
S315080289E07B685B6813607B681B7C012B08D17B68FC
S315080289F01B689A697B681B6822F040029A6107E045
S31508028A007B681B689A697B681B6842F040029A6118
S31508028A107B685B7C012B08D17B681B689A697B683B
S31508028A201B6842F480429A6107E07B681B689A6970
S31508028A307B681B6822F480429A617B689B7C012BC7
S31508028A4008D17B681B689A697B681B6822F4805286
S31508028A509A6107E07B681B689A697B681B6842F41F
S31508028A6080529A617B681B689B6923F440717B6814
S31508028A709A687B681B680A439A617B681B689A69CD
S31508028A807B681B6822F0A4029A617B681B681A69D4
S31508028A907B681B6822F010021A617B68DB68012B6F
S31508028AA008D17B681B689A697B681B6842F00402D6
S31508028AB09A612CE07B68DB68002B28D07B68DB6830
S31508028AC0022B1CD07B681B689A697B681B6842F07C
S31508028AD080029A617B681B681A697B681B6842F088
S31508028AE010021A617B68DB68032B10D17B681B684E
S31508028AF09A697B681B6842F020029A6107E07B68E4
S31508028B001B689A697B681B6842F020029A617B6837
S31508028B109B69013B5A067B68DB69013B1B021A43C8
S31508028B207B681B6A013B42EA03017B685B69013B7E
S31508028B301A047B681B680A43DA617B689B68B3F58B
S31508028B40407F15D17B689B6A5A1E7B68DB6A013BAC
S31508028B501B021A437B681B6B013B1B0142EA03019A
S31508028B607B685B6A013B1A047B681B680A43DA6006
S31508028B707B681B68D3F8C0107B68DA6B7B681B6856
S31508028B800A43C3F8C020786800F018FD7B68002203
S31508028B909A657B6800221A667B68012283F85C2044
S31508028BA0002318461037BD4680BD00BF00A400400A
S31508028BB000A5004080B487B000AF786039607B6852
S31508028BC093F85C30FB75FB7D012B02D0FB7D022BF3
S31508028BD03DD13B681B68002B19D13B689B689A07F5
S31508028BE03B68DB68DB061A433B681B691B041A43AE
S31508028BF03B685B6913433B617B681A6C3B685B683D
S31508028C009B001344BB60BB683A691A601DE03B6867
S31508028C10DB685A073B681B6913433B613B689B68E1
S31508028C209A073B685B691343FB607B685A6C3B682F
S31508028C305B68DB001344BB60BB683A691A60BB68B1
S31508028C400433BB60BB68FA681A60002306E07B68D7
S31508028C501B6E43F002027B681A66012318461C370C
S31508028C60BD465DF8047B704780B485B000AFF860F6
S31508028C70B9607A603B60FB6893F85C30DBB2012B23
S31508028C8016D1FB681B68D3F8803023F03F01BB6816
S31508028C901A017B689B001A433B685B001A43BB694F
S31508028CA01A43FB681B680A43C3F88020002306E0C0
S31508028CB0FB681B6E43F00402FB681A66012318461A
S31508028CC01437BD465DF8047B704780B483B000AFA5
S31508028CD078607B6893F85C30DBB2012B10D17B6835
S31508028CE0022283F85C207B681B689A697B681B688A
S31508028CF022F001029A617B6800221A66002306E0C6
S31508028D007B681B6E43F004027B681A6601231846C9
S31508028D100C37BD465DF8047B704780B586B000AF58
S31508028D20F860B9607A60FB6893F85C30DBB2022BB4
S31508028D302CD1FB681B68D3F8C43003F40013002B4C
S31508028D4007D0FB681B6E43F40072FB681A660123A0
S31508028D5023E0FB681B68D3F8C4301B0C03F003033B
S31508028D607B617B697A68B968F86800F089FCFB68F8
S31508028D701B6801217A6901FA02F2C3F8CC200122A2
S31508028D807B699A40FB689A65002306E0FB681B6EBE
S31508028D9043F00802FB681A66012318461837BD46CF
S31508028DA080BD80B483B000AF78607B689B6D18463F
S31508028DB00C37BD465DF8047B704780B483B000AFBC
S31508028DC0786039607B6893F85C30DBB2022B06D197
S31508028DD07B681B683A68C3F8D020002306E07B68E4
S31508028DE01B6E43F008027B681A66012318460C3785
S31508028DF0BD465DF8047B704780B48BB000AFF8605F
S31508028E00B9607A603B600023FB61FB6893F85C30CB
S31508028E10FB76FB7E022B40F0E880BB68402B37D1FD
S31508028E20FB681B68D3F8903003F00F03002B07D1B9
S31508028E30FB681B6E43F48072FB681A660123DBE04B
S31508028E40FB681B68D3F890301B0E03F00103012B55
S31508028E500AD1FB681B68D3F880305B0A03F001036A
S31508028E60012B01D10123FB61FB681B68D3F8903003
S31508028E701B0A03F00303FA691344FB61FB68996C46
S31508028E80FA691346DB001344DB000B447B6236E0C7
S31508028E90FB681B68D3F8983003F00F03002B07D141
S31508028EA0FB681B6E43F48072FB681A660123A3E013
S31508028EB0FB681B68D3F898301B0E03F00103012BDD
S31508028EC00AD1FB681B68D3F880301B0A03F001033A
S31508028ED0012B01D10123FB61FB681B68D3F898308B
S31508028EE01B0A03F00303FA691344FB61FB68D96C96
S31508028EF0FA691346DB001344DB000B447B627B6A88
S31508028F001B6803F080427B685A607B685B68002BAB
S31508028F1007D17B6A1B689B0CC3F30A027B681A603B
S31508028F2005E07B6A1B6823F060427B681A607B6AED
S31508028F301B6803F000527B689A607B6A1B6803F021
S31508028F4000427B681A617B6A04337B627B6A1B6810
S31508028F509AB27B68DA617B6A1B681B0C03F00F0204
S31508028F607B68DA607B6A1B6803F480127B685A6145
S31508028F707B6A1B6803F400127B689A617B6A1B682A
S31508028F801B0E03F07F027B681A627B6A1B68DA0F84
S31508028F907B685A627B6A04337B627B6A7B61002345
S31508028FA03B620AE07A693B6A1A4439683B6A0B44AF
S31508028FB012781A703B6A01333B627B68DB68114A96
S31508028FC0D35C1A463B6A9342ECD3BB68402B05D165
S31508028FD0FB681B68FA69C3F8942004E0FB681B68FF
S31508028FE0FA69C3F89C20002306E0FB681B6E43F06F
S31508028FF00802FB681A66012318462C37BD465DF837
S31508029000047B70478018040880B485B000AF786086
S3150802901039607B681B685B6CFB60FB6803F00702C0
S315080290203B681A60FB681B0A03F007023B685A6032
S31508029030FB6803F018023B689A60FB685B0903F059
S3150802904001023B68DA60FB689B0903F001023B6890
S315080290501A61FB68DB0903F001023B685A61FB6887
S31508029060DB0A03F001023B689A61FB681B0B03F0FB
S3150802907001023B68DA61FB685B0B03F001023B689D
S315080290801A62FB689B0B03F001023B685A62FB6893
S315080290901B0C03F07F023B689A62002318461437BA
S315080290A0BD465DF8047B704780B483B000AF786034
S315080290B039607B681B68D3F8C8203B681340002BCD
S315080290C001D1002300E0012318460C37BD465DF89E
S315080290D0047B704780B487B000AFF860B9607A60E5
S315080290E0FB6893F85C30FB75FB7D012B03D0FB7D97
S315080290F0022B40F0C880FB681B689B6D3B61BB680E
S3150802910003F00703002B04D03B6903F00103002B8D
S315080291103BD0BB6803F03803002B04D03B6903F04D
S315080291200203002B31D0BB6803F4E073002B04D092
S315080291303B6903F00403002B27D0BB6803F4F05302
S31508029140002B04D03B6903F00803002B1DD0BB6833
S3150802915003F46043002B04D03B6903F01003002B91
S3150802916013D0BB6803F44033002B04D03B6903F0E9
S315080291702003002B09D0BB6803F47C03002B0CD018
S315080291803B6903F04003002B07D1FB681B68DA6DC5
S31508029190FB681B6842F00102DA65BB6803F0070345
S315080291A0002B04D03B6903F00103002B3BD1BB68BB
S315080291B003F03803002B04D03B6903F00203002BAB
S315080291C031D1BB6803F4E073002B04D03B6903F08A
S315080291D00403002B27D1BB6803F4F053002B04D0F9
S315080291E03B6903F00803002B1DD1BB6803F46043F7
S315080291F0002B04D03B6903F01003002B13D1BB6884
S3150802920003F44033002B04D03B6903F02003002B00
S3150802921009D1BB6803F47C03002B0CD03B6903F02D
S315080292204003002B07D0FB681B68DA6DFB681B68D6
S3150802923042F00202DA65BB6803F08003002B09D00C
S31508029240FB681B68D3F8DC10FB681B687A680A435C
S31508029250C3F8DC20BB6803F48073002B09D0FB68D3
S315080292601B68D3F8E010FB681B687A680A43C3F8E0
S31508029270E020FB681B68596DFB681B68BA680A43DD
S315080292805A65002306E0FB681B6E43F00202FB6880
S315080292901A66012318461C37BD465DF8047B7047DB
S315080292A080B58CB000AF78607B681B681B6D03F4D1
S315080292B0E053FB627B681B685B6DFA6A1340FB62CC
S315080292C07B681B681B6D03F00703BB627B681B6820
S315080292D05B6DBA6A1340BB627B681B681B6D03F041
S315080292E038037B627B681B685B6D7A6A13407B6214
S315080292F07B681B681B6D03F471033B627B681B6802
S315080293005B6D3A6A13403B627B681B681B6D03F40C
S315080293106023FB617B681B685B6DFA691340FB611E
S315080293207B681B685B6DBB617B681B681B6D7B6119
S315080293307B6903F04003002B0BD0BB6903F04003A3
S31508029340002B06D07B681B6840221A65786800F0F5
S3150802935016F97B6903F48073002B19D0BB6903F4F1
S315080293608073002B14D07B681B68D3F8D8303B6116
S315080293707B681B68D3F8E0303A6913403B617B6827
S315080293801B684FF480721A653969786800F0D8F854
S31508029390FB6A002B07D07B681B68FA6A1A65F96AAA
S315080293A0786800F0A2F8BB6A002B07D07B681B68B6
S315080293B0BA6A1A65B96A7868FBF7CEFB7B6A002B2C
S315080293C007D07B681B687A6A1A65796A786800F03A
S315080293D097F87B6903F40073002B0CD0BB6903F47E
S315080293E00073002B07D07B681B684FF400721A655E
S315080293F0786800F090F87B6903F08003002B18D098
S31508029400BB6903F08003002B13D07B681B68D3F873
S31508029410D430FB607B681B68D3F8DC30FA681340EB
S31508029420FB607B681B6880221A65F968786800F019
S315080294307CF87B6903F40053002B0CD0BB6903F458
S315080294400053002B07D07B681B684FF400521A653D
S31508029450786800F080F87B6903F40043002B0CD08F
S31508029460BB6903F40043002B07D07B681B684FF4E3
S3150802947000421A65786800F078F87B6903F480433D
S31508029480002B0FD0BB6903F48043002B0AD07B68FC
S315080294901B684FF480421A657B681B6E43F0800294
S315080294A07B681A66FB69002B07D07B681B68FA691A
S315080294B01A65F969786800F076F83B6A002B09D0D4
S315080294C07B681B683A6A1A657B681A6E3B6A1A4396
S315080294D07B681A667B681B6E002B02D0786800F0E0
S315080294E058F800BF3037BD4680BD80B483B000AFA0
S315080294F07860396000BF0C37BD465DF8047B70475B
S3150802950080B483B000AF7860396000BF0C37BD46BF
S315080295105DF8047B704780B483B000AF786000BF03
S315080295200C37BD465DF8047B704780B483B000AF44
S315080295307860396000BF0C37BD465DF8047B70471A
S3150802954080B483B000AF7860396000BF0C37BD467F
S315080295505DF8047B704780B483B000AF786000BFC3
S315080295600C37BD465DF8047B704780B483B000AF04
S31508029570786000BF0C37BD465DF8047B704780B43F
S3150802958083B000AF786000BF0C37BD465DF8047B38
S31508029590704780B483B000AF786000BF0C37BD4611
S315080295A05DF8047B704780B483B000AF7860396099
S315080295B000BF0C37BD465DF8047B704780B485B0A2
S315080295C000AF78602C4BBB607B681B682B4A9342C2
S315080295D003D1BB6803F55473BB607B68BA681A6427
S315080295E07B681B68D3F8803023F4F8117B685B6BC1
S315080295F01A047B681B680A43C3F88020BB6803F118
S3150802960070027B685A647B681B68D3F8803023F043
S3150802961070617B689B6B1A067B681B680A43C3F8F2
S315080296208020BB6803F1B0027B689A64BB6803F5C5
S31508029630C4727B68DA64BB6803F518727B681A65BC
S31508029640BB6803F51E727B685A65BB68FB6005E05A
S31508029650FB6800221A60FB680433FB60BB6803F5EB
S315080296605473FA689A42F3D300BF00BF1437BD4653
S315080296705DF8047B704700BF00AC004000A80040BC
S3150802968080B489B000AFF860B9607A603B60BB68A5
S315080296905B68002B0AD1BB681A69BB689B681A43C8
S315080296A0BB681B689B041343FB610AE0BB681A6923
S315080296B0BB689B681A43BB681B68134343F0804325
S315080296C0FB61BB681B6A1A06BB68DB691A43BB687F
S315080296D09B691A43BB685B691A43BB68DB681B0450
S315080296E013433B61FB68596D3A681346DB00134422
S315080296F0DB000B44BB61BB69FA691A60BB690433B8
S31508029700BB61BB693A691A60BB690433BB61002352
S315080297107B6120E07B6903337A6813441B781A0657
S315080297207B69023379680B441B781B041A437B69ED
S31508029730013379680B441B781B02134379687A69EB
S315080297400A4412781A43BB691A60BB690433BB61BF
S315080297507B6904337B61BB68DB68064AD35C1A46BD
S315080297607B699342D6D300BF00BF2437BD465DF856
S31508029770047B70478018040880B588B000AFF8608B
S31508029780B9607A60324B1B78012B01D102235AE069
S315080297902F4B01221A702E4B00225A604FF47A7010
S315080297A000F0A4F80346FB77FB7F002B47D1284A33
S315080297B0FB689360274BBB61FB6823F00043022BCF
S315080297C004D17968B86800F0DFF81BE0FB68224A22
S315080297D0934203D0FB68214A934204D17968B86858
S315080297E000F00EF90EE0FB6823F000431C4A934290
S315080297F004D17968B86800F04FF903E07968B86867
S3150802980000F04AF94FF47A7000F070F80346FB77D5
S31508029810BB691A68FB6823F0304323F00403DB4371
S315080298201A40BB691A60FB680C4A934207D10D4B72
S315080298307B617B691B6823F004027B691A60044B0F
S3150802984000221A70FB7F18462037BD4680BD00BF2E
S31508029850D411002028200240020000100600001041
S31508029860020000404020024080B483B000AF0023CB
S31508029870FB710D4B9B6A03F00103002B0DD00A4BBB
S315080298800A4A5A60084B0A4A5A60074B9B6A03F00F
S315080298900103002B01D00123FB71FB7918460C3713
S315080298A0BD465DF8047B70470020024023016745E8
S315080298B0AB89EFCD80B483B000AF0023FB710A4BAE
S315080298C09B6A094A43F001039362074B9B6A03F0BA
S315080298D00103002B01D10123FB71FB7918460C37D2
S315080298E0BD465DF8047B70470020024080B586B00D
S315080298F000AF7860FEF740FE7861204B3B6110E0CE
S315080299007B68B3F1FF3F0CD0FEF736FE02467B6951
S31508029910D31A7A689A4202D37B68002B01D10323B1
S3150802992027E03B691B6803F00B03002BE8D1144BB5
S31508029930FB603B691B6803F47E03BB60BB68002BB4
S315080299400CD0104B5A68BB6813430E4A5360BB6867
S3150802995003F47E02FB681A6001230AE03B691B686E
S3150802996003F48033002B03D0FB684FF480321A606D
S31508029970002318461837BD4680BD00BF2020024086
S3150802998030200240D411002080B48BB000AF78603A
S315080299903960042387F827307B683B623B68FB61A2
S315080299A0164BBB61BB691B6843F00202BB691A60AE
S315080299B0EFF310833B613B697B6172B600BFFB69BB
S315080299C01A683B6A1A603B6A04333B62FB690433D2
S315080299D0FB6197F82730013B87F8273097F827303D
S315080299E0002BECD17B69FB60FB6883F3108800BF10
S315080299F000BF2C37BD465DF8047B7047282002401D
S31508029A0080B48BB000AF78603960042387F82730BA
S31508029A107B683B623B68FB611C4BBB611C4B7B61F1
S31508029A20BB691B6843F00202BB691A607B691A6844
S31508029A30184B9B6803F004031A437B691A60EFF319
S31508029A401083FB60FB683B6172B600BFFB691A684C
S31508029A503B6A1A603B6A04333B62FB690433FB6167
S31508029A6097F82730013B87F8273097F82730002BDD
S31508029A70ECD13B69BB60BB6883F3108800BF00BFAB
S31508029A802C37BD465DF8047B704700BF282002408C
S31508029A9040200240D411002080B485B000AF78601F
S31508029AA03960094BFB60FB681B6843F00202FB68DE
S31508029AB01A603A687B68128892B21A8000BF143715
S31508029AC0BD465DF8047B70472820024080B586B003
S31508029AD000AF786039603A4B1B78012B01D102231B
S31508029AE06AE0374B01221A70354B00225A604FF44E
S31508029AF07A70FFF7FBFE0346FB75FB7D002B57D1F9
S31508029B007B681B682E4A93602E4BFB607B681B683A
S31508029B1023F0004348F2080293420BD17B685B6844
S31508029B20184600F053F84FF47A70FFF7DFFE034643
S31508029B30FB7533E07B681B68234A934208D100F021
S31508029B40B5F84FF47A70FFF7D1FE0346FB7525E0A8
S31508029B503B684FF0FF321A607B689B683B6115E0F1
S31508029B607B685B681946386900F068F84FF47A70C2
S31508029B70FFF7BCFE0346FB75FB7D002B03D03B6853
S31508029B803A691A600AE03B6901333B617B68DA6825
S31508029B907B689B6813443A699A42E1D3FB681A6860
S31508029BA07B681B6823F00043DB431A40FB681A6094
S31508029BB0034B00221A70FB7D18461837BD4680BD36
S31508029BC0D4110020282002400800008080B485B005
S31508029BD000AF7860184BFB607B6803F00303032B26
S31508029BE008D1FB681B6843F4004343F02003FA6874
S31508029BF013601BE07B6803F00103002B09D0FB68A6
S31508029C001B6823F0004323F0280343F02802FB686D
S31508029C101A607B6803F00203002B07D0FB681B68F7
S31508029C2043F0004343F02803FA68136000BF143771
S31508029C30BD465DF8047B70472820024080B485B093
S31508029C4000AF78603960184BFB603B6803F001038C
S31508029C50002B11D0FB681B6823F0004323F4FE5344
S31508029C60FA681360FB681A687B689B01134343F022
S31508029C702402FB681A6010E0FB681B6823F4FE5294
S31508029C80FB681A60FB681A687B689B01134343F0FA
S31508029C90004343F02403FA68136000BF1437BD4635
S31508029CA05DF8047B704700BF2820024080B483B069
S31508029CB000AF074B7B607B681B6843F008027B6832
S31508029CC01A6000BF0C37BD465DF8047B704700BFBB
S31508029CD04020024080B487B000AF78603960002324
S31508029CE03B6136E13B681A6801213B6901FA03F3D5
S31508029CF01340FB60FB68002B00F028813B685B6819
S31508029D00022B03D03B685B68122B25D13B69DA0824
S31508029D107B68083253F822307B613B6903F00703FC
S31508029D209B000F2202FA03F3DB437A6913407B6135
S31508029D303B681B6903F00F023B6903F007039B00AC
S31508029D4002FA03F37A6913437B613B69DA087B6893
S31508029D500832796943F822107B681B687B613B6984
S31508029D605B00032202FA03F3DB437A6913407B6141
S31508029D703B685B6803F003023B695B0002FA03F384
S31508029D807A6913437B617B687A691A603B685B6808
S31508029D90012B0BD03B685B68022B07D03B685B68DC
S31508029DA0112B03D03B685B68122B30D17B689B680A
S31508029DB07B613B695B00032202FA03F3DB437A69A0
S31508029DC013407B613B68DA683B695B0002FA03F37E
S31508029DD07A6913437B617B687A699A607B685B68F8
S31508029DE07B6101223B6902FA03F3DB437A6913407A
S31508029DF07B613B685B681B0903F001023B6902FA57
S31508029E0003F37A6913437B617B687A695A603B6814
S31508029E105B68032B17D07B68DB687B613B695B0059
S31508029E20032202FA03F3DB437A6913407B613B6838
S31508029E309A683B695B0002FA03F37A6913437B610A
S31508029E407B687A69DA603B685B6803F08053002BAB
S31508029E507CD0474A3B699B08183352F823307B610A
S31508029E603B6903F00303DB000F2202FA03F3DB4329
S31508029E707A6913407B617B689A0A3E4B13403A69BA
S31508029E8002F00302D20093407A6913437B61384990
S31508029E903B699B0818337A6941F82320344B1B68BF
S31508029EA07B61FB68DB437A6913407B613B685B68CD
S31508029EB003F48013002B03D07A69FB6813437B6192
S31508029EC02B4A7B6913602A4B5B687B61FB68DB4321
S31508029ED07A6913407B613B685B6803F40013002BC5
S31508029EE003D07A69FB6813437B61214A7B69536015
S31508029EF01F4BD3F884307B61FB68DB437A691340D6
S31508029F007B613B685B6803F40033002B03D07A69F4
S31508029F10FB6813437B61164A7B69C2F88430144B8B
S31508029F20D3F880307B61FB68DB437A6913407B6137
S31508029F303B685B6803F48033002B03D07A69FB68BD
S31508029F4013437B610A4A7B69C2F880303B69013355
S31508029F503B613B681A683B6922FA03F3002B7FF4DC
S31508029F60C1AE00BF00BF1C37BD465DF8047B704713
S31508029F70002002447F7F2F0080B487B000AF78604C
S31508029F80396000237B61A0E001227B6902FA03F3B0
S31508029F903A6813403B613B69002B00F09380524AB2
S31508029FA07B699B08183352F82330FB607B6903F000
S31508029FB00303DB000F2202FA03F3FA681340FB607D
S31508029FC07B689A0A494B13407A6902F00302D20067
S31508029FD09340FA689A4236D1434BD3F880203B69BC
S31508029FE0DB4341491340C1F880303F4BD3F8842004
S31508029FF03B69DB433C491340C1F884303A4B1A6843
S3150802A0003B69DB43384913400B60374B5A683B6957
S3150802A010DB43354913404B607B6903F00303DB00DE
S3150802A0200F2202FA03F3FB602F4A7B699B08183357
S3150802A03052F82310FB68DA432B487B699B080A40CF
S3150802A040183340F823207B681A687B695B00032172
S3150802A05001FA03F31A437B681A607B69DA087B689C
S3150802A060083253F822107B6903F007039B000F227C
S3150802A07002FA03F3DB437A69D20819407B6808328D
S3150802A08043F822107B689A687B695B00032101FA10
S3150802A09003F3DB431A407B689A607B685A6801219E
S3150802A0A07B6901FA03F3DB431A407B685A607B68D3
S3150802A0B0DA687B695B00032101FA03F3DB431A4082
S3150802A0C07B68DA607B6901337B613A687B6922FACD
S3150802A0D003F3002B7FF458AF00BF00BF1C37BD4601
S3150802A0E05DF8047B704700BF002002447F7F2F0083
S3150802A0F080B485B000AF78600B467B807B681A69AE
S3150802A1007B881340002B02D00123FB7301E0002356
S3150802A110FB73FB7B18461437BD465DF8047B704714
S3150802A12080B483B000AF78600B467B8013467B70A1
S3150802A1307B78002B03D07A887B689A6102E07A885A
S3150802A1407B689A6200BF0C37BD465DF8047B704790
S3150802A15080B485B000AF78600B467B807B685B690C
S3150802A160FB607A88FB6813401A04FB68D9437B882C
S3150802A1700B401A437B689A6100BF1437BD465DF8E7
S3150802A180047B704780B584B000AF78607B68002B8B
S3150802A19001D1012370E0786800F072F87B681B68C9
S3150802A1A04CF6CC421A607B681B6845F255521A6017
S3150802A1B07B681B687A6852685A607B681B687A688B
S3150802A1C092689A60FEF7D8F9F8600FE0FEF7D4F9BC
S3150802A1D00246FB68D31A212B08D97B681B68DB6801
S3150802A1E003F00203002B01D0032345E07B681B68BA
S3150802A1F0DB6803F00203002BE8D17B681B69002B9E
S3150802A20005D17B681B684FF480425A6106E07B6879
S3150802A2101A697B681B6842F440425A61FEF7ACF938
S3150802A220F8600FE0FEF7A8F90246FB68D31A212B5D
S3150802A23008D97B681B68DB6803F00F03002B01D083
S3150802A240032319E07B681B68DB6803F00F03002B06
S3150802A250E8D17B681B681A697B68DB689A4205D075
S3150802A2607B681B687A68D2681A6104E07B681B6897
S3150802A2704AF6AA221A60002318461037BD4680BD40
S3150802A28080B483B000AF786000BF0C37BD465DF876
S3150802A290047B704780B483B000AF78607B681B6824
S3150802A2A04AF6AA221A60002318460C37BD465DF8FC
S3150802A2B0047B704780B588B000AF78607B68002B56
S3150802A2C002D1012300F028BC944BDB6903F0180382
S3150802A2D0FB61924B9B6A03F00303BB617B681B68B5
S3150802A2E003F01003002B5BD0FB69082B05D0FB6932
S3150802A2F0182B14D1BB69022B11D17B68DB69002BA1
S3150802A30002D1012300F008BC844B9B6923F47C121A
S3150802A3107B681B6A1B04814913438B6140E07B6897
S3150802A320DB69002B23D07D4B1B687C4A43F4807380
S3150802A3301360FEF721F9786108E0FEF71DF9024677
S3150802A3407B69D31A022B01D90323E5E3734B1B68F6
S3150802A35003F40073002BF0D0704B9B6923F47C1234
S3150802A3607B681B6A1B046D4913438B6118E06B4BB0
S3150802A3701B686A4A23F480731360FEF7FDF8786156
S3150802A38008E0FEF7F9F802467B69D31A022B01D9CF
S3150802A3900323C1E3614B1B6803F40073002BF0D15E
S3150802A3A07B681B6803F00103002B00F0A080FB69A1
S3150802A3B0102B05D0FB69182B09D1BB69032B06D1D3
S3150802A3C07B685B68002B40F092800123A4E37B68DC
S3150802A3D05B68B3F5803F06D1504B1B684F4A43F47E
S3150802A3E08033136058E07B685B68002B12D14B4BB5
S3150802A3F01B684A4A23F480331360484B1B68474A52
S3150802A40023F480131360454B1B68444A23F48023C4
S3150802A410136041E07B685B68B3F5A02F12D13F4B0E
S3150802A4201B683E4A43F4802313603C4B1B683B4A35
S3150802A43023F480131360394B1B68384A43F480337C
S3150802A440136029E07B685B68B3F5A81F12D1334B0A
S3150802A4501B68324A43F480231360304B1B682F4A29
S3150802A46043F4801313602D4B1B682C4A43F4803344
S3150802A470136011E0294B1B68284A23F480331360C2
S3150802A480264B1B68254A23F480231360234B1B683B
S3150802A490224A23F4801313607B685B68002B13D06F
S3150802A4A0FEF76AF8786108E0FEF766F802467B6905
S3150802A4B0D31A642B01D903232EE3184B1B6803F422
S3150802A4C00033002BF0D012E0FEF756F8786108E068
S3150802A4D0FEF752F802467B69D31A642B01D9032385
S3150802A4E01AE30E4B1B6803F40033002BF0D17B688A
S3150802A4F01B6803F00203002B00F09A80FB69002B0D
S3150802A50005D0FB69182B49D1BB69012B46D17B685B
S3150802A510DB68002B04D10123FEE200BF000C0244D3
S3150802A520FB69002B1CD19A4B1B6803F018027B6847
S3150802A5301B699A4214D0964B1B6823F018027B6853
S3150802A5401B69934913430B6000F0D0FD914B1B68BE
S3150802A5501846FCF71FFA0346002B01D00123DBE25B
S3150802A560FEF70AF8786108E0FEF706F802467B6904
S3150802A570D31A022B01D90323CEE2854B1B6803F0BB
S3150802A5800203002BF0D0824B1B6923F4FE027B6880
S3150802A5905B691B047E4913430B6149E07B68DB68F0
S3150802A5A0002B2CD07A4B1B6823F018027B681B6998
S3150802A5B0774913430B60764B1B68754A43F00103D0
S3150802A5C01360FDF7D9FF786108E0FDF7D5FF02466B
S3150802A5D07B69D31A022B01D903239DE26C4B1B68B4
S3150802A5E003F00203002BF0D0694B1B6923F4FE0229
S3150802A5F07B685B691B04664913430B6118E0644B6D
S3150802A6001B68634A23F001031360FDF7B5FF7861FF
S3150802A61008E0FDF7B1FF02467B69D31A022B01D97E
S3150802A620032379E25A4B1B6803F00203002BF0D18D
S3150802A6307B681B6803F00803002B3CD07B689B6988
S3150802A640002B1CD0524BD3F8F030514A43F08063AA
S3150802A650C2F8F030FDF790FF786108E0FDF78CFF4D
S3150802A66002467B69D31A022B01D9032354E2484BCB
S3150802A670D3F8F03003F00063002BEFD01BE0444B15
S3150802A680D3F8F030424A23F08063C2F8F030FDF77F
S3150802A69073FF786108E0FDF76FFF02467B69D31AFC
S3150802A6A0022B01D9032337E2394BD3F8F03003F0F2
S3150802A6B00063002BEFD17B681B6803F00403002BB1
S3150802A6C000F0D280344B5B6A03F00103002B18D1E9
S3150802A6D0314B5B6A304A43F001035362FDF74CFF84
S3150802A6E0786108E0FDF748FF02467B69D31A022B18
S3150802A6F001D9032310E2284B5B6A03F00103002BFE
S3150802A700F0D07B689B68012B08D1214BD3F8F03037
S3150802A7101F4A43F00103C2F8F03074E07B689B6875
S3150802A720002B18D11A4BD3F8F030194A23F001033B
S3150802A730C2F8F030164BD3F8F030154A23F08003EE
S3150802A740C2F8F030124BD3F8F030114A23F0040362
S3150802A750C2F8F03057E07B689B68052B1ED10C4B7C
S3150802A760D3F8F0300A4A43F00403C2F8F030084B33
S3150802A770D3F8F030064A23F08003C2F8F030044BCF
S3150802A780D3F8F030024A43F00103C2F8F0303AE057
S3150802A790000C0244CC110020000802447B689B6826
S3150802A7A0852B18D1A24BD3F8F030A14A43F0040303
S3150802A7B0C2F8F0309E4BD3F8F0309D4A43F080033E
S3150802A7C0C2F8F0309A4BD3F8F030994A43F00103B5
S3150802A7D0C2F8F03017E0964BD3F8F030944A23F0DB
S3150802A7E00103C2F8F030924BD3F8F030904A23F0C6
S3150802A7F00403C2F8F0308E4BD3F8F0308C4A23F0BB
S3150802A8008003C2F8F0307B689B68002B16D0FDF7F0
S3150802A810B3FE78610AE0FDF7AFFE02467B69D31AFA
S3150802A82041F28832934201D9032375E1804BD3F86A
S3150802A830F03003F00203002BEDD015E0FDF79CFE85
S3150802A84078610AE0FDF798FE02467B69D31A41F25F
S3150802A8508832934201D903235EE1754BD3F8F0306F
S3150802A86003F00203002BEDD17B681B6803F020037B
S3150802A870002B36D07B685B6A002B19D06C4B1B68A1
S3150802A8806B4A43F480531360FDF776FE786108E05D
S3150802A890FDF772FE02467B69D31A022B01D90323FE
S3150802A8A03AE1634B1B6803F40053002BF0D018E01F
S3150802A8B05F4B1B685E4A23F480531360FDF75CFE08
S3150802A8C0786108E0FDF758FE02467B69D31A022B27
S3150802A8D001D9032320E1564B1B6803F40053002BCE
S3150802A8E0F0D17B689B6A002B00F01581FB69182B57
S3150802A8F000F0AF807B689B6A022B40F086804C4B47
S3150802A9001B684B4A23F080731360FDF735FE7861A6
S3150802A91008E0FDF731FE02467B69D31A022B01D9FC
S3150802A9200323F9E0424B1B6803F00073002BF0D1B6
S3150802A9303F4B9B6A23F47C5323F003037A68D16A5C
S3150802A9407A68126B12020A43394913438B627B688F
S3150802A9505B6B013BC3F308027B689B6B013B5B02A3
S3150802A9609BB21A437B68DB6B013B1B0403F4FE03B1
S3150802A9701A437B681B6C013B1B0603F0FE432C49FA
S3150802A98013434B632A4B9B6A294A23F010039362AB
S3150802A9907B68DB6C264ADB009363254B9B6A244A59
S3150802A9A043F010039362224B9B6A23F00C027B68E6
S3150802A9B05B6C1F4913438B621D4B9B6A23F0200273
S3150802A9C07B689B6C1A4913438B62194B9B6A184A1C
S3150802A9D043F480339362164B1B68154A43F080731F
S3150802A9E01360FDF7C9FD786108E0FDF7C5FD02466B
S3150802A9F07B69D31A022B01D903238DE00C4B1B6802
S3150802AA0003F00073002BF0D085E0094B1B68084A57
S3150802AA1023F080731360FDF7AFFD78610AE0FDF756
S3150802AA20ABFD02467B69D31A022B03D9032373E0D3
S3150802AA30000C02443A4B1B6803F00073002BEED15C
S3150802AA40374B9B6A364A23F4E02323F003039362C7
S3150802AA5061E0334B9B6A3B61314B5B6BFB607B6806
S3150802AA609B6A012B31D03B6903F003027B68DB6AE0
S3150802AA709A422AD13B691B0A03F03F027B681B6B89
S3150802AA809A4222D1FB68C3F308027B685B6B013BDF
S3150802AA909A421AD1FB685B0A03F07F027B689B6BBA
S3150802AAA0013B9A4211D1FB681B0C03F07F027B68BB
S3150802AAB0DB6B013B9A4208D1FB681B0E03F07F024F
S3150802AAC07B681B6C013B9A4201D0012324E0144B9C
S3150802AAD09B6BDB08C3F30C027B68DB6C9A421AD0C9
S3150802AAE00F4B9B6A0E4A23F010039362FDF744FD4F
S3150802AAF0786100BFFDF740FD02467B699342F9D0B3
S3150802AB007B68DB6C064ADB009363054B9B6A044A47
S3150802AB1043F010039362002318462037BD4680BDD2
S3150802AB20000C024480B584B000AF786039607B6857
S3150802AB30002B01D101239EE1834B1B6803F00F030F
S3150802AB403A689A4210D9804B1B6823F00F027E4955
S3150802AB503B6813430B607C4B1B6803F00F033A6890
S3150802AB609A4201D0012386E17B681B6803F0100331
S3150802AB70002B12D07B685A69744B1B6A1B0A03F0B6
S3150802AB8070039A4209D9714B1B6A23F4E0427B6827
S3150802AB905B691B026D4913430B627B681B6803F0F2
S3150802ABA00803002B12D07B681A69684B1B6A1B09BB
S3150802ABB003F070039A4209D9644B1B6A23F4E062D4
S3150802ABC07B681B691B01614913430B627B681B681F
S3150802ABD003F00403002B10D07B68DA685B4B1B6A10
S3150802ABE003F070039A4208D9584B1B6A23F0700285
S3150802ABF07B68DB68554913430B627B681B6803F065
S3150802AC000203002B10D07B689A68504B1B6A03F02C
S3150802AC100F039A4208D94D4B1B6A23F00F027B6831
S3150802AC209B684A4913430B627B681B6803F001035E
S3150802AC30002B00F093807B685B68032B07D1434B9C
S3150802AC401B6803F00073002B21D1012313E17B68F3
S3150802AC505B68022B07D13D4B1B6803F40033002BBC
S3150802AC6015D1012307E17B685B68012B07D1374BB6
S3150802AC701B6803F40073002B09D10123FBE0334B55
S3150802AC801B6803F00203002B01D10123F3E02F4BCB
S3150802AC90DB6923F003027B685B682C491343CB61AB
S3150802ACA0FDF76AFCF8607B685B68032B12D10AE041
S3150802ACB0FDF762FC0246FB68D31A41F288329342D8
S3150802ACC001D90323D7E0214BDB6903F01803182BBC
S3150802ACD0EED143E07B685B68022B12D10AE0FDF7EE
S3150802ACE04BFC0246FB68D31A41F28832934201D9D9
S3150802ACF00323C0E0154BDB6903F01803102BEED1D2
S3150802AD002CE07B685B68012B22D10AE0FDF734FC54
S3150802AD100246FB68D31A41F28832934201D90323C9
S3150802AD20A9E00A4BDB6903F01803082BEED115E0FC
S3150802AD30FDF722FC0246FB68D31A41F28832934297
S3150802AD4006D9032397E000BF00200240000C024404
S3150802AD504B4BDB6903F01803002BE9D17B681B68B0
S3150802AD6003F00203002B10D07B689A68444B1B6AD7
S3150802AD7003F00F039A4208D2414B1B6A23F00F02D3
S3150802AD807B689B683E4913430B623E4B1B6803F084
S3150802AD900F033A689A4210D23A4B1B6823F00F0205
S3150802ADA038493B6813430B60364B1B6803F00F03A5
S3150802ADB03A689A4201D001235DE07B681B6803F07A
S3150802ADC00403002B10D07B68DA682D4B1B6A03F04C
S3150802ADD070039A4208D22A4B1B6A23F070027B68D8
S3150802ADE0DB68274913430B627B681B6803F0080379
S3150802ADF0002B12D07B681A69214B1B6A1B0903F0C8
S3150802AE0070039A4209D21E4B1B6A23F4E0627B68DE
S3150802AE101B691B011A4913430B627B681B6803F003
S3150802AE201003002B12D07B685A69154B1B6A1B0A42
S3150802AE3003F070039A4209D2114B1B6A23F4E042CB
S3150802AE407B685B691B020E4913430B6200F022F80A
S3150802AE5002460B4B1B6A03F00F030B49CB5C22FA23
S3150802AE6003F30A4A13600A4B1B681846FBF792FD5E
S3150802AE700346FB72FB7A18461037BD4680BD00BFF3
S3150802AE80000C02440020024068180408C811002079
S3150802AE90CC11002080B489B000AF8C4BDB6903F07B
S3150802AEA01803082B02D18A4BFB6107E1874BDB6942
S3150802AEB003F01803002B12D1844B1B6803F02003FE
S3150802AEC0002B09D0814B1B68DB0803F00303814A78
S3150802AED022FA03F3FB61F1E07E4BFB61EEE07B4B6A
S3150802AEE0DB6903F01803102B02D17B4BFB61E5E00B
S3150802AEF0764BDB6903F01803182B40F0DD80734BA1
S3150802AF009B6A03F003037B61704B9B6A1B0A03F07F
S3150802AF103F033B616D4B9B6A1B0903F00103FB6010
S3150802AF206A4B9B6BDB08C3F30C03FA6802FB03F359
S3150802AF3007EE903AF8EE677AC7ED027A3B69002B7C
S3150802AF4000F0B7807B69012B03D07B69032B56D0AF
S3150802AF5077E05E4B1B6803F02003002B2DD05B4B7A
S3150802AF601B68DB0803F003035A4A22FA03F37B60E1
S3150802AF707B6807EE903AF8EE676A3B6907EE903A05
S3150802AF80F8EE677A86EEA77A504B5B6BC3F3080333
S3150802AF9007EE903AF8EE676A97ED026ADFED4F5AC6
S3150802AFA0C6EE257A76EEA77AF7EE006A77EEA67AE5
S3150802AFB067EE277AC7ED067A65E03B6907EE903AAF
S3150802AFC0F8EE677ADFED466A86EEA77A3F4B5B6B49
S3150802AFD0C3F3080307EE903AF8EE676A97ED026A3A
S3150802AFE0DFED3E5AC6EE257A76EEA77AF7EE006AC6
S3150802AFF077EEA67A67EE277AC7ED067A43E03B69CB
S3150802B00007EE903AF8EE677ADFED366A86EEA77AA9
S3150802B0102E4B5B6BC3F3080307EE903AF8EE676AAA
S3150802B02097ED026ADFED2D5AC6EE257A76EEA77AF5
S3150802B030F7EE006A77EEA67A67EE277AC7ED067A02
S3150802B04021E03B6907EE903AF8EE677ADFED266A69
S3150802B05086EEA77A1D4B5B6BC3F3080307EE903A9D
S3150802B060F8EE676A97ED026ADFED1C5AC6EE257A94
S3150802B07076EEA77AF7EE006A77EEA67A67EE277A71
S3150802B080C7ED067A00BF114B5B6B5B0A03F07F03C1
S3150802B09001333B603B6807EE903AB8EE677AD7ED24
S3150802B0A0066AC6EE877AFCEEE77A17EE903AFB61F5
S3150802B0B004E00023FB6101E0064BFB61FB691846CD
S3150802B0C02437BD465DF8047B704700BF000C024476
S3150802B0D000093D000090D003001BB700000000469F
S3150802B0E00024744C001B374B0024744A80B500AF09
S3150802B0F0FFF7D0FE0246084B1B6A03F00F03074907
S3150802B100CB5C03F01F0322FA03F3054A1360044BD0
S3150802B1101B68184680BD00BF000C02446818040864
S3150802B120C811002080B500AFFFF7E0FF0246064BC4
S3150802B1301B6A1B0903F007030449CB5C03F01F03D0
S3150802B14022FA03F3184680BD000C02447818040854
S3150802B15080B500AFFFF7CAFF0246064B1B6A1B0AF9
S3150802B16003F007030449CB5C03F01F0322FA03F337
S3150802B170184680BD000C02447818040880B500AF52
S3150802B180FFF7B4FF0246064B1B6A1B0B03F00703C5
S3150802B1900449CB5C03F01F0322FA03F3184680BD69
S3150802B1A0000C02447818040880B485B000AF7860B1
S3150802B1B039607B681F221A60154BDB6903F00302AC
S3150802B1C07B685A60124B1B6AFB60FB6803F00F022E
S3150802B1D07B689A60FB6803F070027B68DA60FB683A
S3150802B1E01B0903F070027B681A61FB681B0A03F0ED
S3150802B1F070027B685A61074B1B6803F00F023B68B3
S3150802B2001A6000BF1437BD465DF8047B704700BF5D
S3150802B210000C0244002002402DE9B04FD8B000AF1E
S3150802B220C7F84C01002387F85B31002387F85A31A7
S3150802B230D7F84C31D3E9002302F08074002554EA8A
S3150802B24005030BD0CD4BD3F8E83023F04041D7F8AD
S3150802B2504C319B6DC94A0B43C2F8E830D7F84C31DA
S3150802B260D3E9002302F001084FF0000958EA09035E
S3150802B27042D0D7F84C31DB6D052B23D801A252F800
S3150802B28023F000BFCDB202089DB20208B1B202088D
S3150802B290CDB20208CDB20208CDB20208D7F84C31B7
S3150802B2A00833184604F0DAFE034687F85B310EE0E7
S3150802B2B0D7F84C313033184604F068FF034687F84E
S3150802B2C05B3104E0012387F85B3100E000BF97F8A1
S3150802B2D05B31002B0CD1A94BD3F8D83023F00701E8
S3150802B2E0D7F84C31DB6DA54A0B43C2F8D83003E0D8
S3150802B2F097F85B3187F85A31D7F84C31D3E90023EE
S3150802B30002F0020A4FF0000B5AEA0B0300F088809B
S3150802B310D7F84C311B6E282B68D801A252F823F0B5
S3150802B320F5B30208EDB30208EDB30208EDB302085D
S3150802B330EDB30208EDB30208EDB30208EDB3020855
S3150802B340C5B30208EDB30208EDB30208EDB302086D
S3150802B350EDB30208EDB30208EDB30208EDB3020835
S3150802B360D9B30208EDB30208EDB30208EDB3020839
S3150802B370EDB30208EDB30208EDB30208EDB3020815
S3150802B380F5B30208EDB30208EDB30208EDB30208FD
S3150802B390EDB30208EDB30208EDB30208EDB30208F5
S3150802B3A0F5B30208EDB30208EDB30208EDB30208DD
S3150802B3B0EDB30208EDB30208EDB30208EDB30208D5
S3150802B3C0F5B30208D7F84C310833184604F046FE9E
S3150802B3D0034687F85B310EE0D7F84C31303318460E
S3150802B3E004F0D4FE034687F85B3104E0012387F8AC
S3150802B3F05B3100E000BF97F85B31002B0CD15F4B45
S3150802B400D3F8D83023F03801D7F84C311B6E5B4A93
S3150802B4100B43C2F8D83003E097F85B3187F85A3104
S3150802B420D7F84C31D3E9002302F00403C7F84031B8
S3150802B4300023C7F84431D7E950120B4613434ED0BE
S3150802B440D7F84C315B6EB3F5A07F2CD0B3F5A07F4D
S3150802B45025D8B3F5807F28D0B3F5807F1FD8C02BB7
S3150802B46025D0C02B1BD8802B0FD0802B17D8002BAA
S3150802B4701FD0402B13D1D7F84C310833184604F0A5
S3150802B480EDFD034687F85B3114E0D7F84C313033CB
S3150802B490184604F07BFE034687F85B310AE001236F
S3150802B4A087F85B3106E000BF04E000BF02E000BF98
S3150802B4B000E000BF97F85B31002B0CD12F4BD3F875
S3150802B4C0D83023F4E071D7F84C315B6E2B4A0B4324
S3150802B4D0C2F8D83003E097F85B3187F85A31D7F8C3
S3150802B4E04C31D3E9002302F00803C7F838310023A8
S3150802B4F0C7F83C31D7E94E120B46134356D0D7F854
S3150802B5004C319B6EB3F5206F31D0B3F5206F2AD834
S3150802B510B3F5006F2DD0B3F5006F24D8B3F5C06F1D
S3150802B52029D0B3F5C06F1ED8B3F5806F11D0B3F525
S3150802B530806F18D8002B23D0B3F5007F13D1D7F824
S3150802B5404C310833184604F089FD034687F85B3107
S3150802B55017E0D7F84C313033184604F017FE034685
S3150802B56087F85B310DE0012387F85B3109E000BFFC
S3150802B57007E000BF05E000BF03E000BF000C02447D
S3150802B58000BF97F85B31002B0CD1BB4BD3F8D830F0
S3150802B59023F46061D7F84C319B6EB74A0B43C2F865
S3150802B5A0D83003E097F85B3187F85A31D7F84C312F
S3150802B5B0D3E9002302F01003C7F830310023C7F895
S3150802B5C03431D7E94C120B46134353D0D7F84C31D2
S3150802B5D0DB6EB3F5A04F31D0B3F5A04F2AD8B3F539
S3150802B5E0804F2DD0B3F5804F24D8B3F5405F29D0CC
S3150802B5F0B3F5405F1ED8B3F5005F11D0B3F5005F0F
S3150802B60018D8002B20D0B3F5805F13D1D7F84C3168
S3150802B6100833184604F022FD034687F85B3114E026
S3150802B620D7F84C313033184604F0B0FD034687F894
S3150802B6305B310AE0012387F85B3106E000BF04E0CC
S3150802B64000BF02E000BF00E000BF97F85B31002BA5
S3150802B6500CD1894BD3F8D83023F4E041D7F84C31D2
S3150802B660DB6E854A0B43C2F8D83003E097F85B31A4
S3150802B67087F85A31D7F84C31D3E9002302F0200370
S3150802B680C7F828310023C7F82C31D7E94A120B46E6
S3150802B690134353D0D7F84C311B6FB3F5203F31D043
S3150802B6A0B3F5203F2AD8B3F5003F2DD0B3F5003FB6
S3150802B6B024D8B3F5C03F29D0B3F5C03F1ED8B3F599
S3150802B6C0803F11D0B3F5803F18D8002B20D0B3F5B0
S3150802B6D0004F13D1D7F84C310833184604F0BEFC94
S3150802B6E0034687F85B3114E0D7F84C3130331846F5
S3150802B6F004F04CFD034687F85B310AE0012387F81C
S3150802B7005B3106E000BF04E000BF02E000BF00E0D4
S3150802B71000BF97F85B31002B0CD1574BD3F8D830C2
S3150802B72023F46031D7F84C311B6F534A0B43C2F8E6
S3150802B730D83003E097F85B3187F85A31D7F84C319D
S3150802B740D3E9002302F04003C7F820310023C7F8E3
S3150802B7502431D7E948120B46134353D0D7F84C3154
S3150802B7605B6FB3F5A01F31D0B3F5A01F2AD8B3F586
S3150802B770801F2DD0B3F5801F24D8B3F5402F29D0CA
S3150802B780B3F5402F1ED8B3F5002F11D0B3F5002F0D
S3150802B79018D8002B20D0B3F5802F13D1D7F84C3107
S3150802B7A00833184604F05AFC034687F85B3114E05E
S3150802B7B0D7F84C313033184604F0E8FC034687F8CC
S3150802B7C05B310AE0012387F85B3106E000BF04E03B
S3150802B7D000BF02E000BF00E000BF97F85B31002B14
S3150802B7E00CD1254BD3F8D83023F4E011D7F84C31D5
S3150802B7F05B6F214A0B43C2F8D83003E097F85B31F6
S3150802B80087F85A31D7F84C31D3E9002302F080037E
S3150802B810C7F818310023C7F81C31D7E946120B4678
S3150802B820134355D0D7F84C319B6FB3F5200F33D05D
S3150802B830B3F5200F2CD8B3F5000F2FD0B3F5000FB0
S3150802B84026D8B3F5C00F2BD0B3F5C00F20D8B3F561
S3150802B850800F13D0B3F5800F1AD8002B22D0B3F578
S3150802B860001F15D1D7F84C310833184604F0F6FBF9
S3150802B870034687F85B3116E0000C0244D7F84C31D0
S3150802B8803033184604F082FC034687F85B310AE037
S3150802B890012387F85B3106E000BF04E000BF02E03F
S3150802B8A000BF00E000BF97F85B31002B0CD1BB4B01
S3150802B8B0D3F8D83023F46001D7F84C319B6FB74AD6
S3150802B8C00B43C2F8D83003E097F85B3187F85A3150
S3150802B8D0D7F84C31D3E9002302F48073C7F8103144
S3150802B8E00023C7F81431D7E944120B46134353D041
S3150802B8F0D7F84C31DB6FB3F1A06F31D0B3F1A06F3B
S3150802B9002AD8B3F1806F2DD0B3F1806F24D8B3F162
S3150802B910407F29D0B3F1407F1ED8B3F1007F11D002
S3150802B920B3F1007F18D8002B20D0B3F1807F13D152
S3150802B930D7F84C310833184604F090FB034687F8CB
S3150802B9405B3114E0D7F84C313033184604F01EFC4C
S3150802B950034687F85B310AE0012387F85B3106E084
S3150802B96000BF04E000BF02E000BF00E000BF97F896
S3150802B9705B31002B0CD1894BD3F8D83023F0E06128
S3150802B980D7F84C31DB6F854A0B43C2F8D83003E04F
S3150802B99097F85B3187F85A31D7F84C31D3E9002347
S3150802B9A002F40073C7F808310023C7F80C31D7E947
S3150802B9B042120B46134355D0D7F84C31D3F8803090
S3150802B9C0B3F1205F31D0B3F1205F2AD8B3F1005F1B
S3150802B9D02DD0B3F1005F24D8B3F1C05F29D0B3F1FB
S3150802B9E0C05F1ED8B3F1805F11D0B3F1805F18D85B
S3150802B9F0002B20D0B3F1006F13D1D7F84C3108339E
S3150802BA00184604F02BFB034687F85B3114E0D7F897
S3150802BA104C313033184604F0B9FB034687F85B31DC
S3150802BA200AE0012387F85B3106E000BF04E000BFA5
S3150802BA3002E000BF00E000BF97F85B31002B0DD192
S3150802BA40564BD3F8D83023F06051D7F84C31D3F897
S3150802BA508030524A0B43C2F8D83003E097F85B317C
S3150802BA6087F85A31D7F84C31D3E9002302F48063B8
S3150802BA70C7F800310023C7F80431D7E940120B464C
S3150802BA80134344D0D7F84C31D3F88430052B23D846
S3150802BA9001A252F823F000BFE1BA0208B1BA0208BD
S3150802BAA0C5BA0208E1BA0208E1BA0208E1BA02080E
S3150802BAB0D7F84C310833184604F0D0FA034687F80B
S3150802BAC05B310EE0D7F84C313033184604F05EFB92
S3150802BAD0034687F85B3104E0012387F85B3100E00F
S3150802BAE000BF97F85B31002B0DD12C4BD3F8DC3015
S3150802BAF023F00701D7F84C31D3F88430274A0B4391
S3150802BB00C2F8DC3003E097F85B3187F85A31D7F888
S3150802BB104C31D3E9002302F40063C7F8F830002356
S3150802BB20C7F8FC30D7E93E120B4613434FD0D7F875
S3150802BB304C31D3F88830502B29D0502B23D8402BA0
S3150802BB4027D0402B1FD8302B25D0302B1BD8202BA3
S3150802BB500FD0202B17D8002B22D0102B13D1D7F8B1
S3150802BB604C310833184604F079FA034687F85B31F4
S3150802BB7017E0D7F84C313033184604F007FB034672
S3150802BB8087F85B310DE0012387F85B3109E000BFD6
S3150802BB9007E000BF05E000BF03E000BF000C024457
S3150802BBA000BF97F85B31002B0DD1AF4BD3F8DC30D1
S3150802BBB023F07001D7F84C31D3F88830AA4A0B43E0
S3150802BBC0C2F8DC3003E097F85B3187F85A31D7F8C8
S3150802BBD04C31D3E9002302F48053C7F8F03000232E
S3150802BBE0C7F8F430D7E93C120B46134355D0D7F8B9
S3150802BBF04C31D3F88C30B3F1A06F31D0B3F1A06FCA
S3150802BC002AD8B3F1806F2DD0B3F1806F24D8B3F15F
S3150802BC10407F29D0B3F1407F1ED8B3F1007F11D0FF
S3150802BC20B3F1007F18D8002B20D0B3F1807F13D14F
S3150802BC30D7F84C310833184604F010FA034687F849
S3150802BC405B3114E0D7F84C313033184604F09EFACB
S3150802BC50034687F85B310AE0012387F85B3106E081
S3150802BC6000BF04E000BF02E000BF00E000BF97F893
S3150802BC705B31002B0DD17C4BD3F8E03023F0E06129
S3150802BC80D7F84C31D3F88C30774A0B43C2F8E030F8
S3150802BC9003E097F85B3187F85A31D7F84C31D3E984
S3150802BCA0002302F40053C7F8E8300023C7F8EC3043
S3150802BCB0D7E93A120B4613433DD0D7F84C31D3F89D
S3150802BCC09030B3F5403F1BD0B3F5403F14D8B3F5D7
S3150802BCD0003F17D0B3F5003F0ED8002B14D0B3F5AA
S3150802BCE0803F09D1D7F84C313033184604F04EFA62
S3150802BCF0034687F85B3108E0012387F85B3104E0E5
S3150802BD0000BF02E000BF00E000BF97F85B31002BDE
S3150802BD100DD1554BD3F8E43023F44031D7F84C31E2
S3150802BD20D3F89030504A0B43C2F8E43003E097F850
S3150802BD305B3187F85A31D7F84C31D3E9002302F43C
S3150802BD408043C7F8E0300023C7F8E430D7E9381251
S3150802BD500B4613433DD0D7F84C31D3F89430B3F59C
S3150802BD60402F1BD0B3F5402F14D8B3F5002F17D0A8
S3150802BD70B3F5002F0ED8002B14D0B3F5802F09D1B6
S3150802BD80D7F84C313033184604F000FA034687F8E0
S3150802BD905B3108E0012387F85B3104E000BF02E06B
S3150802BDA000BF00E000BF97F85B31002B0DD12E4B88
S3150802BDB0D3F8E43023F44021D7F84C31D3F8943041
S3150802BDC0294A0B43C2F8E43003E097F85B3187F857
S3150802BDD05A31D7F84C31D3E9002302F40043C7F8A5
S3150802BDE0D8300023C7F8DC30D7E936120B4613439E
S3150802BDF040D0D7F84C31D3F89830B3F5401F1BD052
S3150802BE00B3F5401F14D8B3F5001F17D0B3F5001FBA
S3150802BE100ED8002B14D0B3F5801F09D1D7F84C31B0
S3150802BE203033184604F0B2F9034687F85B3108E066
S3150802BE30012387F85B3104E000BF02E000BF00E09F
S3150802BE4000BF97F85B31002B10D1074BD3F8E430CB
S3150802BE5023F44011D7F84C31D3F89830024A0B43F1
S3150802BE60C2F8E43006E000BF000C024497F85B31E2
S3150802BE7087F85A31D7F84C31D3E900230021C7F89D
S3150802BE80D01003F48063C7F8D430D7E934120B46CE
S3150802BE9013433DD0D7F84C31D3F89C30B3F5400F55
S3150802BEA01BD0B3F5400F14D8B3F5000F17D0B3F56E
S3150802BEB0000F0ED8002B14D0B3F5800F09D1D7F88E
S3150802BEC04C313033184604F061F9034687F85B3182
S3150802BED008E0012387F85B3104E000BF02E000BFF7
S3150802BEE000E000BF97F85B31002B0DD1BE4BD3F8AB
S3150802BEF0E43023F44001D7F84C31D3F89C30BA4ADF
S3150802BF000B43C2F8E43003E097F85B3187F85A31FD
S3150802BF10D7F84C31D3E9002302F48033C7F8C83086
S3150802BF200023C7F8CC30D7E932120B46134335D073
S3150802BF30D7F84C31D3F8A030B3F1007F15D0B3F15E
S3150802BF40007F0ED8002B12D0B3F1807F09D1D7F823
S3150802BF504C313033184604F019F9034687F85B3139
S3150802BF6006E0012387F85B3102E000BF00E000BF6C
S3150802BF7097F85B31002B0DD19B4BD3F8E43023F0B5
S3150802BF804071D7F84C31D3F8A030974A0B43C2F820
S3150802BF90E43003E097F85B3187F85A31D7F84C3129
S3150802BFA0D3E900230021C7F8C01003F40063C7F8D9
S3150802BFB0C430D7E930120B4613430ED08A4BDB69DD
S3150802BFC0894A23F40043D361874BD969D7F84C31A0
S3150802BFD0D3F80431844A0B43D361D7F84C31D3E9F9
S3150802BFE0002302F40033C7F8B8300023C7F8BC3080
S3150802BFF0D7E92E120B46134355D0D7F84C31D3F84E
S3150802C000A430B3F5A06F31D0B3F5A06F2AD8B3F533
S3150802C010806F2DD0B3F5806F24D8B3F5407F29D031
S3150802C020B3F5407F1ED8B3F5007F11D0B3F5007F74
S3150802C03018D8002B20D0B3F5807F13D1D7F84C310E
S3150802C0400833184604F00AF8034687F85B3114E009
S3150802C050D7F84C313033184604F098F8034687F877
S3150802C0605B310AE0012387F85B3106E000BF04E092
S3150802C07000BF02E000BF00E000BF97F85B31002B6B
S3150802C0800DD1594BD3F8DC3023F4E061D7F84C31A3
S3150802C090D3F8A430544A0B43C2F8DC3003E097F8CD
S3150802C0A05B3187F85A31D7F84C31D3E9002302F4C9
S3150802C0B08023C7F8B0300023C7F8B430D7E92C126A
S3150802C0C00B46134355D0D7F84C31D3F8A830B3F5FD
S3150802C0D0A04F31D0B3F5A04F2AD8B3F5804F2DD053
S3150802C0E0B3F5804F24D8B3F5405F29D0B3F5405F46
S3150802C0F01ED8B3F5005F11D0B3F5005F18D8002B30
S3150802C10020D0B3F5805F13D1D7F84C3108331846DF
S3150802C11003F0A4FF034687F85B3114E0D7F84C31E5
S3150802C1203033184604F032F8034687F85B310AE0E2
S3150802C130012387F85B3106E000BF04E000BF02E096
S3150802C14000BF00E000BF97F85B31002B0DD1264BEC
S3150802C150D3F8DC3023F4E041D7F84C31D3F8A830D1
S3150802C160214A0B43C2F8DC3003E097F85B3187F8C3
S3150802C1705A31D7F84C31D3E900230021C7F8A81061
S3150802C18003F02003C7F8AC30D7E92A120B4613434B
S3150802C19057D0D7F84C31D3F8AC30B3F5A02F33D0FB
S3150802C1A0B3F5A02F2CD8B3F5802F2FD0B3F5802F57
S3150802C1B026D8B3F5403F2BD0B3F5403F20D8B3F588
S3150802C1C0003F13D0B3F5003F1AD8002B22D0B3F59F
S3150802C1D0803F15D1D7F84C310833184603F03EFF95
S3150802C1E0034687F85B3116E0000C0244D7F84C3157
S3150802C1F03033184603F0CAFF034687F85B310AE074
S3150802C200012387F85B3106E000BF04E000BF02E0C5
S3150802C21000BF00E000BF97F85B31002B0DD1BB4B86
S3150802C220D3F8DC3023F4E021D7F84C31D3F8AC301C
S3150802C230B64A0B43C2F8DC3003E097F85B3187F85D
S3150802C2405A31D7F84C31D3E900230021C7F8A01098
S3150802C25003F04003C7F8A430D7E928120B46134364
S3150802C26055D0D7F84C31D3F8B030B3F5A00F31D04A
S3150802C270B3F5A00F2AD8B3F5800F2DD0B3F5800FEA
S3150802C28024D8B3F5401F29D0B3F5401F1ED8B3F5FD
S3150802C290001F11D0B3F5001F18D8002B20D0B3F514
S3150802C2A0801F13D1D7F84C310833184603F0D6FE4F
S3150802C2B0034687F85B3114E0D7F84C313033184619
S3150802C2C003F064FF034687F85B310AE0012387F827
S3150802C2D05B3106E000BF04E000BF02E000BF00E0F9
S3150802C2E000BF97F85B31002B0DD1884BD3F8DC30B1
S3150802C2F023F4E001D7F84C31D3F8B030834A0B4324
S3150802C300C2F8DC3003E097F85B3187F85A31D7F880
S3150802C3104C31D3E900230021C7F8981003F08003B3
S3150802C320C7F89C30D7E926120B46134355D0D7F8DF
S3150802C3304C31D3F8B430B3F1A06F31D0B3F1A06F5A
S3150802C3402AD8B3F1806F2DD0B3F1806F24D8B3F118
S3150802C350407F29D0B3F1407F1ED8B3F1007F11D0B8
S3150802C360B3F1007F18D8002B20D0B3F1807F13D108
S3150802C370D7F84C310833184603F070FE034687F89F
S3150802C3805B3114E0D7F84C313033184603F0FEFE21
S3150802C390034687F85B310AE0012387F85B3106E03A
S3150802C3A000BF04E000BF02E000BF00E000BF97F84C
S3150802C3B05B31002B0DD1554BD3F8DC3023F0E0610D
S3150802C3C0D7F84C31D3F8B430504A0B43C2F8DC30B4
S3150802C3D003E097F85B3187F85A31D7F84C31D3E93D
S3150802C3E000230021C7F8901003F48073C7F894302D
S3150802C3F0D7E924120B46134355D0D7F84C31D3F854
S3150802C400B830B3F1A04F31D0B3F1A04F2AD8B3F167
S3150802C410804F2DD0B3F1804F24D8B3F1405F29D095
S3150802C420B3F1405F1ED8B3F1005F11D0B3F1005FDC
S3150802C43018D8002B20D0B3F1805F13D1D7F84C312E
S3150802C4400833184603F00AFE034687F85B3114E000
S3150802C450D7F84C313033184603F098FE034687F86E
S3150802C4605B310AE0012387F85B3106E000BF04E08E
S3150802C47000BF02E000BF00E000BF97F85B31002B67
S3150802C4800DD1224BD3F8DC3023F0E041D7F84C31FA
S3150802C490D3F8B8301D4A0B43C2F8DC3003E097F8EC
S3150802C4A05B3187F85A31D7F84C31D3E9002302F4C5
S3150802C4B00023C7F888300023C7F88C30D7E9221240
S3150802C4C00B46134355D0D7F84C31D3F8C030B3F5E1
S3150802C4D0802F35D0B3F5802F2ED8B3F5403F31D013
S3150802C4E0B3F5403F28D8B3F5003F1BD0B3F5003F5C
S3150802C4F022D8002B03D0B3F5803F09D01CE0034BAA
S3150802C5009B6A024A43F4003393621CE0000C02441D
S3150802C510D7F84C310833184603F0A0FD034687F8CE
S3150802C5205B3110E0D7F84C313033184603F02EFE53
S3150802C530034687F85B3106E0012387F85B3102E0A0
S3150802C54000BF00E000BF97F85B31002B0DD1C34B4B
S3150802C550D3F8E83023F4E021D7F84C31D3F8C030C9
S3150802C560BE4A0B43C2F8E83003E097F85B3187F816
S3150802C5705A31D7F84C31D3E9002302F48013C7F8AD
S3150802C58080300023C7F88430D7E920120B461343BC
S3150802C59051D0D7F84C31D3F8C430B3F5001F33D095
S3150802C5A0B3F5001F2CD8B3F5C01F2DD0B3F5C01FA5
S3150802C5B026D8B3F5801F19D0B3F5801F20D8002BD3
S3150802C5C003D0B3F5002F07D01AE0A44B9B6AA34AFF
S3150802C5D043F40033936218E0D7F84C31083318460F
S3150802C5E003F03CFD034687F85B310EE0D7F84C3181
S3150802C5F03033184603F0CAFD034687F85B3104E078
S3150802C600012387F85B3100E000BF97F85B31002B06
S3150802C6100DD1924BD3F8E83023F46011D7F84C3198
S3150802C620D3F8C4308D4A0B43C2F8E83003E097F8D2
S3150802C6305B3187F85A31D7F84C31D3E9002302F433
S3150802C6400013BB670023FB67D7E91E120B46134389
S3150802C65032D0D7F84C31D3F8D430052B0FD8032B68
S3150802C66011D2012B11D9022B09D1D7F84C31083333
S3150802C670184603F0F3FC034687F85B3106E001230C
S3150802C68087F85B3102E000BF00E000BF97F85B3134
S3150802C690002B0DD1714BD3F8E83023F00701D7F8F8
S3150802C6A04C31D3F8D4306D4A0B43C2F8E83003E074
S3150802C6B097F85B3187F85A31D7F84C31D3E900231A
S3150802C6C00021396703F400737B67D7E91C120B460E
S3150802C6D0134324D0D7F84C31D3F8D830002B05D0E1
S3150802C6E0082B05D0012387F85B3102E000BF00E082
S3150802C6F000BF97F85B31002B0DD1584BD3F8E830C1
S3150802C70023F00801D7F84C31D3F8D830534A0B43F3
S3150802C710C2F8E83003E097F85B3187F85A31D7F860
S3150802C7204C31D3E9002302F00073BB660023FB6693
S3150802C730D7E91A120B46134300F0B980484B5B6AD5
S3150802C740474A43F001035362FBF716FFC7F8540141
S3150802C7500BE0FBF711FF0246D7F85431D31A022B26
S3150802C76003D9032387F85B3105E03D4B5B6A03F087
S3150802C7700103002BEDD097F85B31002B40F0938034
S3150802C780364BD3F8F03003F44073C7F85C31D7F868
S3150802C7905C31002B23D0D7F84C31D3F8F820D7F8E0
S3150802C7A05C3193421BD02D4BD3F8F03023F44073FF
S3150802C7B0C7F85C31294BD3F8F030284A43F4803362
S3150802C7C0C2F8F030254BD3F8F030244A23F48033EC
S3150802C7D0C2F8F030214AD7F85C31C2F8F030D7F8FF
S3150802C7E05C3103F00103002B19D0FBF7C5FEC7F82D
S3150802C7F054010DE0FBF7C0FE0246D7F85431D21AAF
S3150802C80041F288339A4203D9032387F85B3106E05B
S3150802C810124BD3F8F03003F00203002BEAD097F854
S3150802C8205B31002B3AD1D7F84C31D3F8F83003F400
S3150802C8304073B3F5407F15D1084BDB6923F47C516D
S3150802C840D7F84C31D3F8F8301B0923F07F4323F08D
S3150802C8503003024A0B43D3610AE000BF000C0244CC
S3150802C860000802449F4BDB699E4A23F47C53D3613A
S3150802C8709C4BD3F8F0309B4A23F44073C2F8F0304D
S3150802C880984BD3F8F010D7F84C31D3F8F830C3F3F5
S3150802C8900B03944A0B43C2F8F03008E097F85B3171
S3150802C8A087F85A3103E097F85B3187F85A31D7F897
S3150802C8B04C31D3E9002302F080633B6600237B6692
S3150802C8C0D7E918120B46134335D0D7F84C31D3F8AB
S3150802C8D0C830302B14D0302B0ED8202B12D0202B58
S3150802C8E00AD8002B10D0102B06D17E4B9B6A7D4AA4
S3150802C8F043F40033936208E0012387F85B3104E0CE
S3150802C90000BF02E000BF00E000BF97F85B31002BD2
S3150802C9100DD1744BD3F8E83023F03001D7F84C31F7
S3150802C920D3F8C8306F4A0B43C2F8E83003E097F8E9
S3150802C9305B3187F85A31D7F84C31D3E9002302F430
S3150802C9408003BB650023FB65D7E916120B46134322
S3150802C95033D0D7F84C31D3F8CC30002B02D0402B49
S3150802C96007D010E05F4B9B6A5E4A43F4003393623A
S3150802C9700DE0D7F84C310833184603F06FFB03462F
S3150802C98087F85B3103E0012387F85B3100BF97F82C
S3150802C9905B31002B0DD1534BD3F8E43023F0400121
S3150802C9A0D7F84C31D3F8CC304E4A0B43C2F8E430B0
S3150802C9B003E097F85B3187F85A31D7F84C31D3E957
S3150802C9C0002302F400033B6500237B65D7E91412B2
S3150802C9D00B46134333D0D7F84C31D3F8D030002B5B
S3150802C9E002D0802B07D010E03E4B9B6A3D4A43F4A7
S3150802C9F0003393620DE0D7F84C310833184603F03A
S3150802CA002DFB034687F85B3103E0012387F85B3188
S3150802CA1000BF97F85B31002B0DD1324BD3F8E430C7
S3150802CA2023F08001D7F84C31D3F8D0302D4A0B4386
S3150802CA30C2F8E43003E097F85B3187F85A31D7F841
S3150802CA404C31D3E9002302F00063BB640023FB6484
S3150802CA50D7E912120B4613434AD0D7F84C31D3F80A
S3150802CA60E030042B27D801A252F823F081CA020823
S3150802CA708FCA0208A3CA0208BFCA0208BFCA0208A6
S3150802CA80184B9B6A174A43F40033936218E0D7F8A7
S3150802CA904C310833184603F0E1FA034687F85B314E
S3150802CAA00EE0D7F84C313033184603F06FFB0346D5
S3150802CAB087F85B3104E0012387F85B3100E000BFA9
S3150802CAC097F85B31002B0FD1064BD3F8E03023F0F1
S3150802CAD00701D7F84C31D3F8E030024A0B43C2F8C3
S3150802CAE0E03005E0000C024497F85B3187F85A31CA
S3150802CAF0D7F84C31D3E9002302F080533B64002374
S3150802CB007B64D7E910120B46134300F08180D7F8ED
S3150802CB104C31D3F8E430202B5FD801A252F823F027
S3150802CB20A5CB0208DBCB0208DBCB0208DBCB02086B
S3150802CB30DBCB0208DBCB0208DBCB0208DBCB020825
S3150802CB40B3CB0208DBCB0208DBCB0208DBCB02083D
S3150802CB50DBCB0208DBCB0208DBCB0208DBCB020805
S3150802CB60C7CB0208DBCB0208DBCB0208DBCB020809
S3150802CB70DBCB0208DBCB0208DBCB0208DBCB0208E5
S3150802CB80E3CB0208DBCB0208DBCB0208DBCB0208CD
S3150802CB90DBCB0208DBCB0208DBCB0208DBCB0208C5
S3150802CBA0E3CB0208AB4B9B6AAA4A43F4003393626F
S3150802CBB018E0D7F84C310833184603F04FFA034603
S3150802CBC087F85B310EE0D7F84C313033184603F05C
S3150802CBD0DDFA034687F85B3104E0012387F85B3107
S3150802CBE000E000BF97F85B31002B0DD1994BD3F8C3
S3150802CBF0E03023F03801D7F84C31D3F8E430954ABF
S3150802CC000B43C2F8E03003E097F85B3187F85A31F4
S3150802CC10D7F84C31D3E9002302F00053BB63002353
S3150802CC20FB63D7E90E120B4613434ED0D7F84C31A5
S3150802CC30D3F8E830B3F5807F2ED0B3F5807F27D8B6
S3150802CC40C02B2BD0C02B23D8802B17D0802B1FD8D4
S3150802CC50002B02D0402B07D01AE07E4B9B6A7D4AF6
S3150802CC6043F4003393621AE0D7F84C310833184676
S3150802CC7003F0F4F9034687F85B3110E0D7F84C3134
S3150802CC803033184603F082FA034687F85B3106E02A
S3150802CC90012387F85B3102E000BF00E000BF97F886
S3150802CCA05B31002B0DD16B4BD3F8E03023F4E071E6
S3150802CCB0D7F84C31D3F8E830664A0B43C2F8E0306D
S3150802CCC003E097F85B3187F85A31D7F84C31D3E944
S3150802CCD0002302F080433B6300237B63D7E90C12EF
S3150802CCE00B46134355D0D7F84C31D3F8EC30B3F58D
S3150802CCF0206F31D0B3F5206F2AD8B3F5006F2DD047
S3150802CD00B3F5006F24D8B3F5C06F29D0B3F5C06F59
S3150802CD101ED8B3F5806F11D0B3F5806F18D8002BE3
S3150802CD2020D0B3F5007F13D1D7F84C310833184613
S3150802CD3003F094F9034687F85B3114E0D7F84C31CF
S3150802CD403033184603F022FA034687F85B310AE0C5
S3150802CD50012387F85B3106E000BF04E000BF02E06A
S3150802CD6000BF00E000BF97F85B31002B0DD1394BAD
S3150802CD70D3F8E03023F46061D7F84C31D3F8EC30BD
S3150802CD80344A0B43C2F8E03003E097F85B3187F880
S3150802CD905A31D7F84C31D3E9002302F00043BB627B
S3150802CDA00023FB62D7E90A120B46134358D0D7F879
S3150802CDB04C31D3F8F030B3F5A04F31D0B3F5A04FCC
S3150802CDC02AD8B3F5804F2DD0B3F5804F24D8B3F5C2
S3150802CDD0405F29D0B3F5405F1ED8B3F5005F11D086
S3150802CDE0B3F5005F18D8002B20D0B3F5805F13D1B6
S3150802CDF0D7F84C310833184603F030F9034687F85A
S3150802CE005B3114E0D7F84C313033184603F0BEF9DB
S3150802CE10034687F85B310AE0012387F85B3106E0AF
S3150802CE2000BF04E000BF02E000BF00E000BF97F8C1
S3150802CE305B31002B10D1074BD3F8E03023F4E042E4
S3150802CE40D7F84C31D3F8F03002491343C1F8E03031
S3150802CE5006E000BF000C024497F85B3187F85A31A6
S3150802CE60D7F84C31D3E900230021396203F00103D4
S3150802CE707B62D7E908120B46134355D0D7F84C31D3
S3150802CE80D3F8F430B3F5203F31D0B3F5203F2AD892
S3150802CE90B3F5003F2DD0B3F5003F24D8B3F5C03F14
S3150802CEA029D0B3F5C03F1ED8B3F5803F11D0B3F5EC
S3150802CEB0803F18D8002B20D0B3F5004F13D1D7F8EE
S3150802CEC04C310833184603F0C9F8034687F85B3134
S3150802CED014E0D7F84C313033184603F057F90346B5
S3150802CEE087F85B310AE0012387F85B3106E000BF69
S3150802CEF004E000BF02E000BF00E000BF97F85B3124
S3150802CF00002B0DD1884BD3F8E03023F46032D7F8E2
S3150802CF104C31D3F8F43084491343C1F8E03003E0C6
S3150802CF2097F85B3187F85A31D7F84C31D3E90023A1
S3150802CF300021B96103F00203FB61D7E906120B4629
S3150802CF4013433DD0D7F84C31D3F8DC30032B1CD829
S3150802CF5001A252F823F000BF93CF020869CF020854
S3150802CF6077CF020893CF02086F4B9B6A6E4A43F447
S3150802CF70003393620EE0D7F84C310833184603F0B3
S3150802CF806DF8034687F85B3104E0012387F85B31C5
S3150802CF9000E000BF97F85B31002B0DD1624BD3F846
S3150802CFA0E43023F00302D7F84C31D3F8DC305E497B
S3150802CFB01343C1F8E43003E097F85B3187F85A3136
S3150802CFC0D7F84C31D3E900230021396103F0040371
S3150802CFD07B61D7E904120B4613433AD0D7F84C3192
S3150802CFE0D3F8BC30B3F5007F0ED0B3F5007F15D861
S3150802CFF0002B17D0B3F5807F10D14B4B9B6A4A4A58
S3150802D00043F4003393620EE0D7F84C3108331846DE
S3150802D01003F024F8034687F85B3104E0012387F816
S3150802D0205B3100E000BF97F85B31002B0DD13E4B18
S3150802D030D3F8E83023F44072D7F84C31D3F8BC3031
S3150802D04039491343C1F8E83003E097F85B3187F8AA
S3150802D0505A31D7F84C31D3E900230021B96003F0DD
S3150802D0601003FB60D7E902120B46134338D0D7F8F0
S3150802D0704C31D3F80031302B1BD0302B15D8102B5E
S3150802D08002D0202B07D010E0274B9B6A264A43F48E
S3150802D090003393620EE0D7F84C313033184603F06A
S3150802D0A075F8034687F85B3104E0012387F85B319C
S3150802D0B000E000BF97F85B31002B0DD11A4BD3F86D
S3150802D0C0E43023F03002D7F84C31D3F80031164950
S3150802D0D01343C1F8E43003E097F85B3187F85A3115
S3150802D0E0D7F84C31D3E900230021396003F008034D
S3150802D0F07B60D7E900120B4613430CD00A4BD3F8D0
S3150802D100E83023F0C002D7F84C31D3F8FC30064990
S3150802D1101343C1F8E83097F85A31184607F5B0773D
S3150802D120BD46BDE8B08F00BF000C024480B48BB088
S3150802D13000AF7860AD4B5B6BC3F308033B62AB4B46
S3150802D1409B6A03F00303FB61A84B9B6A1B0A03F065
S3150802D1503F03BB61A54B9B6A03F010037B61A34B9C
S3150802D1609B6BDB08C3F30C037A6902FB03F307EE36
S3150802D170903AF8EE677AC7ED047ABB69002B00F09D
S3150802D1802681FB69032B53D0FB69032B6FD8FB69F6
S3150802D190012B03D0FB69022B2BD068E0934B1B684B
S3150802D1A0DB0803F00303924A22FA03F3FB60FB68E7
S3150802D1B007EE903AF8EE676ABB6907EE903AF8EE20
S3150802D1C0677A86EEA77A3B6A07EE903AF8EE676ABE
S3150802D1D097ED046ADFED875AC6EE257A76EEA77AC8
S3150802D1E0F7EE006A77EEA67A67EE277AC7ED097A2E
S3150802D1F068E0BB6907EE903AF8EE677ADFED7E6A79
S3150802D20086EEA77A3B6A07EE903AF8EE676A97EDDA
S3150802D210046ADFED785AC6EE257A76EEA77AF7EE35
S3150802D220006A77EEA67A67EE277AC7ED097A49E0A9
S3150802D230BB6907EE903AF8EE677ADFED706A86EE1A
S3150802D240A77A3B6A07EE903AF8EE676A97ED046AA0
S3150802D250DFED685AC6EE257A76EEA77AF7EE006A09
S3150802D26077EEA67A67EE277AC7ED097A2AE05F4B48
S3150802D2701B68DB0803F003035D4A22FA03F3FB602B
S3150802D280FB6807EE903AF8EE676ABB6907EE903AD2
S3150802D290F8EE677A86EEA77A3B6A07EE903AF8EED8
S3150802D2A0676A97ED046ADFED535AC6EE257A76EE7B
S3150802D2B0A77AF7EE006A77EEA67A67EE277AC7EDBF
S3150802D2C0097A00BF494B1B6803F00073B3F1007F6C
S3150802D2D021D1464B9B6A03F48033002B17D0434B6C
S3150802D2E05B6B5B0A03F07F0307EE903AF8EE677A08
S3150802D2F0B7EE007A37EE877AD7ED096AC6EE877AED
S3150802D300FCEEE77A17EE902A7B681A6006E07B68DD
S3150802D31000221A6002E07B6800221A60334B1B68FF
S3150802D32003F00073B3F1007F21D1304B9B6A03F4FB
S3150802D3300033002B17D02D4B5B6B1B0C03F07F03BE
S3150802D34007EE903AF8EE677AB7EE007A37EE877A02
S3150802D350D7ED096AC6EE877AFCEEE77A17EE902AC7
S3150802D3607B685A6006E07B6800225A6002E07B68A6
S3150802D37000225A601D4B1B6803F00073B3F1007F4D
S3150802D38021D11A4B9B6A03F48023002B17D0174B23
S3150802D3905B6B1B0E03F07F0307EE903AF8EE677A93
S3150802D3A0B7EE007A37EE877AD7ED096AC6EE877A3C
S3150802D3B0FCEEE77A17EE902A7B689A6010E07B68A3
S3150802D3C000229A600CE07B6800229A6008E07B687B
S3150802D3D000221A607B6800225A607B6800229A60E3
S3150802D3E000BF2C37BD465DF8047B7047000C02442B
S3150802D3F00090D003000000460024744A001B374BF5
S3150802D40080B48BB000AF7860AD4BDB6BC3F3080317
S3150802D4103B62AB4BDB6A03F00303FB61A84BDB6A97
S3150802D4201B0A03F03F03BB61A54BDB6A03F010033B
S3150802D4307B61A34B1B6CDB08C3F30C037A6902FB03
S3150802D44003F307EE903AF8EE677AC7ED047ABB69FA
S3150802D450002B00F02681FB69032B53D0FB69032BB3
S3150802D4606FD8FB69012B03D0FB69022B2BD068E02E
S3150802D470934B1B68DB0803F00303924A22FA03F371
S3150802D480FB60FB6807EE903AF8EE676ABB6907EE3F
S3150802D490903AF8EE677A86EEA77A3B6A07EE903AF2
S3150802D4A0F8EE676A97ED046ADFED875AC6EE257AC3
S3150802D4B076EEA77AF7EE006A77EEA67A67EE277A0D
S3150802D4C0C7ED097A68E0BB6907EE903AF8EE677A23
S3150802D4D0DFED7E6A86EEA77A3B6A07EE903AF8EEA9
S3150802D4E0676A97ED046ADFED785AC6EE257A76EE14
S3150802D4F0A77AF7EE006A77EEA67A67EE277AC7ED7D
S3150802D500097A49E0BB6907EE903AF8EE677ADFEDE9
S3150802D510706A86EEA77A3B6A07EE903AF8EE676A71
S3150802D52097ED046ADFED685AC6EE257A76EEA77A93
S3150802D530F7EE006A77EEA67A67EE277AC7ED097ADA
S3150802D5402AE05F4B1B68DB0803F003035D4A22FAF5
S3150802D55003F3FB60FB6807EE903AF8EE676ABB696D
S3150802D56007EE903AF8EE677A86EEA77A3B6A07EEF6
S3150802D570903AF8EE676A97ED046ADFED535AC6EEFB
S3150802D580257A76EEA77AF7EE006A77EEA67A67EE3E
S3150802D590277AC7ED097A00BF494B1B6803F0006377
S3150802D5A0B3F1006F21D1464BDB6A03F48033002BBB
S3150802D5B017D0434BDB6B5B0A03F07F0307EE903A07
S3150802D5C0F8EE677AB7EE007A37EE877AD7ED096A08
S3150802D5D0C6EE877AFCEEE77A17EE902A7B681A601F
S3150802D5E006E07B6800221A6002E07B6800221A6065
S3150802D5F0334B1B6803F00063B3F1006F21D1304B44
S3150802D600DB6A03F40033002B17D02D4BDB6B1B0CA4
S3150802D61003F07F0307EE903AF8EE677AB7EE007AE0
S3150802D62037EE877AD7ED096AC6EE877AFCEEE77A8D
S3150802D63017EE902A7B685A6006E07B6800225A60D9
S3150802D64002E07B6800225A601D4B1B6803F00063E8
S3150802D650B3F1006F21D11A4BDB6A03F48023002B46
S3150802D66017D0174BDB6B1B0E03F07F0307EE903ABE
S3150802D670F8EE677AB7EE007A37EE877AD7ED096A57
S3150802D680C6EE877AFCEEE77A17EE902A7B689A60EE
S3150802D69010E07B6800229A600CE07B6800229A60A0
S3150802D6A008E07B6800221A607B6800225A607B6861
S3150802D6B000229A6000BF2C37BD465DF8047B70478E
S3150802D6C0000C02440090D003000000460024744A6D
S3150802D6D0001B374B80B48BB000AF7860AD4B5B6CE8
S3150802D6E0C3F308033B62AB4B1B6B03F00303FB61FB
S3150802D6F0A84B1B6B1B0A03F03F03BB61A54B1B6BB5
S3150802D70003F010037B61A34B9B6CDB08C3F30C038A
S3150802D7107A6902FB03F307EE903AF8EE677AC7EDE9
S3150802D720047ABB69002B00F02681FB69032B53D0D0
S3150802D730FB69032B6FD8FB69012B03D0FB69022B0C
S3150802D7402BD068E0934B1B68DB0803F00303924A6D
S3150802D75022FA03F3FB60FB6807EE903AF8EE676A73
S3150802D760BB6907EE903AF8EE677A86EEA77A3B6AC5
S3150802D77007EE903AF8EE676A97ED046ADFED875A84
S3150802D780C6EE257A76EEA77AF7EE006A77EEA67ADD
S3150802D79067EE277AC7ED097A68E0BB6907EE903A21
S3150802D7A0F8EE677ADFED7E6A86EEA77A3B6A07EEBF
S3150802D7B0903AF8EE676A97ED046ADFED785AC6EE94
S3150802D7C0257A76EEA77AF7EE006A77EEA67A67EEFC
S3150802D7D0277AC7ED097A49E0BB6907EE903AF8EE6F
S3150802D7E0677ADFED706A86EEA77A3B6A07EE903AA9
S3150802D7F0F8EE676A97ED046ADFED685AC6EE257A8F
S3150802D80076EEA77AF7EE006A77EEA67A67EE277AB9
S3150802D810C7ED097A2AE05F4B1B68DB0803F00303AE
S3150802D8205D4A22FA03F3FB60FB6807EE903AF8EECC
S3150802D830676ABB6907EE903AF8EE677A86EEA77AC8
S3150802D8403B6A07EE903AF8EE676A97ED046ADFEDEF
S3150802D850535AC6EE257A76EEA77AF7EE006A77EE7F
S3150802D860A67A67EE277AC7ED097A00BF494B1B6885
S3150802D87003F00053B3F1005F21D1464B1B6B03F44F
S3150802D8808033002B17D0434B5B6C5B0A03F07F0394
S3150802D89007EE903AF8EE677AB7EE007A37EE877AAD
S3150802D8A0D7ED096AC6EE877AFCEEE77A17EE902A72
S3150802D8B07B681A6006E07B6800221A6002E07B68D1
S3150802D8C000221A60334B1B6803F00053B3F1005F62
S3150802D8D021D1304B1B6B03F40033002B17D02D4B91
S3150802D8E05B6C1B0C03F07F0307EE903AF8EE677A3F
S3150802D8F0B7EE007A37EE877AD7ED096AC6EE877AE7
S3150802D900FCEEE77A17EE902A7B685A6006E07B6897
S3150802D91000225A6002E07B6800225A601D4B1B688F
S3150802D92003F00053B3F1005F21D11A4B1B6B03F4CA
S3150802D9308023002B17D0174B5B6C1B0E03F07F035B
S3150802D94007EE903AF8EE677AB7EE007A37EE877AFC
S3150802D950D7ED096AC6EE877AFCEEE77A17EE902AC1
S3150802D9607B689A6010E07B6800229A600CE07B680C
S3150802D97000229A6008E07B6800221A607B6800220F
S3150802D9805A607B6800229A6000BF2C37BD465DF854
S3150802D990047B7047000C02440090D0030000004646
S3150802D9A00024744A001B374B90B58FB000AFC7E905
S3150802D9B00001D7E9000100F17E44214350D1264BEC
S3150802D9C0D3F8F03003F440733B63234BD3F8F030BB
S3150802D9D003F00203022B08D13B6BB3F5807F04D117
S3150802D9E04FF400437B6302F02ABB1B4BD3F8F0309B
S3150802D9F003F00063B3F1006F08D13B6BB3F5007F08
S3150802DA0004D14FF4FA437B6302F019BB124B1B682D
S3150802DA1003F40033B3F5003F19D13B6BB3F5407FEE
S3150802DA2015D10D4BDB6903F47C53B3F5007F0AD39A
S3150802DA30094BDB691B0A03F03F03084AB2FBF3F3FF
S3150802DA407B6302F0FCBA00237B6302F0F8BA002378
S3150802DA507B6302F0F4BA00BF000C0244001BB70055
S3150802DA60D7E90001A1F5806450EA040101F0758244
S3150802DA70D7E90001012871F5806182F0DD82D7E9D4
S3150802DA800001A1F5007450EA040101F06C81D7E99E
S3150802DA900001012871F5007182F0CE82D7E90001F2
S3150802DAA0A1F5807450EA040101F00286D7E9000163
S3150802DAB0012871F5807182F0BF82D7E90001A1F1D0
S3150802DAC0800450EA040101F04C85D7E900010128D7
S3150802DAD071F1800182F0B082D7E90001A1F1400418
S3150802DAE050EA040101F09E84D7E90001012871F188
S3150802DAF0400182F0A182D7E90001A1F1200450EA8F
S3150802DB00040101F0E883D7E90001012871F1200137
S3150802DB1082F09282D7E90001A1F1100450EA0401C9
S3150802DB2002F05682D7E90001012871F1100182F04C
S3150802DB308382D7E90001A1F1080450EA040102F040
S3150802DB40CC81D7E90001012871F1080182F07482BB
S3150802DB50D7E900010C1F50EA040101F04886D7E90B
S3150802DB600001012871F1040182F06682D7E90001F9
S3150802DB708C1E50EA040102F04381D7E9000101280C
S3150802DB8071F1020182F05882D7E900014C1E50EA6F
S3150802DB90040102F0CE80D7E90001012871F10101E2
S3150802DBA082F04A82D7E9000100F10044214302F0DB
S3150802DBB05980D7E90001D94CA04271F1000182F0DF
S3150802DBC03B82D7E9000100F14044214301F0D9879D
S3150802DBD0D7E90001D24CA04271F1000182F02C82F1
S3150802DBE0D7E9000100F16044214301F05187D7E9E2
S3150802DBF00001CC4CA04271F1000182F01D82D7E9E6
S3150802DC00000100F17044214301F09A86D7E9000128
S3150802DC10C54CA04271F1000182F00E82D7E90001DB
S3150802DC2000F17844214301F01286D7E90001BF4C7E
S3150802DC30A04271F1000182F0FF81D7E9000100F1EB
S3150802DC407C44214302F07E81D7E90001B84CA04208
S3150802DC5071F1000182F0F081D7E90001A0F5000414
S3150802DC60214300F09E82D7E90001B24CA04271F12D
S3150802DC70000182F0E181D7E90001A0F58004214381
S3150802DC8000F06D82D7E90001AB4CA04271F10001A8
S3150802DC9082F0D281D7E90001A0F50014214301F0F0
S3150802DCA00D80D7E90001A54CA04271F1000182F06E
S3150802DCB0C381D7E90001A0F58014214300F0D08181
S3150802DCC0D7E900019E4CA04271F1000182F0B481AD
S3150802DCD0D7E90001A0F50024214300F04281D7E9E3
S3150802DCE00001984CA04271F1000182F0A581D7E9A2
S3150802DCF00001A0F58024214301F04E82D7E90001F4
S3150802DD00914CA04271F1000182F09681D7E9000197
S3150802DD10A0F50034214301F09781D7E900018B4C25
S3150802DD20A04271F1000182F08781D7E90001A0F5CE
S3150802DD308034214301F05481D7E90001B0F1011F73
S3150802DD4071F1000182F07881D7E90001A0F500445B
S3150802DD50214301F0B780D7E9000148F20104A04245
S3150802DD6071F1000182F06881D7E90001A0F58044CB
S3150802DD70214301F06480D7E9000144F20104A0427C
S3150802DD8071F1000182F05881D7E90001A0F500542B
S3150802DD90214301F01180D7E9000142F20104A042B1
S3150802DDA071F1000182F04881D7E90001A0F580549B
S3150802DDB0214300F01E87D7E9000141F20104A0427F
S3150802DDC071F1000182F03881D7E90001A0F50064FB
S3150802DDD0214300F0A886D7E9000140F60104A042D3
S3150802DDE071F1000182F02881D7E90001A0F580646B
S3150802DDF0214300F03286D7E9000140F20144A042ED
S3150802DE0071F1000182F01881D7E90001A0F50074CA
S3150802DE10214300F0B085D7E9000140F20124A0426F
S3150802DE2071F1000182F00881D7E90001A0F580743A
S3150802DE30214300F03585D7E9000140F20114A042DA
S3150802DE4071F1000182F0F880D7E90001A0F180049F
S3150802DE50214300F0BA84D7E90001812871F1000153
S3150802DE6082F0EA80D7E90001212871F100016FD218
S3150802DE70D7E90001014302F0DF80D7E90001421E1B
S3150802DE8041F1FF33202A73F1000182F0D5801F2A5F
S3150802DE9002F2D28001A151F822F000BFFDE1020888
S3150802DEA0C9E202083900030889E3020839000308AF
S3150802DEB0390003083900030859E40208390003083F
S3150802DEC03900030839000308390003083900030832
S3150802DED039000308390003083BE50208390003083C
S3150802DEE03900030839000308390003083900030812
S3150802DEF03900030839000308390003083900030802
S3150802DF0039000308390003083900030839000308F1
S3150802DF10390003083900030811E6020801000080E7
S3150802DF200100004001000020010000100100000865
S3150802DF3001000004010080000100400001002000E9
S3150802DF40010010000100080001000400010002009F
S3150802DF50D7E90023A2F140010B4300F0C48302F083
S3150802DF606BB8A14BD3F8E83003F4E0233B633B6B71
S3150802DF70B3F5802F36D03B6BB3F5802F6BD83B6B4E
S3150802DF80B3F5403F2BD03B6BB3F5403F63D83B6BB1
S3150802DF90B3F5003F1BD03B6BB3F5003F5BD83B6B39
S3150802DFA0002B04D03B6BB3F5803F08D053E007F152
S3150802DFB020031846FFF7BAF87B6A7B634EE007F13F
S3150802DFC014031846FFF71CFA7B697B6346E007F1E0
S3150802DFD008031846FFF77EFBBB687B633EE0834B6C
S3150802DFE07B633BE0804BD3F8E83003F04043FB62A7
S3150802DFF07D4B1B6803F00203022B0CD1FB6A002B34
S3150802E00009D1794B1B68DB0803F00303784A22FA25
S3150802E01003F37B631EE0744B1B6803F40073B3F5CA
S3150802E020007F06D1FB6AB3F1804F02D1714B7B6345
S3150802E03010E06D4B1B6803F40033B3F5003F06D1BD
S3150802E040FB6AB3F1004F02D16B4B7B6302E00023FC
S3150802E0507B6303E002E000237B6300BF01F0EFBFAE
S3150802E060614BD3F8E83003F460133B633B6BB3F5BB
S3150802E070001F36D03B6BB3F5001F6BD83B6BB3F56D
S3150802E080C01F2BD03B6BB3F5C01F63D83B6BB3F5F0
S3150802E090801F1BD03B6BB3F5801F5BD83B6B002BF5
S3150802E0A004D03B6BB3F5002F08D053E007F12003E9
S3150802E0B01846FFF73BF87B6A7B634EE007F11403C9
S3150802E0C01846FFF79DF97B697B6346E007F108036B
S3150802E0D01846FFF7FFFABB687B633EE0434B7B6358
S3150802E0E03BE0414BD3F8E83003F04043FB623E4B3A
S3150802E0F01B6803F00203022B0CD1FB6A002B09D121
S3150802E100394B1B68DB0803F00303394A22FA03F387
S3150802E1107B631EE0344B1B6803F40073B3F5007F80
S3150802E12006D1FB6AB3F1804F02D1324B7B6310E012
S3150802E1302D4B1B6803F40033B3F5003F06D1FB6A87
S3150802E140B3F1004F02D12C4B7B6302E000237B63C1
S3150802E15003E002E000237B6300BF01F070BF224B9D
S3150802E160D3F8E43003F040033B633B6B002B08D142
S3150802E17007F120031846FEF7D9FF7B6A7B6301F095
S3150802E1805EBF3B6B402B08D107F114031846FFF715
S3150802E19037F9FB697B6301F052BF00237B6301F009
S3150802E1A04EBF114BD3F8E43003F080033B633B6B5D
S3150802E1B0002B08D107F120031846FEF7B7FF7B6A42
S3150802E1C07B6301F03CBF3B6B802B08D107F114033C
S3150802E1D01846FFF715F9FB697B6301F030BF002388
S3150802E1E07B6301F02CBF00BF000C02440080BB0019
S3150802E1F00090D00300093D00001BB7009D4BD3F8E1
S3150802E200D83003F007033B633B6B002B04D1FCF7C2
S3150802E2109FFF786301F013BF964B1B6803F00063F8
S3150802E220B3F1006F0AD13B6B012B07D107F1140337
S3150802E2301846FFF7E5F8BB697B6343E08D4B1B681D
S3150802E24003F00053B3F1005F0AD13B6B022B07D1EF
S3150802E25007F108031846FFF73DFAFB687B6331E0CE
S3150802E260844B1B6803F00203022B0CD13B6B032B76
S3150802E27009D1804B1B68DB0803F003037E4A22FAA6
S3150802E28003F37B631EE07B4B1B6803F40073B3F551
S3150802E290007F05D13B6B042B02D1784B7B6311E0DF
S3150802E2A0744BD3F8F03003F00203022B06D13B6B12
S3150802E2B0052B03D14FF400437B6303E000237B6302
S3150802E2C001F0BDBE01F0BBBE6A4BD3F8D83003F0ED
S3150802E2D038033B633B6B002B04D1FCF723FF7863BF
S3150802E2E001F0ADBE634B1B6803F00063B3F1006F28
S3150802E2F00AD13B6B082B07D107F114031846FFF71F
S3150802E3007FF8BB697B633DE03B6B102B08D107F1B5
S3150802E31008031846FFF7DEF9FB687B6301F08FBE38
S3150802E320544B1B6803F00203022B0CD13B6B182BD0
S3150802E33009D1504B1B68DB0803F003034E4A22FA45
S3150802E34003F37B631EE04B4B1B6803F40073B3F5C0
S3150802E350007F05D13B6B202B02D1484B7B6311E032
S3150802E360444BD3F8F03003F00203022B06D13B6B81
S3150802E370282B03D14FF400437B6303E000237B631E
S3150802E38001F05DBE01F05BBE3A4BD3F8D83003F418
S3150802E390E0733B633B6B002B04D1FCF7C3FE786347
S3150802E3A001F04DBE334B1B6803F00063B3F1006FF7
S3150802E3B00AD13B6B402B07D107F114031846FFF726
S3150802E3C01FF8BB697B6345E02A4B1B6803F00053C1
S3150802E3D0B3F1005F0AD13B6B802B07D107F1080323
S3150802E3E01846FFF777F9FB687B6333E0214B1B6816
S3150802E3F003F00203022B0CD13B6BC02B09D11D4B38
S3150802E4001B68DB0803F003031B4A22FA03F37B6348
S3150802E41020E0184B1B6803F40073B3F5007F06D19E
S3150802E4203B6BB3F5807F02D1144B7B6312E0114B31
S3150802E430D3F8F03003F00203022B07D13B6BB3F596
S3150802E440A07F03D14FF400437B6303E000237B6381
S3150802E45001F0F5BD01F0F3BD064BD3F8D83003F44D
S3150802E46060633B633B6B002B0AD1FCF75BFE786368
S3150802E47001F0E5BD000C02440090D00300093D00FE
S3150802E480A04B1B6803F00063B3F1006F0BD13B6B23
S3150802E490B3F5007F07D107F114031846FEF7B0FF5C
S3150802E4A0BB697B6347E0974B1B6803F00053B3F1E4
S3150802E4B0005F0BD13B6BB3F5806F07D107F10803F9
S3150802E4C01846FFF707F9FB687B6334E08D4B1B6838
S3150802E4D003F00203022B0DD13B6BB3F5C06F09D1D2
S3150802E4E0884B1B68DB0803F00303874A22FA03F307
S3150802E4F07B6320E0834B1B6803F40073B3F5007F4C
S3150802E50006D13B6BB3F5006F02D1804B7B6312E0F9
S3150802E5107C4BD3F8F03003F00203022B07D13B6B96
S3150802E520B3F5206F03D14FF400437B6303E0002366
S3150802E5307B6301F084BD01F082BD724BD3F8D830FB
S3150802E54003F4E0433B633B6B002B04D1FCF7EAFD83
S3150802E550786301F074BD6B4B1B6803F00063B3F17B
S3150802E560006F0BD13B6BB3F5805F07D107F114033C
S3150802E5701846FEF745FFBB697B6347E0614B1B689C
S3150802E58003F00053B3F1005F0BD13B6BB3F5005FA9
S3150802E59007D107F108031846FFF79CF8FB687B6367
S3150802E5A034E0584B1B6803F00203022B0DD13B6B78
S3150802E5B0B3F5405F09D1534B1B68DB0803F003032D
S3150802E5C0514A22FA03F37B6320E04E4B1B6803F49D
S3150802E5D00073B3F5007F06D13B6BB3F5804F02D1CA
S3150802E5E04A4B7B6312E0474BD3F8F03003F0020341
S3150802E5F0022B07D13B6BB3F5A04F03D14FF400436F
S3150802E6007B6303E000237B6301F019BD01F017BDAC
S3150802E6103C4BD3F8D83003F460333B633B6B002B97
S3150802E62004D1FCF77FFD786301F009BD354B1B6801
S3150802E63003F00063B3F1006F0BD13B6BB3F5004FE8
S3150802E64007D107F114031846FEF7DAFEBB697B63A6
S3150802E65047E02C4B1B6803F00053B3F1005F0BD164
S3150802E6603B6BB3F5803F07D107F108031846FFF75E
S3150802E67031F8FB687B6334E0224B1B6803F0020324
S3150802E680022B0DD13B6BB3F5C03F09D11D4B1B685D
S3150802E690DB0803F003031C4A22FA03F37B6320E038
S3150802E6A0184B1B6803F40073B3F5007F06D13B6B66
S3150802E6B0B3F5003F02D1154B7B6312E0114BD3F839
S3150802E6C0F03003F00203022B07D13B6BB3F5203F70
S3150802E6D003D14FF400437B6303E000237B6301F01D
S3150802E6E0AEBC01F0ACBC074BD3F8D83003F4E01348
S3150802E6F03B633B6B002B0BD1FCF714FD786301F0EF
S3150802E7009EBC00BF000C02440090D00300093D00E5
S3150802E710A04B1B6803F00063B3F1006F0BD13B6B90
S3150802E720B3F5802F07D107F114031846FEF768FEE2
S3150802E730BB697B6347E0974B1B6803F00053B3F151
S3150802E740005F0BD13B6BB3F5002F07D107F1080326
S3150802E7501846FEF7BFFFFB687B6334E08D4B1B68E8
S3150802E76003F00203022B0DD13B6BB3F5402F09D1FF
S3150802E770884B1B68DB0803F00303874A22FA03F374
S3150802E7807B6320E0834B1B6803F40073B3F5007FB9
S3150802E79006D13B6BB3F5801F02D1804B7B6312E037
S3150802E7A07C4BD3F8F03003F00203022B07D13B6B04
S3150802E7B0B3F5A01F03D14FF400437B6303E00023A4
S3150802E7C07B6301F03CBC01F03ABC724BD3F8D830FB
S3150802E7D003F460033B633B6B002B04D1FCF7A2FCFA
S3150802E7E0786301F02CBC6B4B1B6803F00063B3F132
S3150802E7F0006F0BD13B6BB3F5001F07D107F114036A
S3150802E8001846FEF7FDFDBB697B6347E0614B1B6853
S3150802E81003F00053B3F1005F0BD13B6BB3F5800FE6
S3150802E82007D107F108031846FEF754FFFB687B6316
S3150802E83034E0584B1B6803F00203022B0DD13B6BE5
S3150802E840B3F5C00F09D1534B1B68DB0803F003036A
S3150802E850514A22FA03F37B6320E04E4B1B6803F40A
S3150802E8600073B3F5007F06D13B6BB3F5000F02D1F7
S3150802E8704A4B7B6312E0474BD3F8F03003F00203AE
S3150802E880022B07D13B6BB3F5200F03D14FF400439C
S3150802E8907B6303E000237B6301F0D1BB01F0CFBBAE
S3150802E8A03C4BD3F8D83003F0E0633B633B6B002B59
S3150802E8B004D1FCF737FC786301F0C1BB354B1B6802
S3150802E8C003F00063B3F1006F0BD13B6BB3F1807FAA
S3150802E8D007D107F114031846FEF792FDBB697B635D
S3150802E8E047E02C4B1B6803F00053B3F1005F0BD1D2
S3150802E8F03B6BB3F1007F07D107F108031846FEF711
S3150802E900E9FEFB687B6334E0224B1B6803F00203D3
S3150802E910022B0DD13B6BB3F1407F09D11D4B1B680E
S3150802E920DB0803F003031C4A22FA03F37B6320E0A5
S3150802E930184B1B6803F40073B3F5007F06D13B6BD3
S3150802E940B3F1806F02D1154B7B6312E0114BD3F8FA
S3150802E950F03003F00203022B07D13B6BB3F1A06F31
S3150802E96003D14FF400437B6303E000237B6301F08A
S3150802E97066BB01F064BB074BD3F8D83003F060538B
S3150802E9803B633B6B002B0BD1FCF7CCFB786301F0A6
S3150802E99056BB00BF000C02440090D00300093D009C
S3150802E9A0A14B1B6803F00063B3F1006F0BD13B6BFD
S3150802E9B0B3F1006F07D107F114031846FEF720FDDD
S3150802E9C0BB697B6347E0984B1B6803F00053B3F1BE
S3150802E9D0005F0BD13B6BB3F1805F07D107F10803E8
S3150802E9E01846FEF777FEFB687B6334E08E4B1B689E
S3150802E9F003F00203022B0DD13B6BB3F1C05F09D1C1
S3150802EA00894B1B68DB0803F00303884A22FA03F3DF
S3150802EA107B6320E0844B1B6803F40073B3F5007F25
S3150802EA2006D13B6BB3F1005F02D1814B7B6312E0E7
S3150802EA307D4BD3F8F03003F00203022B07D13B6B70
S3150802EA40B3F1205F03D14FF400437B6303E0002355
S3150802EA507B6301F0F4BA01F0F2BA734BD3F8DC30F7
S3150802EA6003F007033B633B6B002B04D1FCF75AFB0D
S3150802EA70786301F0E4BA6C4B1B6803F00063B3F1E8
S3150802EA80006F0AD13B6B012B07D107F11403184615
S3150802EA90FEF7B6FCBB697B6343E0634B1B6803F076
S3150802EAA00053B3F1005F0AD13B6B022B07D107F182
S3150802EAB008031846FEF70EFEFB687B6331E05A4BE5
S3150802EAC01B6803F00203022B0CD13B6B032B09D103
S3150802EAD0554B1B68DB0803F00303544A22FA03F377
S3150802EAE07B631EE0504B1B6803F40073B3F5007F8B
S3150802EAF005D13B6B042B02D14D4B7B6311E04A4B8C
S3150802EB00D3F8F03003F00203022B06D13B6B052B38
S3150802EB1003D14FF400437B6303E000237B6301F0D8
S3150802EB208EBA01F08CBA404BD3F8DC3003F070038E
S3150802EB303B633B6B002B04D1FCF7F4FA786301F0D4
S3150802EB407EBA394B1B6803F00063B3F1006F0AD132
S3150802EB503B6B102B07D107F114031846FEF750FC3E
S3150802EB60BB697B6343E0304B1B6803F00053B3F188
S3150802EB70005F0AD13B6B202B07D107F10803184621
S3150802EB80FEF7A8FDFB687B6331E0274B1B6803F0A1
S3150802EB900203022B0CD13B6B302B09D1224B1B688B
S3150802EBA0DB0803F00303214A22FA03F37B631EE020
S3150802EBB01D4B1B6803F40073B3F5007F05D13B6B4D
S3150802EBC0402B02D11A4B7B6311E0174BD3F8F03076
S3150802EBD003F00203022B06D13B6B502B03D14FF4F1
S3150802EBE000437B6303E000237B6301F028BA01F04C
S3150802EBF026BA0D4BD3F8E03003F0E0633B633B6B78
S3150802EC00002B04D1FCF7BAFA786301F018BA3B6B09
S3150802EC10B3F1807F0ED107F114031846FEF7F0FB15
S3150802EC20BB697B6301F00BBA000C02440090D00367
S3150802EC3000093D003B6BB3F1007F08D107F10803D9
S3150802EC401846FEF747FDFB687B6301F0F8B9A44B4B
S3150802EC501B6803F00203022B0DD13B6BB3F1407F15
S3150802EC6009D19F4B1B68DB0803F003039D4A22FA6E
S3150802EC7003F37B6320E09A4B1B6803F40073B3F536
S3150802EC80007F06D13B6BB3F1806F02D1964B7B6353
S3150802EC9012E0934BD3F8F03003F00203022B07D1AC
S3150802ECA03B6BB3F1A06F03D14FF400437B6303E0E0
S3150802ECB000237B6301F0C3B901F0C1B9884BD3F8CD
S3150802ECC0E83003F007033B633B6B002B04D1FCF7E8
S3150802ECD00DFA786301F0B3B93B6B012B04D1FCF74B
S3150802ECE0D9F8786301F0ABB93B6B022B08D107F16F
S3150802ECF014031846FEF784FBFB697B6301F09FB990
S3150802ED00774B1B6803F40033B3F5003F05D13B6B21
S3150802ED10032B02D1754B7B6323E0714B1B6803F00F
S3150802ED200203022B0CD13B6B042B09D16C4B1B68DB
S3150802ED30DB0803F003036B4A22FA03F37B6310E052
S3150802ED40674B1B6803F40073B3F5007F05D13B6B71
S3150802ED50052B02D1644B7B6303E000237B6301F03E
S3150802ED606EB901F06CB95E4BD3F8E83003F00803CC
S3150802ED703B635B4BD3F8F03003F00203022B06D158
S3150802ED803B6B002B03D14FF400437B6312E0544BD9
S3150802ED90D3F8F03003F00063B3F1006F06D13B6B92
S3150802EDA0082B03D14FF4FA437B6303E000237B630A
S3150802EDB001F045B901F043B9494BD3F8E43003F4FD
S3150802EDC040333B633B6B002B04D1FCF7ABF978630A
S3150802EDD001F035B93B6BB3F5803F08D107F108035B
S3150802EDE01846FEF777FC3B697B6301F028B93C4B72
S3150802EDF01B6803F00203022B0DD13B6BB3F5003FF0
S3150802EE0009D1374B1B68DB0803F00303354A22FA9C
S3150802EE1003F37B6311E0324B1B6803F40073B3F50B
S3150802EE20007F06D13B6BB3F5403F02D12E4B7B6385
S3150802EE3003E000237B6301F002B901F000B9284B15
S3150802EE40D3F8E43003F440233B633B6B002B04D135
S3150802EE50FCF768F9786301F0F2B83B6BB3F5802FDB
S3150802EE6008D107F108031846FEF734FC3B697B63B1
S3150802EE7001F0E5B81A4B1B6803F00203022B0DD109
S3150802EE803B6BB3F5002F09D1154B1B68DB0803F062
S3150802EE900303144A22FA03F37B6311E0104B1B683F
S3150802EEA003F40073B3F5007F06D13B6BB3F5402F2D
S3150802EEB002D10D4B7B6303E000237B6301F0BFB8ED
S3150802EEC001F0BDB8064BD3F8E43003F440133B63B4
S3150802EED03B6B002B0CD1FCF751F9786301F0AFB804
S3150802EEE0000C02440090D00300093D00001BB70045
S3150802EEF03B6BB3F5801F08D107F108031846FEF7E6
S3150802EF00E9FB3B697B6301F09AB89F4B1B6803F0E8
S3150802EF100203022B0DD13B6BB3F5001F09D19A4BA5
S3150802EF201B68DB0803F00303984A22FA03F37B63A0
S3150802EF3011E0954B1B6803F40073B3F5007F06D105
S3150802EF403B6BB3F5401F02D1914B7B6303E0002371
S3150802EF507B6301F074B801F072B88B4BD3F8E430D6
S3150802EF6003F440033B633B6B002B04D1FCF706F921
S3150802EF70786301F064B83B6BB3F5800F08D107F1EB
S3150802EF8008031846FEF7A6FB3B697B6301F057B8F0
S3150802EF907D4B1B6803F00203022B0DD13B6BB3F5C5
S3150802EFA0000F09D1784B1B68DB0803F00303774A85
S3150802EFB022FA03F37B6311E0734B1B6803F40073B5
S3150802EFC0B3F5007F06D13B6BB3F5400F02D1704B08
S3150802EFD07B6303E000237B6301F031B801F02FB8AD
S3150802EFE0694BD3F8E43003F040733B633B6B002B69
S3150802EFF004D1FCF797F8786301F021B83B6BB3F1BB
S3150802F000807F08D107F108031846FEF763FB3B69C0
S3150802F0107B6301F014B85C4B1B6803F00203022BF6
S3150802F0200ED13B6BB3F1007F0AD1574B1B68DB0845
S3150802F03003F00303554A22FA03F37B6300F0FFBF8A
S3150802F04000237B6300F0FBBF4F4BD3F8DC3003F49D
S3150802F050E0633B633B6BB3F5A06F56D03B6BB3F5EE
S3150802F060A06F00F28B803B6BB3F5806F3ED03B6B93
S3150802F070B3F5806F00F282803B6BB3F5407F27D0F1
S3150802F0803B6BB3F5407F79D83B6BB3F5007F17D05E
S3150802F0903B6BB3F5007F71D83B6B002B04D03B6BFF
S3150802F0A0B3F5807F04D069E0FCF768F8786368E016
S3150802F0B007F114031846FEF7A3F97B697B6360E040
S3150802F0C007F108031846FEF705FB3B697B6358E020
S3150802F0D02D4BD3F8F03003F00203022B03D14FF481
S3150802F0E000437B634DE000237B634AE0264BD3F85B
S3150802F0F0F03003F00063B3F1006F03D14FF4FA4323
S3150802F1007B633EE000237B633BE01F4BD3F8E8308A
S3150802F11003F04043FB621C4B1B6803F00203022BFD
S3150802F1200CD1FB6A002B09D1174B1B68DB0803F0CD
S3150802F1300303164A22FA03F37B631EE0124B1B688B
S3150802F14003F40073B3F5007F06D1FB6AB3F1804F6F
S3150802F15002D10F4B7B6310E00B4B1B6803F40033A1
S3150802F160B3F5003F06D1FB6AB3F1004F02D1094B52
S3150802F1707B6302E000237B6303E002E000237B63F8
S3150802F18000BF00F05CBF00BF000C02440090D00331
S3150802F19000093D00001BB7009E4BD3F8DC3003F490
S3150802F1A0E0433B633B6BB3F5A04F56D03B6BB3F5DD
S3150802F1B0A04F00F28B803B6BB3F5804F3ED03B6B82
S3150802F1C0B3F5804F00F282803B6BB3F5405F27D0E0
S3150802F1D03B6BB3F5405F79D83B6BB3F5005F17D04D
S3150802F1E03B6BB3F5005F71D83B6B002B04D03B6BCE
S3150802F1F0B3F5805F04D069E0FBF794FF786368E0B3
S3150802F20007F114031846FEF7FBF87B697B6360E097
S3150802F21007F108031846FEF75DFA3B697B6358E077
S3150802F2207C4BD3F8F03003F00203022B03D14FF4E0
S3150802F23000437B634DE000237B634AE0754BD3F8BA
S3150802F240F03003F00063B3F1006F03D14FF4FA43D1
S3150802F2507B633EE000237B633BE06E4BD3F8E830EA
S3150802F26003F04043FB626B4B1B6803F00203022B5D
S3150802F2700CD1FB6A002B09D1664B1B68DB0803F02D
S3150802F2800303654A22FA03F37B631EE0614B1B689C
S3150802F29003F40073B3F5007F06D1FB6AB3F1804F1E
S3150802F2A002D15E4B7B6310E05A4B1B6803F40033B2
S3150802F2B0B3F5003F06D1FB6AB3F1004F02D1584BB2
S3150802F2C07B6302E000237B6303E002E000237B63A7
S3150802F2D000BF00F0B4BE4F4BD3F8DC3003F4E02392
S3150802F2E03B633B6BB3F5A02F56D03B6BB3F5A02F10
S3150802F2F000F28B803B6BB3F5802F3ED03B6BB3F5A8
S3150802F300802F00F282803B6BB3F5403F27D03B6BE0
S3150802F310B3F5403F79D83B6BB3F5003F17D03B6B4B
S3150802F320B3F5003F71D83B6B002B04D03B6BB3F5AA
S3150802F330803F04D069E0FBF721FF786368E007F1B4
S3150802F34014031846FEF75CF87B697B6360E007F1F5
S3150802F35008031846FEF7BEF93B697B6358E02D4B56
S3150802F360D3F8F03003F00203022B03D14FF4004323
S3150802F3707B634DE000237B634AE0264BD3F8F030EB
S3150802F38003F00063B3F1006F03D14FF4FA437B63D2
S3150802F3903EE000237B633BE01E4BD3F8E83003F0E4
S3150802F3A04043FB621B4B1B6803F00203022B0CD182
S3150802F3B0FB6A002B09D1174B1B68DB0803F0030312
S3150802F3C0154A22FA03F37B631EE0124B1B6803F409
S3150802F3D00073B3F5007F06D1FB6AB3F1804F02D101
S3150802F3E00E4B7B6310E00B4B1B6803F40033B3F53B
S3150802F3F0003F06D1FB6AB3F1004F02D1084B7B638B
S3150802F40002E000237B6303E002E000237B6300BF84
S3150802F41000F015BE000C02440090D00300093D001E
S3150802F420001BB7009E4BD3F8DC3003F4E0033B63C2
S3150802F4303B6BB3F5A00F56D03B6BB3F5A00F00F2AA
S3150802F4408B803B6BB3F5800F3ED03B6BB3F5800FD9
S3150802F45000F282803B6BB3F5401F27D03B6BB3F5B6
S3150802F460401F79D83B6BB3F5001F17D03B6BB3F53A
S3150802F470001F71D83B6B002B04D03B6BB3F5801F82
S3150802F48004D069E0FBF77AFE786368E007F11403B3
S3150802F4901846FDF7B5FF7B697B6360E007F1080351
S3150802F4A01846FEF717F93B697B6358E07C4BD3F89D
S3150802F4B0F03003F00203022B03D14FF400437B63BF
S3150802F4C04DE000237B634AE0754BD3F8F03003F036
S3150802F4D00063B3F1006F03D14FF4FA437B633EE056
S3150802F4E000237B633BE06E4BD3F8E83003F04043DE
S3150802F4F0FB626B4B1B6803F00203022B0CD1FB6AFF
S3150802F500002B09D1664B1B68DB0803F00303654A27
S3150802F51022FA03F37B631EE0614B1B6803F4007354
S3150802F520B3F5007F06D1FB6AB3F1804F02D15E4B79
S3150802F5307B6310E05A4B1B6803F40033B3F5003FB4
S3150802F54006D1FB6AB3F1004F02D1584B7B6302E046
S3150802F55000237B6303E002E000237B6300BF00F025
S3150802F5606EBD4F4BD3F8DC3003F0E0633B633B6B75
S3150802F570B3F1A06F56D03B6BB3F1A06F00F28B804C
S3150802F5803B6BB3F1806F3ED03B6BB3F1806F00F2F9
S3150802F59082803B6BB3F1407F27D03B6BB3F1407F50
S3150802F5A079D83B6BB3F1007F17D03B6BB3F1007F81
S3150802F5B071D83B6B002B04D03B6BB3F1807F04D030
S3150802F5C069E0FBF7DBFD786368E007F11403184688
S3150802F5D0FDF716FF7B697B6360E007F108031846AF
S3150802F5E0FEF778F83B697B6358E02D4BD3F8F03089
S3150802F5F003F00203022B03D14FF400437B634DE071
S3150802F60000237B634AE0264BD3F8F03003F000630D
S3150802F610B3F1006F03D14FF4FA437B633EE0002354
S3150802F6207B633BE01E4BD3F8E83003F04043FB62B2
S3150802F6301B4B1B6803F00203022B0CD1FB6A002B3F
S3150802F64009D1174B1B68DB0803F00303154A22FA94
S3150802F65003F37B631EE0124B1B6803F40073B3F5D6
S3150802F660007F06D1FB6AB3F1804F02D10E4B7B6352
S3150802F67010E00B4B1B6803F40033B3F5003F06D1C9
S3150802F680FB6AB3F1004F02D1084B7B6302E0002309
S3150802F6907B6303E002E000237B6300BF00F0CFBC7C
S3150802F6A0000C02440090D00300093D00001BB7007D
S3150802F6B09E4BD3F8DC3003F0E0433B633B6BB3F17C
S3150802F6C0A04F56D03B6BB3F1A04F00F28B803B6B39
S3150802F6D0B3F1804F3ED03B6BB3F1804F00F282808C
S3150802F6E03B6BB3F1405F27D03B6BB3F1405F79D8F0
S3150802F6F03B6BB3F1005F17D03B6BB3F1005F71D878
S3150802F7003B6B002B04D03B6BB3F1805F04D069E0FE
S3150802F710FBF734FD786368E007F114031846FDF732
S3150802F7206FFE7B697B6360E007F108031846FDF705
S3150802F730D1FF3B697B6358E07C4BD3F8F03003F08A
S3150802F7400203022B03D14FF400437B634DE00023EF
S3150802F7507B634AE0754BD3F8F03003F00063B3F1EC
S3150802F760006F03D14FF4FA437B633EE000237B63C9
S3150802F7703BE06E4BD3F8E83003F04043FB626B4B39
S3150802F7801B6803F00203022B0CD1FB6A002B09D17A
S3150802F790664B1B68DB0803F00303654A22FA03F388
S3150802F7A07B631EE0614B1B6803F40073B3F5007FAD
S3150802F7B006D1FB6AB3F1804F02D15E4B7B6310E040
S3150802F7C05A4B1B6803F40033B3F5003F06D1FB6AB4
S3150802F7D0B3F1004F02D1584B7B6302E000237B63EF
S3150802F7E003E002E000237B6300BF00F028BC4F4B16
S3150802F7F0D3F8E83003F440733B634C4B1B6803F4BD
S3150802F8000033B3F5003F06D13B6B002B03D14A4BBD
S3150802F8107B6300F014BC3B6BB3F5807F08D107F11C
S3150802F82020031846FDF782FC7B6A7B6300F007BC5F
S3150802F8303B6BB3F5007F07D107F114031846FDF7B2
S3150802F840DFFDBB697B63FAE300237B63F7E3374B90
S3150802F850D3F8E03003F007033B633B6B042B61D814
S3150802F86001A252F823F000BF7DF802088DF80208BB
S3150802F8709DF80208ADF80208B3F8020807F120035A
S3150802F8801846FDF753FC7B6A7B634EE007F11403C7
S3150802F8901846FDF7B5FD7B697B6346E007F1080369
S3150802F8A01846FDF717FFBB687B633EE0234B7B6375
S3150802F8B03BE01E4BD3F8E83003F04043FB621B4B98
S3150802F8C01B6803F00203022B0CD1FB6A002B09D139
S3150802F8D0164B1B68DB0803F00303154A22FA03F3E7
S3150802F8E07B631EE0114B1B6803F40073B3F5007FBC
S3150802F8F006D1FB6AB3F1804F02D10E4B7B6310E04F
S3150802F9000A4B1B6803F40033B3F5003F06D1FB6AC2
S3150802F910B3F1004F02D1084B7B6302E000237B63FD
S3150802F92003E002E000237B6300BF88E3000C024485
S3150802F9300090D00300093D00001BB7000080BB0001
S3150802F940A94BD3F8E03003F038033B633B6B202B1B
S3150802F95000F29A8001A252F823F000BFE1F90208E8
S3150802F96089FA020889FA020889FA020889FA020853
S3150802F97089FA020889FA020889FA0208F1F90208DC
S3150802F98089FA020889FA020889FA020889FA020833
S3150802F99089FA020889FA020889FA020801FA0208AB
S3150802F9A089FA020889FA020889FA020889FA020813
S3150802F9B089FA020889FA020889FA020811FA02087B
S3150802F9C089FA020889FA020889FA020889FA0208F3
S3150802F9D089FA020889FA020889FA020817FA020855
S3150802F9E007F120031846FDF7A1FB7B6A7B634EE00D
S3150802F9F007F114031846FDF703FD7B697B6346E0AE
S3150802FA0007F108031846FDF765FEBB687B633EE00F
S3150802FA10764B7B633BE0744BD3F8E83003F0404304
S3150802FA20FB62714B1B6803F00203022B0CD1FB6AC3
S3150802FA30002B09D16C4B1B68DB0803F003036C4AE5
S3150802FA4022FA03F37B631EE0674B1B6803F4007319
S3150802FA50B3F5007F06D1FB6AB3F1804F02D1654B3D
S3150802FA607B6310E0604B1B6803F40033B3F5003F79
S3150802FA7006D1FB6AB3F1004F02D15F4B7B6302E00A
S3150802FA8000237B6303E002E000237B6300BFD6E228
S3150802FA90554BD3F8E03003F4E0733B633B6BB3F5A5
S3150802FAA0807F31D03B6BB3F5807F66D83B6BC02B2A
S3150802FAB027D03B6BC02B60D83B6B802B19D03B6B96
S3150802FAC0802B5AD83B6B002B03D03B6B402B08D0BC
S3150802FAD053E007F120031846FDF728FB7B6A7B6390
S3150802FAE04EE007F114031846FDF78AFC7B697B632F
S3150802FAF046E007F108031846FDF7ECFDBB687B6391
S3150802FB003EE03A4B7B633BE0374BD3F8E83003F0F1
S3150802FB104043FB62344B1B6803F00203022B0CD1F1
S3150802FB20FB6A002B09D1304B1B68DB0803F0030381
S3150802FB302F4A22FA03F37B631EE02B4B1B6803F45E
S3150802FB400073B3F5007F06D1FB6AB3F1804F02D189
S3150802FB50284B7B6310E0244B1B6803F40033B3F590
S3150802FB60003F06D1FB6AB3F1004F02D1224B7B63F9
S3150802FB7002E000237B6303E002E000237B6300BF0D
S3150802FB805DE2194BD3F8E03003F460633B633B6BE9
S3150802FB90002B03D1FBF7DCFA786350E2124B1B68A1
S3150802FBA003F00063B3F1006F0BD13B6BB3F5007F33
S3150802FBB007D107F114031846FDF722FCBB697B63DC
S3150802FBC04FE0094B1B6803F00053B3F1005F15D1F0
S3150802FBD03B6BB3F5806F11D107F108031846FDF7A1
S3150802FBE079FDFB687B633CE0000C02440080BB00A5
S3150802FBF00090D00300093D00001BB700944B1B6818
S3150802FC0003F00203022B0DD13B6BB3F5C06F09D18A
S3150802FC108F4B1B68DB0803F003038E4A22FA03F3B1
S3150802FC207B631EE08A4B1B6803F40073B3F5007FFF
S3150802FC3006D13B6BB3F5006F02D1874B7B6310E0AD
S3150802FC40834B1B6803F40033B3F5003F06D13B6BC5
S3150802FC50B3F5206F02D1814B7B6302E000237B63FD
S3150802FC60EDE1ECE17A4BD3F8E03003F4E0433B6391
S3150802FC703B6B002B03D1FBF781FA7863DFE1744B08
S3150802FC801B6803F00063B3F1006F0BD13B6BB3F54E
S3150802FC90805F07D107F114031846FDF7B1FBBB696C
S3150802FCA07B6345E06A4B1B6803F00053B3F1005FC0
S3150802FCB00BD13B6BB3F5005F07D107F10803184672
S3150802FCC0FDF708FDFB687B6332E0614B1B6803F0B6
S3150802FCD00203022B0DD13B6BB3F5405F09D15C4B96
S3150802FCE01B68DB0803F003035A4A22FA03F37B6311
S3150802FCF01EE0574B1B6803F40073B3F5007F06D169
S3150802FD003B6BB3F5804F02D1534B7B6310E0504BEC
S3150802FD101B6803F40033B3F5003F06D13B6BB3F51A
S3150802FD20A04F02D14D4B7B6302E000237B6386E141
S3150802FD3085E1474BD3F8E03003F460333B633B6B12
S3150802FD40002B03D1FBF704FA786378E1404B1B6872
S3150802FD5003F00063B3F1006F0BD13B6BB3F5004FB1
S3150802FD6007D107F114031846FDF74AFBBB697B6303
S3150802FD7045E0374B1B6803F00053B3F1005F0BD124
S3150802FD803B6BB3F5803F07D107F108031846FDF729
S3150802FD90A1FCFB687B6332E02D4B1B6803F0020370
S3150802FDA0022B0DD13B6BB3F5C03F09D1284B1B681B
S3150802FDB0DB0803F00303274A22FA03F37B631EE0F8
S3150802FDC0234B1B6803F40073B3F5007F06D13B6B24
S3150802FDD0B3F5003F02D1204B7B6310E01C4B1B6836
S3150802FDE003F40033B3F5003F06D13B6BB3F5203F6E
S3150802FDF002D11A4B7B6302E000237B631FE11EE1FB
S3150802FE00134BD3F8E43003F003033B633B6B032B3A
S3150802FE105FD801A252F823F029FE020831FE020831
S3150802FE2041FE020861FE0208FBF760F9786353E0B7
S3150802FE3007F120031846FDF779F97B6A7B634BE0E5
S3150802FE4007F114031846FDF7DBFAFB697B6343E007
S3150802FE50000C02440090D00300093D00001BB700C5
S3150802FE60794BD3F8E83003F04043FB62764B1B68C4
S3150802FE7003F00203022B0CD1FB6A002B09D1724B49
S3150802FE801B68DB0803F00303704A22FA03F37B6359
S3150802FE901EE06D4B1B6803F40073B3F5007F06D1B1
S3150802FEA0FB6AB3F1804F02D1694B7B6310E0664B64
S3150802FEB01B6803F40033B3F5003F06D1FB6AB3F1BE
S3150802FEC0004F02D1634B7B6302E000237B6303E0AE
S3150802FED002E000237B6300BFB1E05B4BD3F8E83056
S3150802FEE003F0C0033B63584BD3F8F03003F0020328
S3150802FEF0022B06D13B6B002B03D14FF400437B63E5
S3150802FF001FE0514BD3F8F03003F00063B3F1006FF2
S3150802FF1006D13B6B402B03D14FF4FA437B6310E0C7
S3150802FF20494B1B6803F40073B3F5007F06D13B6B9C
S3150802FF30802B03D148F212037B6302E000237B6322
S3150802FF407DE07CE0404BD3F8E83003F030033B63B6
S3150802FF503D4B1B6803F40053B3F5005F05D13B6BB9
S3150802FF60002B02D13C4B7B6331E0374B1B6803F015
S3150802FF700073B3F1007F0AD13B6B102B07D107F14F
S3150802FF8020031846FDF7D2F87B6A7B631FE02E4BE7
S3150802FF90D3F8F03003F00203022B06D13B6B202B79
S3150802FFA003D14FF400437B6311E0274BD3F8F030BB
S3150802FFB003F00063B3F1006F06D13B6B302B03D11C
S3150802FFC04FF4FA437B6302E000237B6337E036E0B3
S3150802FFD01D4BD3F8E43003F030033B633B6B102B25
S3150802FFE007D107F120031846FDF7A0F87B6A7B6361
S3150802FFF025E0154B1B6803F00053B3F1005F0AD1E5
S315080300003B6B202B07D107F108031846FDF762FB64
S31508030010FB687B630FE00C4B1B6803F40053B3F5D3
S31508030020005F05D13B6B302B02D10B4B7B6302E0A0
S3150803003000237B6303E002E000237B6300BF7B6B43
S3150803004018463C37BD4690BD000C02440090D003C9
S3150803005000093D00001BB700006CDC0280B584B0C4
S3150803006000AF7860484B1B68474A23F080631360E8
S31508030070F8F782FAF86008E0F8F77EFA0246FB68B2
S31508030080D31A022B01D903237AE03F4B1B6803F0EB
S315080300900063002BF0D13C4BDB6A23F47C5323F03B
S315080300A003037A6811687A68526812020A43364962
S315080300B01343CB627B689B68013BC3F308027B68E7
S315080300C0DB68013B5B029BB21A437B681B69013BF6
S315080300D01B0403F4FE031A437B685B69013B1B0697
S315080300E003F0FE4328491343CB63274BDB6A23F00C
S315080300F00C027B689B6924491343CB62224BDB6A58
S3150803010023F020027B68DB691F491343CB621E4B2E
S31508030110DA6A7B685B6A1C491343CB621A4BDB6A50
S31508030120194A23F01003D362174B1B6C23F47F433E
S3150803013023F0F8037A68126AD200134913430B644F
S31508030140114BDB6A104A43F01003D3620E4B1B684C
S315080301500D4A43F080631360F8F70EFAF86008E077
S31508030160F8F70AFA0246FB68D31A022B01D90323C6
S3150803017006E0054B1B6803F00063002BF0D0002351
S3150803018018461037BD4680BD000C024480B584B0BE
S3150803019000AF7860484B1B68474A23F080531360C7
S315080301A0F8F7EAF9F86008E0F8F7E6F90246FB68B3
S315080301B0D31A022B01D903237AE03F4B1B6803F0BA
S315080301C00053002BF0D13C4B1B6B23F47C5323F0D9
S315080301D003037A6811687A68526812020A43364931
S315080301E013430B637B689B68013BC3F308027B6875
S315080301F0DB68013B5B029BB21A437B681B69013BC5
S315080302001B0403F4FE031A437B685B69013B1B0665
S3150803021003F0FE43284913434B64274B1B6B23F018
S315080302200C027B689B69244913430B63224B1B6BA4
S3150803023023F020027B68DB691F4913430B631E4BBC
S315080302401A6B7B685B6A1C4913430B631A4B1B6B5C
S31508030250194A23F010031363174B9B6C23F47F434C
S3150803026023F0F8037A68126AD200134913438B649E
S31508030270114B1B6B104A43F0100313630E4B1B6899
S315080302800D4A43F080531360F8F776F9F86008E0EF
S31508030290F8F772F90246FB68D31A022B01D903232E
S315080302A006E0054B1B6803F00053002BF0D0002330
S315080302B018461037BD4680BD000C024480B582B08F
S315080302C000AF78607B68002B01D1012349E07B6886
S315080302D093F83D30DBB2002B06D17B68002283F806
S315080302E03C20786800F041F87B68022283F83D20B9
S315080302F07B681A687B6804331946104600F0E4FDE8
S315080303007B68012283F848207B68012283F83E2014
S315080303107B68012283F83F207B68012283F840200B
S315080303207B68012283F841207B68012283F84220F7
S315080303307B68012283F843207B68012283F84420E3
S315080303407B68012283F845207B68012283F84620CF
S315080303507B68012283F847207B68012283F83D20C6
S31508030360002318460837BD4680BD80B483B000AF66
S31508030370786000BF0C37BD465DF8047B7047000004
S3150803038080B485B000AF78607B6893F83D30DBB204
S31508030390012B01D001237CE07B68022283F83D20F0
S315080303A07B681B68DA687B681B6842F00102DA60BF
S315080303B07B681B683A4A93424AD07B681B68394A6A
S315080303C0934245D07B681B68B3F1804F40D07B6866
S315080303D01B68B3F1A04F3BD07B681B68324A934234
S315080303E036D07B681B68314A934231D07B681B68D9
S315080303F02F4A93422CD07B681B682E4A934227D0F8
S315080304007B681B682C4A934222D07B681B682B4A5D
S3150803041093421DD07B681B68294A934218D07B6890
S315080304201B68284A934213D07B681B68264A934263
S315080304300ED07B681B68254A934209D07B681B68E4
S31508030440234A934204D07B681B68224A934215D1F8
S315080304507B681B689A68204B1340FB60FB68062B76
S3150803046015D0FB68B3F5803F11D07B681B681A6803
S315080304707B681B6842F001021A6008E07B681B6808
S315080304801A687B681B6842F001021A6000E000BF25
S31508030490002318461437BD465DF8047B704700BF32
S315080304A0002C0140002C01500004004000040050B9
S315080304B00008004000080050000C0040000C0050E3
S315080304C00034014000340150001800400018005061
S315080304D000400140004001500700010080B582B08A
S315080304E000AF78607B68002B01D1012349E07B6864
S315080304F093F83D30DBB2002B06D17B68002283F8E4
S315080305003C207868F6F770F87B68022283F83D206A
S315080305107B681A687B6804331946104600F0D4FCD6
S315080305207B68012283F848207B68012283F83E20F2
S315080305307B68012283F83F207B68012283F84020E9
S315080305407B68012283F841207B68012283F84220D5
S315080305507B68012283F843207B68012283F84420C1
S315080305607B68012283F845207B68012283F84620AD
S315080305707B68012283F847207B68012283F83D20A4
S31508030580002318460837BD4680BD000080B584B0F1
S3150803059000AF786039603B68002B09D17B6893F814
S315080305A03E30DBB2012B14BF01230023DBB23CE050
S315080305B03B68042B09D17B6893F83F30DBB2012BE8
S315080305C014BF01230023DBB22FE03B68082B09D1B4
S315080305D07B6893F84030DBB2012B14BF0123002359
S315080305E0DBB222E03B680C2B09D17B6893F84130D8
S315080305F0DBB2012B14BF01230023DBB215E03B68F2
S31508030600102B09D17B6893F84230DBB2012B14BF58
S3150803061001230023DBB208E07B6893F84330DBB29F
S31508030620012B14BF01230023DBB2002B01D00123C6
S31508030630E2E03B68002B04D17B68022283F83E2064
S3150803064023E03B68042B04D17B68022283F83F200E
S315080306501BE03B68082B04D17B68022283F8402001
S3150803066013E03B680C2B04D17B68022283F84120F4
S315080306700BE03B68102B04D17B68022283F84220E7
S3150803068003E07B68022283F843207B681B68012208
S315080306903968184601F00CF97B681B68584A934277
S315080306A02CD07B681B68574A934227D07B681B6804
S315080306B0554A934222D07B681B68544A93421DD0FD
S315080306C07B681B68524A934218D07B681B68514A59
S315080306D0934213D07B681B684F4A93420ED07B68BC
S315080306E01B684E4A934209D07B681B684C4A93425F
S315080306F004D07B681B684B4A934201D1012300E06F
S315080307000023002B07D07B681B685A6C7B681B6821
S3150803071042F400425A647B681B68394A93424AD0BA
S315080307207B681B68374A934245D07B681B68B3F1DD
S31508030730804F40D07B681B68B3F1A04F3BD07B68E2
S315080307401B68394A934236D07B681B68374A9342FB
S3150803075031D07B681B68364A93422CD07B681B686A
S31508030760344A934227D07B681B68334A934222D084
S315080307707B681B68314A93421DD07B681B68224AF3
S31508030780934218D07B681B68204A934213D07B6830
S315080307901B682B4A93420ED07B681B68294A9342EF
S315080307A009D07B681B681A4A934204D07B681B6886
S315080307B0184A934215D17B681B689A68224B1340E3
S315080307C0FB60FB68062B15D0FB68B3F5803F11D099
S315080307D07B681B681A687B681B6842F001021A600B
S315080307E008E07B681B681A687B681B6842F001028D
S315080307F01A6000E000BF002318461037BD4680BDC7
S31508030800002C0140002C01500034014000340150F3
S31508030810004001400040015000440140004401509B
S3150803082000480140004801500004004000040050FD
S315080308300008004000080050000C0040000C00505F
S3150803084000180040001800500700010080B582B068
S3150803085000AF786039607B681B68002239681846E0
S3150803086001F026F87B681B684A4A93422CD07B68BA
S315080308701B68494A934227D07B681B68474A9342B9
S3150803088022D07B681B68464A93421DD07B681B6847
S31508030890444A934218D07B681B68434A934213D051
S315080308A07B681B68414A93420ED07B681B68404AA3
S315080308B0934209D07B681B683E4A934204D07B68FF
S315080308C01B683D4A934201D1012300E00023002B14
S315080308D017D07B681B681A6A41F211131340002B61
S315080308E00FD17B681B681A6A44F244431340002BF2
S315080308F007D17B681B685A6C7B681B6822F4004225
S315080309005A647B681B681A6A41F211131340002B59
S315080309100FD17B681B681A6A44F244431340002BC1
S3150803092007D17B681B681A687B681B6822F001027B
S315080309301A603B68002B04D17B68012283F83E20AA
S3150803094023E03B68042B04D17B68012283F83F200C
S315080309501BE03B68082B04D17B68012283F84020FF
S3150803096013E03B680C2B04D17B68012283F84120F2
S315080309700BE03B68102B04D17B68012283F84220E5
S3150803098003E07B68012283F84320002318460837CF
S31508030990BD4680BD002C0140002C015000340140A7
S315080309A0003401500040014000400150004401401A
S315080309B000440150004801400048015080B584B006
S315080309C000AF78607B681B68DB68FB607B681B6825
